S00A000047572E737265637C
S214400000A55AA55A0100000000000000001040005C
S21440100000F042202114440025504500275045005A
S214401010295045002B5045002D504500000000004B
S2144010200000000000000000000000002F504500B7
S214401030635045000000000065504500675045007D
S21444010047573334342056302E322E352032303250
S214440110332E31312E362031323A30300A0D00003B
S20C4401803412AA5500000000E9
S214440200A55AA55A01000000000000000010440052
S2144402100000000000104400000000000000000041
S2144402200000000000000000000000000000000085
S2144402300000000000000000000000000000000075
S2144402400000000000000000000000000000000065
S2144402500000000000000000000000000000000055
S21444100000F0422021144400255045002750450056
S214441010295045002B5045002D5045000000000047
S2144410200000000000000000000000002F504500B3
S2144410306350450000000000655045006750450079
S214441040695045006950450069504500695045005F
S214441050695045006950450069504500695045004F
S214441060695045006950450069504500695045003F
S214441070695045006950450069504500695045002F
S214441400695045006950450000BF00BF00BF00BF9B
S214441410FFF7FABF000000000000000000000000D4
S21444142072B64FF000004FF000014FF000024FF04C
S21444143000034FF000044FF000054FF000064FF055
S21444144000074F4801684FF0807201EA0201002904
S2144414501CD14C4801684FF0807241EA0201016099
S214441460494801684FF0010241EA020101604748D9
S21444147045F6F02101604AF20F5101604048016888
S2144414804FF0807201EA02010029F7D040484149F2
S2144414900160414801684FF00000814200D003E0FB
S2144414A03E4880F3088803E03D4880F3088822E0FD
S2144414B03C484CF2205101604DF6281101603A48F0
S2144414C03A4901600AE03A484CF2205101604DF630
S2144414D028110160374835490160FFE7364800283F
S2144414E009D03649364A521A013A04DD0020002310
S2144414F009C1083AFCDA3348002810D03249086853
S2144415004FF0010240EA020008603049304A521A5D
S214441510013A04DD0020002309C1083AFCDA2D48CC
S214441520002810D02C4908684FF0010240EA020017
S21444153008602A492A4A521A013A04DD0020002348
S21444154009C1083AFCDA274800684FF05A31884205
S214441550F9D0114801684FF00000814200D001E004
S21444156013F084FD13F0AEFD62B613F0A9FD00F04F
S2144415703BF800BFFEE700BFAFF30080AFF3008048
S21444158010C32D4030C32D4004C32D4000C02D4011
S21444159008ED00E0001043200400264000F04220FE
S2144415A0000043201000274000002740400000FF72
S2144415B010C0464000C046400100000000004020E5
S2144415C0004044200100000094EF00E000000020AA
S2144415D0000001200100000090EF00E00000000041
S2144415E000800000E42440202DE9F04F87B05B4C97
S2144415F001F072FC5A4815F087FA5A494E200025E5
S21444160025F032FC58481CF00FFC58481CF030FCBF
S21444161001F0D5FB4CF24453E05800F017F901F0C2
S21444162011FE00F03BFA00F017FA00F095F9504925
S21444163000201FF075FD4F4900201FF087FD002154
S21444164008461FF02DFE002144F6206208461FF08F
S214441650E3FD2846013501F06FFF062DF9D101F070
S214441660ABFB4CF23853444D4FF47A7054F8038035
S214441670E75805F1040BE25854F803900592E258F3
S2144416800292E2580392E2580492E25854F803A0B5
S214441690E6582C46019201F056FB08F03DFA3748CE
S2144416A001F082FC00F0B4F82A6806F57A739A4290
S2144416B002D32E6808F01FFA22680AF1C8039A4239
S2144416C003D3D4F800A008F00FFA019B22686433D1
S2144416D09A4203D32368019308F0F3F9049B2268E3
S2144416E032339A4201D323680493039B226814330B
S2144416F09A4203D32368039303F0F9FB029B2268C0
S2144417000A339A4203D32368029308F09EF9226868
S21444171009F105039A4203D3D4F8009008F013F96C
S214441720059B226802339A4203D32368059300F04C
S21444173070F822687B1C9A4200D32768DBF80020A6
S21444174008F101039A4203D3DBF8008008F0A8F9B5
S21444175008F0E8F90CF00EFFA6E700BF6C484120FD
S21444176090894600E8034020D496460004924600FA
S2144417707417402068174020A40D4220F47F46008A
S214441780024B586800F00300704700BF0000264034
S214441790024600F03F00931010B583EA5203540803
S2144417A0534084EA121483EA121384EAD2049B0157
S2144417B084EA521403F0400314F0010F43EA000392
S2144417C00CBF80240024234319B99A4218BFFF2033
S2144417D010BD01290CBF1846FF20F9E73C2A0CD05F
S2144417E07D2A0AD0FE2A08D0BF2A06D092B20144E7
S2144417F0814204D1D043C0B270470022F7E710F8C4
S214441800013B1A4492B2FF2A84BFFF3A92B2EFE7F2
S21444181070470AF03FBF704710B5074C002001F0F0
S214441820F5F92080012001F0F1F9044B2288188054
S214441830034B1A8010BD00BF361840203418402091
S214441840E01740207047704770477047002110B536
S2144418500446084618F012FB0121002018F00EFB3F
S2144418600221002018F00AFB0321002018F006FB92
S214441870002018F0FFF90E49002018F011F90D4B1E
S214441880A2B20020197818F049FA0B49002018F043
S214441890BBFD0A49002018F0B7FD0949002018F09E
S2144418A0B3FD08490020BDE8104018F0ADBD00BFA8
S2144418B04C8E4600848E4600D48F4600B48F460035
S2144418C0948F4600748F4600F8B50D4606461F4969
S2144418D028461F4F0EF0A0F8044670B14CF244530D
S2144418E0F85806F54553123307EB83077D60032EFD
S2144418F02BD8DFE806F01A212427002128460EF0CC
S21444190081F880B94CF24453F8580DF07BFE2946D2
S2144419100DF0D0FE0DF020FA00220E4B0DF09EFB8B
S2144419200DF04AFDDDE72046DBE782B200210020C9
S214441930BDE8F84018F0B2BF82B20121F7E782B2A0
S2144419400221F4E782B20321F1E7F8BD0000C84261
S2144419506C4841200000594008B503481DF056FC29
S214441960024B187008BD00BFCC994600AC474020D7
S214441970F7B50123104C114D6370A21CEB68A91CEB
S2144419800F480235009335F8023C1DF0E1FA002278
S2144419902073A01C6178134615F8017B013310F8B8
S2144419A0016BDBB2B7421CBF012200210A2BF3D1E4
S2144419B002B1617003B0F0BDAC474020A01F402088
S2144419C0E09946004B7C062B0AD10122054B1A743B
S2144419D0CA7B1A2A04D1032203F111011DF0F8BD73
S2144419E0704700BFA01F40204B7C062B0AD1012223
S2144419F0054B1A74CA7B2A2A04D1032203F1110127
S214441A001DF0E6BD704700BFA01F40201FB5002351
S214441A101A210446039301238DF807301DF01EFF58
S214441A200B4B03930B4B1A7C002AFCD01B7C63B1F4
S214441A3002A920461DF016FE8DF80700039B5A1E89
S214441A40039213B19DF80730F1E704B010BD00BF10
S214441A50006A1800A01F402008B5A1201CF02AFAEE
S214441A6000220A49A1201CF024FA094B0949022203
S214441A700120C3F8F413C3F8982DC3F8F813C3F839
S214441A80902D0549BDE808401CF014BFABEC45005A
S214441A9000002940040028004099460008B5A220CA
S214441AA01CF008FA00220B49A2201CF002FA0A4B4A
S214441AB00A4A01210020C3F8E023C3F8AC1DC3F84A
S214441AC0E42302220649C3F8A42DBDE808401CF0CE
S214441AD031BC00BFB1EC450000002940020028009C
S214441AE06499460010B50822174901204FF4803403
S214441AF01CF09CFF01230822144900201CF006FD1C
S214441B00002108461CF050FE022801D1013CF7D1C2
S214441B104FF48034002101201CF092FF022801D1AA
S214441B20013CF7D1094A0823A2F1080012F8011B28
S214441B30013B10F8014BA14204BF013102F8011CDD
S214441B4013F0FF03F2D110BDB41F4020BC1F402049
S214441B5082B00190019B5A1E0192002BFAD102B02A
S214441B607047044B4FF400224FF4FA70C3F8C02277
S214441B70FFF7EEBF00002940044B4FF420124FF409
S214441B80FA70C3F8C022FFF7E3BF00BF0000294045
S214441B902DE9F04104460D46104600293ED1DFF8B3
S214441BA0908050260B46C1B2564308F1100728468B
S214441BB0BA19B04419F082FE1C484FF4FB534FF454
S214441BC0FB62D8F81410083603FB04033744D3F8F2
S214441BD0FC3802FB043203F17A0602F5107C02F567
S214441BE0427240F82C1098F8581040F82210FB2205
S214441BF012FB046200EB4212A94211D84FF4FB5286
S214441C000133642102FB0404B3FBF1F201FB1233FB
S214441C10C4F8FC3804F5215401232360BDE8F08160
S214441C2017F8016B013502F8016BE5E76C48412073
S214441C30AC4740202DE9F04104460D4610460029A5
S214441C403ED1DFF8908050260B46C1B2564308F585
S214441C5021670120BA19B04419F030FE1C484FF4ED
S214441C60FB534FF4FB62D8F8141A083603FB0403FC
S214441C703744D3F8FC3802FB043203F17A0602F503
S214441C80107C02F5427240F82C1098F8581A40F826
S214441C902210FB2212FB046200EB4212A94211D826
S214441CA04FF4FB520133642102FB0404B3FBF1F20C
S214441CB001FB1233C4F8FC3804F521540123236095
S214441CC0BDE8F08117F8016B013502F8016BE5E7D2
S214441CD06C484120AC4740202DE9F04104460D466F
S214441CE0104600293ED1DFF8908050260B46C1B2FC
S214441CF0564308F546770220BA19B04419F0DEFD7B
S214441D001C484FF4FB534FF4FB62D8F81C130836B8
S214441D1003FB04033744D3F8FC3802FB043203F1D4
S214441D207A0602F5107C02F5427240F82C1098F8B8
S214441D30601340F82210FB2212FB046200EB4212AE
S214441D40A94211D84FF4FB520133642102FB040428
S214441D50B3FBF1F201FB1233C4F8FC3804F521540A
S214441D6001232360BDE8F08117F8016B013502F8C2
S214441D70016BE5E76C484120A45840202DE9F0412A
S214441D8004460D46104600293ED1DFF89080502682
S214441D900B46C1B2564308F618570320BA19B04446
S214441DA019F08CFD1C484FF4FB534FF4FB62D8F8F3
S214441DB01C1D083603FB04033744D3F8FC3802FBE7
S214441DC0043203F17A0602F5107C02F5427240F8BA
S214441DD02C1098F8601D40F82210FB2212FB046277
S214441DE000EB4212A94211D84FF4FB52013364214E
S214441DF002FB0404B3FBF1F201FB1233C4F8FC38D3
S214441E0004F5215401232360BDE8F08117F8016BE3
S214441E10013502F8016BE5E76C484120A4584020A0
S214441E202DE9F04104460D46104600293ED1DFF820
S214441E30908050260B46C1B2564308F5C46704202A
S214441E40BA19B04419F03AFD1C484FF4FB534FF40A
S214441E50FB62D8F82416083603FB04033744D3F849
S214441E60FC3802FB043203F17A0602F5107C02F5D4
S214441E70427240F82C1098F8681640F82210FB225C
S214441E8012FB046200EB4212A94211D84FF4FB52F3
S214441E900133642102FB0404B3FBF1F201FB123369
S214441EA0C4F8FC3804F5215401232360BDE8F081CE
S214441EB017F8016B013502F8016BE5E76C484120E1
S214441EC09C6940202DE9F04104460D461046002901
S214441ED03ED1DFF8908050260B46C1B25643A8F157
S214441EE0D8070520BA19B04419F0E8FC1C484FF44A
S214441EF0FB534FF4FB6258F8D41C083603FB040328
S214441F003744D3F8FC3802FB043203F17A0602F570
S214441F10107C02F5427240F82C1018F8901C40F8D9
S214441F202210FB2212FB046200EB4212A94211D893
S214441F304FF4FB520133642102FB0404B3FBF1F279
S214441F4001FB1233C4F8FC3804F521540123236002
S214441F50BDE8F08117F8016B013502F8016BE5E73F
S214441F606C484120947A40204FF4FB52054B02FBC8
S214441F700033D3F8F808D3F8FC38C31A584258410B
S214441F80704700BF6C4841202DE9F74FCC4D0021E7
S214441F90CC4E4FF4FB692C4641F6987837464FF0C2
S214441FA0640A0846FFF7E0FF50BBD6F8F83809FB4A
S214441FB0013202F5427257F822C008FB01420092F1
S214441FC04FF4FB524A4302EB43123A44019200F167
S214441FD0010EC0B2844534D809FB0132013385F87A
S214441FE020C002F5107257F822206A624FF00102B0
S214441FF085F82120B3FBFAF20AFB1233C6F8F83808
S2144420000131454406F5FB560629CAD194F82130D9
S214442010012B2DD1002384F82130636AB3F5BE7FAB
S21444202000F0E18000F29480452B14D83F2B1FD952
S214442030413B042B00F2CB80DFE803F0CCDEE1E446
S214442040E700019A02EB000B009A9BF840BF02F8A7
S21444205000B07046BBE7B3F5BA7F00F0BE80B3F578
S214442060BC7F00F0BD8040F25512934200F0BE8023
S21444207041F6B973E25C012A0FD10022E25441F6DC
S214442080BC73E358932B00F0D08000F2C180912BB0
S21444209000F0C580922B00F0C58043F65173E25C95
S2144420A0012A14D10022E25443F65473E358962B83
S2144420B000F0E38000F2C480822B00F0DB8000F264
S2144420C0B780722B00F0DF80732B00F0DF8045F67C
S2144420D0E963E25C012A14D10022E25445F6EC633B
S2144420E0E3589B2B00F0F88000F2DE808D2B00F046
S2144420F0028100F2D180722B00F0F780732B00F03F
S214442100F78047F68163E25C012A0BD10022E25451
S21444211047F68463E358722B00F0F380732B01D1A7
S21444212002F0A8FD49F61963E25C012A40F0F1800A
S2144421300022E25449F61C63E358722B00F0E48014
S214442140732B40F0E68003B0BDE8F04F02F0C2BD0A
S214442150B3F5B06F2FD016D840F20132934233D045
S2144421600AD840F22122934243D0B3F5407F7FF40D
S2144421707FAF01F0DBFD7BE7B3F5AE6F7FF478AF5E
S21444218001F000FE74E740F29552934216D00AD806
S21444219040F28552934214D0B3F5B26F7FF468AFE1
S2144421A001F0B2FE64E740F2777293427FF460AF88
S2144421B001F0D4FE5CE701F035FE59E701F0B6FEC7
S2144421C056E701F079FE53E701F0D0FD50E701F001
S2144421D054FC4DE701F064FC4AE701F0E5FC47E7B0
S2144421E001F004FD44E701F023FD41E701F0B4FCAF
S2144421F03EE701F03BFD3BE701F070FC38E701F0B9
S21444220079FC35E701F086FC32E701F093FC2FE7D2
S214442210B3F5A87F7FF441AF01F008FF3DE701F036
S214442220AFFE3AE701F0D2FE37E701F0E1FE34E7CD
S2144422308C2B25D0922B7FF44AAF02F059F846E710
S214442240AA2B26D007D89A2B0ED0A02B7FF43FAFCC
S21444225002F06EF93BE7C82B09D0B3F5F36F7FF471
S21444226036AF02F02FFA32E702F022F92FE702F0F7
S214442270EBF92CE701F0AAFF29E702F0C1F826E7BC
S21444228001F0CEFF23E701F027FF20E701F06CFFC3
S2144422901DE702F099F91AE7932B2FD0972B7FF47A
S2144422A030AF02F0FFFA2CE7C92B18D00CD8A12B7C
S2144422B018D0AA2B7FF425AF02F0C4FB21E700BF59
S2144422C0488740206C48412040F2997293427FF4FC
S2144422D018AF02F09DFC14E702F03CFB11E702F055
S2144422E0F1FB0EE702F076FB0BE702F0FFF908E796
S2144422F002F044FA05E702F023FC02E702F070FA23
S214442300FFE602F099FC0DE703B0BDE8F04F02F09B
S214442310C3BC03B0BDE8F08FEC4BED489A6D596FE3
S21444232002F07042DFF8CCC301F07F412DE9F0475C
S214442330E84F4FF000089A654FF00009DA6D596788
S2144423403A40996FE44EDA6501401A6E996702F096
S2144423500042996C5C691A6601F06041B3F86420E7
S21444236041F4C821DFF890E33240DFF890A3996443
S214442370A3F86420B3F86820D8493240A3F868200C
S2144423800022C3E90212D64983F86F2021405C6CD0
S2144423901A675961596A5A6539405962196C01F08D
S2144423A000411964CF490C405C64CF4CC3E91342E6
S2144423B0D3F88040D3F8985004F07F4483F88C20B8
S2144423C0C3F8D4E0C3F88040D3F8844004F07F4494
S2144423D0C3E92142B3F8904004EA0C04A3F89040C1
S2144423E0D3F8904062F35034C3F89040D3F8944006
S2144423F004F07C44C3F89440BC4C2540C3F8985041
S214442400D3F8D85005F04045C3F8D850D3F8DC503C
S21444241005F07845C3E9375293F8E45062F3000573
S21444242083F8E450D3F8AC5005F04045C3F8AC50BC
S214442430B3F8B05062F30D05A3F8B050D3F8C050CB
S21444244005F00045C3F8C050B3F8C4503540A3F86F
S214442450C450D3F8C45025F47F15C3F8C450D3F8F9
S214442460C850C3F838E105F07045C3F8C850D3F8EF
S214442470CC5005F07F45C3F8CC50B3F8D05005EAAD
S2144424800A05A3F8D050D3F8B45005F04045C3E944
S2144424902D5293F8BC5025F0030583F8BC50D3F86E
S2144424A09C5005F04045C3F89C50D3F8A0500D40CE
S2144424B0C3E92852D3F8A8500540C3F8A850D3F827
S2144424C0E85005F07E4545F48035C3F8E850D3F827
S2144424D0EC500D40C3F8EC50D3F83C512540C3F8BB
S2144424E03C51D3F8405105F07845C3F84051B3F811
S2144424F0445105F47845C3E94022C3E93E89A3F82C
S2144425004451D3F8485183F8542105F07E45C3F826
S2144425101C21A3F8282145F48035C3F84851D3F844
S2144425204C510D40C3F84C51D3F8505105F060451A
S214442530C3F85051D3F82C5105F07045C3F82C51CC
S214442540D3F8305105F07F45C3F83051B3F83451D1
S21444255005EA0A0AD3F8085105F04045A3F834A121
S214442560C3F80851D3F80C512940614DC3E94312CE
S214442570D3F814110140C3F81411D3F8181101F01C
S2144425807C41C3F81811090E21F03C0183F81B1155
S21444259093F8201121F0030183F82011D3F8241175
S2144425A001F06041C3F82411D3F868113940C3E9F7
S2144425B05689C3F86811A3F86C21D3F87011A3F8B0
S2144425C074210F40D3F8C811C3F8B02101F07C4100
S2144425D083F8B421C3F8B821C3F8C811D3F8CC1192
S2144425E083F8BC212140C3F8C02183F8C421C3F832
S2144425F0CC11D3F8D411C3F8782101F0004183F804
S2144426008021C3F8A021C3F87071C3E97512D3F8CA
S2144426107C1101F07F41C3F87C11D3F88411294022
S214442620C3E9611293F88C1121F00F01C3E97822B3
S21444263083F88C11C3E96422C3E96622A3F8A42173
S21444264093F81012C3F8A82162F30101A3F8AC2151
S21444265083F8142283F81012D3F81012C3F82022F9
S21444266021F07F6183F83822C3F83C2221F47F218D
S21444267083F84022C3F8442221F47F6183F8482239
S214442680C3F84C2221F00C0183F85022C3F854229C
S214442690C3F81012D3F8181283F8622201F00041EE
S2144426A0C3F81812B3F81C120E40D3F8241201F0E3
S2144426B07F41A3F81C62C3F82412D3F828120140C1
S2144426C0C3F82812D3F830121AE000BFC083402063
S2144426D00000FCFF0000F0FF00C0FFFF0000E281A6
S2144426E000F807F8000080FF0080204E0000C0FF7E
S2144426F00000FEFF00E0FFFF0000C04B00F0FFFFBD
S2144427002140C3E98C12D3F858120C40D3F85C121B
S21444271001F07E41C3F85842C3F85C1293F8A41201
S214442720A3F8EC2221F01F01C3F8F02241F0010186
S21444273083F8A412B3F8A81262F30901A3F8A81206
S21444274093F8AC1221F00F0183F8AC1293F8B01250
S21444275062F3020183F8B01293F8B41262F30301F1
S21444276083F8B412D3F8B81201F07E41C3F8B81215
S214442770D3F8BC1201F00041C3F8BC1293F8C0125F
S21444278021F00F0183F8C012D3F8C41201F0784147
S214442790C3F8C412D3F8C81201F07F41C3F8C81274
S2144427A0B3F8CC1201EA0C01A3F8CC12D3F8D01239
S2144427B02940C3F8D012B3F8E81201F40041A3F854
S2144427C0E812D3F8E81221F0FF4121F4FF01C3F8E0
S2144427D0E81293F8F41262F30001C3E9B68983F869
S2144427E0F412D3F8F81201F07F41C3F8F812D3F884
S2144427F0FC120140C3F8FC12D3F8001301F0404128
S214442800C3F80013D3F8041301F07841C3F8041353
S214442810D3F8081301F07841C3E9C21293F81013B1
S21444282062F3000183F81013D3F8141301F07841CF
S214442830C3F81413D3F8181301F07F41C3F81813E0
S214442840B3F81C1301EA0C0CD3F8201301F07E41B4
S214442850A3F81CC3C3F82013D3F824132940C3E9B0
S214442860C91293F82C1362F3000183F82C13D3F89F
S214442870301301F07F41C3F83013D3F834130840C3
S214442880D3F838130D40C3F83403C3F83853C3E9B8
S214442890D089D3F85013C3F8642301F04041C3F8F9
S2144428A07423C3F85013D3F8541301F07841C3F893
S2144428B05413D3F8581301F07841C3E9D61293F869
S2144428C0601362F3000183F8601393F8681362F3AD
S2144428D0000183F86813D3F86C1301F07F41C3F802
S2144428E06C1393F8721321F0030183F8721393F870
S2144428F0781362F3000193F87E2322F0030283F8F0
S214442900781383F87E23BDE8F08741F69873084928
S214442910002258430B182830DA64084483F84820C9
S2144429202023013B00F8012B13F0FF03F9D1704735
S2144429304887402041F6987310B558430B4C41F6EF
S21444294092732218D35A28225A430023111850301F
S214442950104421441A46204481F870304B670133B2
S21444296000F8012BDBB2202BF9D110BD488740205C
S2144429702DE9F8439946234B0546884603EB001356
S2144429809B6A402B31D820494FF4FB5303FB00137A
S21444299042F644015B5843B341F698761B4C0027F5
S2144429A04FF0280C06FB00F3E11801F5FC511031FA
S2144429B0F8B248451BD328467543FFF7A6FF41F6B1
S2144429C09071601928260122435A06FB0355134486
S2144429D02C4484F87120C4F8748084F87090C82419
S2144429E0B3FBF4F204FB12334352BDE8F883088881
S2144429F012F807E00CFB003020443844013780F8D6
S214442A0050E0D5E7A01F40206C484120488740202E
S214442A1041F6987241F692732DE9F34102FB00F1B8
S214442A204E4D04466A18D05A282202FB00122A4405
S214442A3092F87020082A31D8494B082203EB041335
S214442A409A62282341F6947603FB00F241F6987383
S214442A5020466343D118EF18503329441344414A5F
S214442A602B4402EB041200934B6FB95D18F0AEFE94
S214442A70012C80462FD143F62C711C206B5C01330D
S214442A80B3FBF0F200FB12336B54B8F1000F2BD0BB
S214442A90B8F1020F40D002B0BDE8F081102A04D845
S214442AA02F4B102203EB0413CAE7182A05D82C49E7
S214442AB0182301EB04118B62C3E7202A04D8284963
S214442AC0202301EB0411F6E7402ABAD824494023D0
S214442AD001EB0411EFE7BB5D0E210133B3FBF1F2CA
S214442AE001FB1233BB55D0E72046FFF723FF41F6E0
S214442AF0987041F69271604328242E18735A04FB4A
S214442B0003040133C8202544B3FBF0F200FB123320
S214442B1085F871807352BEE72046FFF70BFF41F6F7
S214442B20987041F692710022444328202E19735A15
S214442B3000FB03440133C820254485F87120B3FBC9
S214442B40F0F200FB1233064A7352D2E922310133C3
S214442B5041F10001C2E922319DE700BF4887402089
S214442B60A01F4020C41F4020F8B500240A4D41F65B
S214442B7098760A4F06FB04F22821E0B2D35B01FBA9
S214442B8003232B4493F87130012B01D1FFF740FF08
S214442B900134062CEED1F8BD48874020DAA6402002
S214442BA008B50B21034824F0A7F8034B83F82809FB
S214442BB008BD00BF02172940947A402001290A46DE
S214442BC028BF0122072819D8DFE800F004070B0DB8
S214442BD01012141600210A4801E00A21094824F07C
S214442BE052B80C21F7E702210748F8E70D21F2E72F
S214442BF00E21F0E70F21EEE70021F5E7704700BF0E
S214442C0002172940101729400017294007281AD8C8
S214442C10DFE800F004070B0E1013151708210B48C5
S214442C2001E00B210A4824F067B801210948FAE775
S214442C300B21F4E704210848F5E70521FBE70821C2
S214442C40F9E70A21F7E7FF20704700BF0617294037
S214442C5002172940121729400417294001284FF02B
S214442C6002010CBF0022012210B50446034824F09A
S214442C700AF8034A4CF24053D45010BD0817294072
S214442C806C48412005281DD8DFE800F003080C10E6
S214442C9014180D4A4CF27453D05A70470A4A4CF2F0
S214442CA07653F9E7084A4CF27853F5E7064A4CF26D
S214442CB07A53F1E7044A4CF27C53EDE7024A4CF26D
S214442CC07E53E9E7FF2070476C48412008B506214B
S214442CD0002012F058FD024A4CF27453D05208BDFC
S214442CE06C48412010B50221012012F04CFD064CE0
S214442CF04CF276532B21E052012012F044FD4CF264
S214442D007E53E05210BD00BF6C48412010B50321ED
S214442D10022012F038FD094C4CF278530421E0525C
S214442D20022012F030FD4CF27A530521E052022084
S214442D3012F029FD4CF27C53E05210BD6C48412001
S214442D40002112F00DBC084A4CF2385382B00749B1
S214442D50D35800930B68009A9B1A0193019B8342B5
S214442D60F8D902B0704700BF6C484120A40D4220F9
S214442D7038B50F4D0F4C95F890305BB901234CF2A3
S214442D803C5285F89030A3580133A350BDE83840F0
S214442D9006F086BE0AF0A6F94CF23C52002385F8AB
S214442DA09030A3580133A3504CF23852EBE700BF9F
S214442DB0A01F40206C4841200020FFF74FBF10B5AD
S214442DC08D20244C1BF076F8002223498D201BF0DE
S214442DD070F88F201BF06EF8002220498F201BF0DD
S214442DE068F897201BF066F800221D4997201BF0D0
S214442DF060F89A201BF05EF800221A499A201BF0CD
S214442E0058F8194900201DF09DFB184902201DF072
S214442E1099FB17490A201DF095FB16490D201DF015
S214442E2091FB2146012200201DF00EFE04F596710A
S214442E30012202201DF008FE04F26C5101220A20F1
S214442E401DF002FE04F28C5101220D20BDE8104014
S214442E501DF0FABD784B4120510F4600570F4600EF
S214442E605D0F4600630F4600CC9A4600A09A460083
S214442E70749A4600489A460010B48AB90949D1F86B
S214442E806C3891F8B848CA18013301F6B801DBB279
S214442E9082F8584610BC012241F84C3C1DF024BF31
S214442EA010BC70476C48412010B48AB90949D1F81F
S214442EB0743891F8D848CA18013301F6D801DBB201
S214442EC082F8584710BC012241F8643C1DF00CBF00
S214442ED010BC70476C484120194B012142F644000F
S214442EE00022195044F2A470195046F20470195046
S214442EF048F2646019504AF2C45019504CF22450B7
S214442F00195042F648015A5044F2A8715A5046F2B3
S214442F1008715A5048F268615A504AF2C8515A5099
S214442F204CF22851C3E9C1225A504CF248524CF252
S214442F30503199504CF244524FF44861995070477E
S214442F406C48412010B5064B4FF4FB5404FB00304C
S214442F5042F64803C15042F64C03C25010BD00BF6F
S214442F606C484120094BD3E9C1218A420BD01A440C
S214442F7092F8042202700020D3F804230132D2B21D
S214442F80C3F8042370470120704700BF6C484120B3
S214442F9007B501220DF107018DF8070000201DF04A
S214442FA0A7FB03B05DF804FB0FB470B5C2B00024B1
S214442FB046AA02AE52F8041B304601920EF04CFC70
S214442FC030460BF009FDC5B2E3B29D4204D842B088
S214442FD0BDE8704004B07047305D0134FFF7D8FF59
S214442FE0F2E708B58E201AF065FF96201AF062FFC5
S214442FF00748FFF7D9FF074900201CF023FA0120B1
S21444300005491CF01FFA0548BDE80840FFF7CCBF49
S214443010487E46001C9A4600F0994600507E46007C
S2144430200B2938B5044614D142F644030E4D00220B
S2144430300E48EA50FFF7B8FF42F64803EB581BB178
S21444304042F64C02A85898472046BDE8384019F046
S21444305033B9074B1A6832B1002206481A60BDE8F5
S2144430603840FFF7A1BF38BD6C484120567E460025
S214443070AC704120727E46000B2938B505460E4C8E
S21444308013D144F2A47300220C48E250FFF78CFF9D
S21444309044F2A873E3581BB144F2AC72A058984764
S2144430A02846BDE8384019F007B944F2A073E25800
S2144430B00AB10022E25038BD6C484120917E460059
S2144430C00B2938B5044614D146F204730E4D00223B
S2144430D00E48EA50FFF768FF46F20873EB581BB1F8
S2144430E046F20C72A85898472046BDE8384019F076
S2144430F0E3B8074B1A6832B1002206481A60BDE8A6
S2144431003840FFF751BF38BD6C484120AD7E46007D
S2144431106CAF4120C97E46000B2938B504464FF4AF
S214443120FB55134815D105FB040542F6440300221B
S2144431301048EA50FFF738FF42F64803EB581BB1F5
S21444314042F64C02A85898472046BDE8384019F045
S214443150B3B805FB040404F52154236833B10023B3
S21444316005482360BDE83840FFF71EBF38BD00BFA2
S2144431706C484120E77E4600037F46000B2938B55D
S21444318004464FF4FB55134815D105FB040542F697
S214443190440300221048EA50FFF706FF42F648036D
S2144431A0EB581BB142F64C02A85898472046BDE857
S2144431B0384019F081B805FB040404F5215423680B
S2144431C033B1002305482360BDE83840FFF7ECBE22
S2144431D038BD00BF6C484120227F46003E7F4600F3
S2144431E00B2938B504464FF4FB55134815D105FB57
S2144431F0040542F6440300221048EA50FFF7D4FE82
S21444320042F64803EB581BB142F64C02A85898477E
S2144432102046BDE8384019F04FB805FB040404F5D1
S2144432202154236833B1002305482360BDE8384061
S214443230FFF7BABE38BD00BF6C4841205D7F4600EC
S214443240797F460038B50A243C4D2946002012F0C2
S214443250ABFE38B1013C14F0FF04F6D121463848A1
S214443260FFF7A2FE0A24374D2946012012F09CFEA1
S21444327038B1013C14F0FF04F6D101213048FFF781
S21444328093FE0A24304D2946022012F08DFE38B1B2
S214443290013C14F0FF04F6D102212948FFF784FECE
S2144432A000222A49B4200A241AF003FE00222849A0
S2144432B0B5201AF0FEFD00222649B6201AF0F9FD84
S2144432C0B4201AF0F7FDB5201AF0F4FDB6201AF033
S2144432D0F1FD002012F0FEFA38B1013C14F0FF0470
S2144432E0F7D121461C48FFF75FFE0A24012012F05E
S2144432F0F1FA38B1013C14F0FF04F7D10121164825
S214443300FFF752FE0A24022012F0E4FA38B1013CD8
S21444331014F0FF04F7D102210F48FFF745FE0121C0
S214443320002012F059FB0121084612F055FB0121FA
S2144433300220BDE8384012F04FBB00BFB88D4600AF
S214443340B47F46005C8D4600008D4600856545008A
S2144433508B65450091654500987F460038B51C4C02
S2144433600546206804302044FFF7FCFD012801D1BF
S214443370012038BD2368E21810790A2810D00D2899
S2144433800ED0082815D123B1013B12482360FFF71D
S2144433900BFE2368AB42EBD325440020E87006E0DE
S2144433A00D48FFF701FE236800202344187120606F
S2144433B0DFE7A0F120035E2BEBD8FFF7E9FD236897
S2144433C0E11801330A792360303A81F80421E0E7B2
S2144433D06C484120C97F4600D87F460010B58020FF
S2144433E0FFF7BCFF90B90A4C23797BB10949201DED
S2144433F00BF0E8FA20B90848BDE81040FFF7D4BD02
S214443400211D0648BDE81040FFF7CEBD10BD00BFE5
S2144434106C484120CD7F4600D37F4600DB7F460084
S2144434202DE9F04F082389B0002492463B4A0546CE
S21444343089464FF064081068EDB2516802AF012621
S21444344022468DF810408DF81C40DFF8E8B0CDE9F0
S21444345005346B4403C35146484623F014FC04AA7F
S214443460214640F255532846CDF8048000978DF8FF
S2144434701C608DF81040059418F00CFE284B04AAE6
S2144434802146284602934FF607738DF81060ADF830
S2144434900C300623CDE9007805935B4618F0FAFD18
S2144434A0204A0623214602924FF6FF720593284689
S2144434B05B46ADF80C2004AA8DF81060CDE9007880
S2144434C018F0E8FD184A062321460292284604AA24
S2144434D005935B46ADF80C408DF81060CDE9007856
S2144434E018F0D8FD114B124A214628468DF8106034
S2144434F0CDE90232082304AA05935B46CDE9007859
S21444350018F0C8FD0A20FFF71EFC324651464846CE
S21444351023F0B9FB09B0BDE8F08F00BFE473460062
S2144435201000500010019FFF1002C00071020304F7
S21444353005060708F100DA182DE9F041044600288C
S21444354055D16D201AF0B6FC2246C0496D201AF0BB
S214443550B0FC6E201AF0AEFC2246BD496E201AF02E
S214443560A8FC01220821BB4823F08DFB012205213B
S214443570B84823F088FBB84AB849204618F01CF8E7
S2144435800121204618F0DAFF22460E21204618F084
S21444359031FE204618F0B0FF2346B14A0E2120469D
S2144435A018F048F92346AF4A0E21204618F086F90B
S2144435B0FEF7B2FE2046FFF7A8F9AB4B012242F6CF
S2144435C044015A5003F521531A6041F6987000237B
S2144435D0A64A4443A648A35004441A46013384F8F2
S2144435E071202834C82BF9D10020BDE8F081012889
S2144435F046D0022840F0898074209E4F1AF05AFC28
S21444360000229D4974201AF054FC75201AF052FC8E
S21444361000229A4975201AF04CFC0122042198484D
S21444362023F031FB01220621964823F02CFB00258B
S214443630954A20469549DFF8B88217F0BDFF2046E4
S21444364018F05AFF05F10E0658F83530904A022015
S214443650F6B223F060430135314618F0EBF83A46AB
S214443660002331460220503718F028F90B2DE9D1B3
S2144436707D4B012246F204715A5003F5CE43A3E72C
S2144436807120844F1AF016FC0022834971201AF0E8
S21444369010FC72201AF00EFC0022804972201AF0A8
S2144436A008FC22460721774823F0EDFA22460221F9
S2144436B0734823F0E8FA0025794A20467949DFF82A
S2144436C0348217F079FF204618F016FF05F10E06EF
S2144436D058F83530744A0120F6B223F06043013579
S2144436E0314618F0A7F83A460023314601205037B1
S2144436F018F0E4F8042DE9D144F2A4715A4B01229F
S2144437005A5044F2A0715A505FE7032859D004280F
S21444371000F0F48005287FF458AF7B20634D1AF000
S214443720C9FB002262497B201AF0C3FB7C201AF0B6
S214443730C1FB00225F497C201AF0BBFB01220E210C
S214443740504823F0A0FA01225B48114623F09BFA26
S2144437505A4A5B49204617F02FFF204618F0CCFE05
S214443760012255492046FFF75BFE564A54492046F7
S21444377017F022FF204618F0BFFE2B68524A0E214F
S21444378023F06043204618F055F800234F4A0E2194
S214443790204618F093F8AB684B4A0F2123F0604359
S2144437A0204618F047F80023494A0F21204618F0CF
S2144437B085F84CF224512C4B01225A504CF220519D
S2144437C0A1E77720434F1AF075FB00224249772041
S2144437D01AF06FFB78201AF06DFB00223F497820E0
S2144437E01AF067FB012200213D4823F04CFA0122DF
S2144437F03B4800251146DFF8008123F044FA394A55
S2144438003949204617F0D8FE204618F075FE05F1D3
S2144438100E0658F83530354A0320F6B223F0604396
S2144438200135314618F006F83A460023314603205F
S214443830503718F043F80A2DE9D148F264610A4B30
S21444384001225A5048F260615DE700BFB5DC45008E
S214443850BBDC450008172940AC914600784140201F
S214443860342040201C4C40206C484120D8A64020A0
S214443870488740201C604020FDDC450003DD4500B1
S2144438800E1729400C172940FC9046002838402043
S214443890542040201C564020DFDC4500E5DC450033
S2144438A054914600D03C40204420402014774600A3
S2144438B03FDD450045DD450010172940EC734600C2
S2144438C0302A4020F48F4600842040201C7E40202E
S2144438D06C7E40201C6A40201BDD450021DD4500EF
S2144438E006172940A4904600803340206420402098
S2144438F084774600DC774600347746007920294DA5
S2144439001AF0D8FA0022284979201AF0D2FA7A20F6
S2144439101AF0D0FA002225497A201AF0CAFA01226F
S2144439200A21234823F0AFF901220921204823F035
S214443930AAF9204A2049204617F03EFE204618F0B1
S214443940DBFD09221A492046FFF76AFD1B4A1A493D
S214443950204617F031FE204618F0CEFD2B68184A54
S2144439600E2123F06043204617F064FF0023154AD7
S2144439700E21204617F0A2FFAB68114A0F2123F010
S2144439806043204617F056FF00230F4A0F21204677
S21444399017F094FF4AF2C4510C4B01225A504AF293
S2144439A0C051B0E6247746002DDD450033DD4500A2
S2144439B008172940EC734600D82E40204C90460009
S2144439C0742040201C7440206C7440206C48412075
S2144439D041F69872084B02FB003310B503EB8104A2
S2144439E0E278A07800EB0220627802EB002213F81B
S2144439F0210000EB022010BD4887402010B5094B3B
S214443A0041F6987404FB0030130A00EB810181F8F8
S214443A10282081F82930130C120E81F82A3081F8B8
S214443A202B2010BD4887402013B502AB044603E95B
S214443A30060041F69871094A9DF8043001FB0022BD
S214443A40009903F03F0321F06041FEF791FF2046C2
S214443A5002B0BDE81040FEF758BF00BF7087402054
S214443A60FDF7F2BE7047704770477047704770471F
S214443A7070477047704770477047074B074A196846
S214443A8058799160197941EA002191819979DB79D5
S214443A909173D373704700BF48874020C08340204B
S214443AA00C4A0D4810B55178137801F00104C1F35F
S214443AB0410143EA042343EA41239178D27843EA16
S214443AC0C12343EAC243426902F078421343436146
S214443AD010BD00BF48874020C0834020034B0449A4
S214443AE01A7C097861F300021A747047C083402038
S214443AF0488740200549064B0A7E1B7822F01F0261
S214443B0003F01F0313430B76704700BFC083402067
S214443B10488740200549064B0A7F1B7822F01F023F
S214443B2003F01F0313430B77704700BFC083402046
S214443B30488740200649074B91F820201B7822F0FE
S214443B400F0203F00F03134381F82030704700BF81
S214443B50C083402048874020114B124810B55A78FD
S214443B60997802F003041B7843EA0423C2F38104E1
S214443B7043EA8423C2F30114920943EA043343EA32
S214443B80823301F00302C1F3810143EA0243426AED
S214443B90120D43EA814312051343436210BD00BF2E
S214443BA048874020C08340200E4B0F4A58781978E7
S214443BB041EA002158791185997801F00F0182F87D
S214443BC02A10D97882F82B10197941EA0021918578
S214443BD09979DB7901F00F0182F82F3082F82E10A4
S214443BE0704700BF48874020C08340200E4B0F4A92
S214443BF05878197841EA002158791186997801F065
S214443C000F0182F83210D97882F83310197941EAD4
S214443C10002191869979DB7901F00F0182F83730DB
S214443C2082F83610704700BF48874020C083402043
S214443C300C4B0D4A5878197841EA00215879118777
S214443C40997801F00F0182F83A10197941EA002177
S214443C5091879979DB7901F00F0182F83F3082F839
S214443C603E10704748874020C08340202D492E4A46
S214443C7010B50B78487803F07F0343EAC01388787E
S214443C8043EAC033C87843EAC053106C00F000409F
S214443C90034348791364C0F340040B79897982F866
S214443CA0443000F001031B0243EA4423C0F380047B
S214443CB043EA8423C0F3C00443EAC423C0F3001495
S214443CC043EA0433C0F3401443EA4433C0F3801455
S214443CD0C00943EA843343EAC03301F0010043EAAF
S214443CE00043C1F3400043EA4043C1F3800043EA43
S214443CF08043C1F3C00043EAC043C1F3001043EA23
S214443D000053C1F34010C1F3801143EA405343EAE1
S214443D108153516C21F4FF0121F4FE410B4353645B
S214443D2010BD00BF48874020C08340200D4A0E483F
S214443D3010B55178137801F00F04C1F3001143EA2B
S214443D40042343EA0133917843EA4133D17843EA82
S214443D504153816C01F060410B4383645368C364F0
S214443D6010BD00BF48874020C0834020034A044B10
S214443D701168526819655A65704700BF48874020E5
S214443D80C0834020244A254970B55578137805F0F9
S214443D9003069078D47843EA0623C5F3810643EABB
S214443DA08623C5F30116AD0943EA063343EA853351
S214443DB0C0F3011543EA0543850900F00F0043EAC2
S214443DC0854304F0030543EA0553C4F3810543EAF7
S214443DD08553C4F30115A40943EA056343EA84639F
S214443DE08C6D04F07044234354798B651379D279EF
S214443DF081F85C30230104F0030403F4706343EA5F
S214443E000233CA6D43EA0050054B40EA046013404F
S214443E101843C86570BD00BF48874020C083402013
S214443E20FF0000FC70B5224D224A2C78E878C4F393
S214443E30401604F00F03297943EA0613C4F38016A8
S214443E40E40943EA461343EA84136C7843EAC4130A
S214443E50AC7843EAC43300F0030443EAC453C0F3E3
S214443E60810443EA4463C0F30114800943EAC4630B
S214443E7043EA4073106E00F00040034301F0030031
S214443E8013668B0803F004030343880800F0080015
S214443E9003438808C90900F01000034343EA41136A
S214443EA092F8641021F03F010B4382F8643070BDF1
S214443EB048874020C0834020114A124810B55178A4
S214443EC0137801F0030443EA0423C1F3810443EA6C
S214443ED08423C1F30114890943EA043343EA813352
S214443EE0A0F868305388A0F86A309388A0F86C30FD
S214443EF0937980F86E30D37980F86F3010BD00BF68
S214443F0048874020C0834020064B074A19685879A2
S214443F1011671979DB7941EA002182F87630A2F8F4
S214443F207410704748874020C0834020084A094997
S214443F301378907881F8783053781843D378064AC3
S214443F409B0443EA0023886F024013438B67704701
S214443F5048874020C0834020FF0000FC08B5054B3E
S214443F6018880BF053FB04490BF0A4FB034BD867AB
S214443F7008BD00BF48874020CDCCCC3DC083402000
S214443F80104B41F69871104A595C82F8801041F6FD
S214443F909B71585C41F69A71595C41EA0021A2F83B
S214443FA0811041F69D71585C41F69C71595C41EA1A
S214443FB00021A2F8841041F69F715B5C82F886303B
S214443FC0704700BF48874020C0834020064A41F6D9
S214443FD09871064B5158C3F8881041F69F71525C4D
S214443FE083F88C20704700BF48874020C083402019
S214443FF00C4A41F69F730C4910B541F69974D05C4F
S21444400041F69873D35C125D02F0010243EA022340
S214444010D1F89020520C43EA402352041343C1F88B
S214444020903010BD48874020C0834020284941F640
S2144440309973284A70B5C85C41F69A73CD5C41F6CC
S2144440409B7300F00306CC5C41F69873CB5C43EA62
S2144440500623C0F3810643EA8623C0F3011680098B
S21444406043EA063343EA803305F00300C5F381058B
S21444407043EA004304F0030043EA854343EA00531B
S214444080C4F38100A40943EA8053D2F8940043EA77
S214444090046300F07C40034341F69F70C2F89430BA
S2144440A041F69C73CB5C82F8983041F69D73CB5CAA
S2144440B0095C1B0203F47C5343EA8133D2F898101C
S2144440C021F47F1121F47C510B43C2F8983070BD23
S2144440D048874020C0834020214843F63073214916
S2144440E030B5C35A5BBAA1F89C3043F63373C25C0E
S2144440F043F63273C2F30115C45C930943EA85035D
S21444410004F00F05240943EA051343F63675455D66
S214444110ED0843EA0523C2F3800543EA4533B1F884
S2144441209E5005F440452B43A1F89E3043F6347325
S214444130C55C43F63573C35C43EA0523A1F8A03057
S214444140C2F3C003520143EA440302F060021A4336
S21444415091F8A23023F07F031A4381F8A22030BDA1
S21444416048874020C0834020164A43F63073164999
S21444417010B5D35A5BBAA1F8A43043F63273D05C78
S21444418043F63373D35C43EA0023A1F8A63043F6E0
S2144441903673D05C43F63473D45C43F63573D35CE1
S2144441A043EA042200F00103C0F3400043EA42031A
S2144441B0D1F8A820920C43EA404392041343C1F832
S2144441C0A83010BD48874020C0834020124A43F69A
S2144441D03071124B515A49BAA3F8AC1043F63271B7
S2144441E0505C43F63371515C41EA0021B3F8AE00AB
S2144441F061F30D0043F63671A3F8AE0043F637700C
S214444200515C125C42EA0122B3F8B01062F30D012D
S214444210A3F8B010704700BF48874020C0834020B2
S21444422030B543F63073304C3049E35A5BBAA1F8A4
S214444230B43043F63673E05C43F63773E25C43F6D9
S2144442403273E55C00F0030343EA8503C0F380055C
S21444425043EA8523C2F3800543EAC523850943EA36
S2144442600533B1F8B65005F440452B43C2F3C005B8
S214444270A1F8B63043F63373E35C81F8B830C0F344
S214444280C0031B0243EA452302F0030543EA8523A1
S21444429043F63475655D43EA0533C0F30015C0F351
S2144442A0401043EA0553C2F3001543EA45539509C3
S2144442B0120943EA8553D1F8B85002F0020225F4B5
S2144442C07F05024325F47F452B43C1F8B83043F6B7
S2144442D03573E35C81F8BB3091F8BC3023F00303BC
S2144442E01A4381F8BC2030BD48874020C083402014
S2144442F0F0B543F63273404F404DFE5C43F634739C
S214444300F95C43F63373C6F3801CF85C43F63573A6
S214444310FC5C43F63673FA5CF30943EA4C0343F613
S214444320317C42EA042217F80CC043EA8C03C6F3F5
S214444330401C43EA8C23C6F3001C43EACC23C1F357
S214444340400C43EA0C3343F6307C17F80C7043EACF
S2144443504733C6F3C00743EA4753C6F3800743EAE6
S2144443608753C0F3001743EAC753470943EA076332
S214444370C4F30117A40943EAC763C6F3400706F02B
S214444380010643EA477343EA8673D5F8C06006F0ED
S2144443900046334301F00106C5F8C030C2F30903B2
S2144443A0C0F3C00243EA862343EAC223C0F3800232
S2144443B043EA0233C0F3400200F0010043EA4233CA
S2144443C0C1F3C00243EA803343EAC433C1F3001462
S2144443D043EA44438C09C1F3800143EA844343EAF5
S2144443E0025343EA4151D5F8C4309B0D9B0519430B
S2144443F0C5F8C410F0BD00BF48874020C0834020A5
S214444400284843F6307343F636722749F0B5C35A04
S21444441043F63275845C43F635725BBA455D825C1E
S214444420A709A1F8C83043F6337347EA820743F630
S2144444303772C65C43F63473825CC35CB009B1F829
S214444440CAC042EA042240EA8500C6F3810543EA2C
S2144444500623C6F3011640EA8520144DC3F3090328
S2144444600CEA050C43EA862340EA0C0043EA073389
S214444470A1F8CA00C4F38100C4F3011443EA80538C
S214444480D1F8CC0000F07F400343C1F8CC30C2F3EF
S2144444900903B1F8D02043EA842315402B43A1F8FE
S2144444A0D030F0BD48874020C083402000F0FFFF56
S2144444B01D4943F630731D48F0B5CB5A43F6327463
S2144444C05BBA0E5DA0F8D43043F63373CA5C43F649
S2144444D03573CD5CC2F3810443F634732F09CB5C49
S2144444E044EA870443F6367743EA0223C95D41EA41
S2144444F0052144EA8111A0F8D610C3F30901C2F39A
S214444500001343EA41039109C2F3401243EAC62327
S21444451043EAC16343EA4273D0F8D82002F04042EB
S2144445201343C0F8D830F0BD48874020C0834020AD
S21444453070B5234943F6367443F6357543F63073FF
S2144445400C5D4E5DCB5AA5091E485BBA45EA860506
S21444455043F63776A0F8DC3043F633738E5DCA5C98
S21444456043F6347346EA042443F63276CB5C8E5DD7
S214444570910943EA022341EA8601C2F38006C3F363
S214444580090341EA8621B0F8DE6006F478463143F2
S214444590A0F8DE10C2F3C00143EA8123C2F300113F
S2144445A0520943EAC52343EA415343EA8453C0F8D5
S2144445B0E03090F8E43062F3000380F8E43070BDF5
S2144445C048874020C08340201D4A43F630731D4828
S2144445D070B5D35A5BBAA0F8E83043F63273D45C6D
S2144445E043F63473D55C43F63373D15C2B09C5F379
S2144445F0C00543EA011143F63673D65C43F6357379
S214444600D35CDB0043EA5612C4F3400343EA450353
S21444461004F00105A40843EA850343EAC403B0F85A
S214444620EA4004F47E442343A0F8EA3041EA0233E5
S214444630D0F8EC20D20DD2051343C0F8EC3070BD50
S21444464048874020C08340201B4943F631731B48AB
S21444465030B5CB5C80F8F03043F63273CA5C43F630
S2144446603573CD5C43F63473CC5C43F63073C95C27
S21444467093091B0243EA8123C2F3401143EA814370
S214444680C2F38001C2F3C00243EAC143D0F8F0103B
S21444469043EA02532A0905F00F0543EA4253084AFF
S2144446A043EA45630A401343C0F8F030230943EA1B
S2144446B0041480F8F44030BD48874020C08340202E
S2144446C0FF0000E0074943F63073074ACB581BBA4D
S2144446D0C2F8003143F63473CB581BBAC2F80431DF
S2144446E0704700BF48874020C0834020214845F695
S2144446F0C863214930B5C35A5BBAA1F8083145F6B8
S214444700CB63C25C45F6CA63C2F30115C45C930925
S21444471043EA850304F00F05240943EA051345F6E6
S214444720CE65455DED0843EA0523C2F3800543EABA
S2144447304533B1F80A5105F440452B43A1F80A31F4
S21444474045F6CC63C55C45F6CD63C35C43EA0523B6
S214444750A1F80C31C2F3C003520143EA440302F009
S21444476060021A4391F80E3123F07F031A4381F80E
S2144447700E2130BD48874020C0834020164A45F667
S214444780C863164910B5D35A5BBAA1F8103145F63A
S214444790CA63D05C45F6CB63D35C43EA0023A1F8F6
S2144447A0123145F6CE63D05C45F6CC63D45C45F610
S2144447B0CD63D35C43EA042200F00103C0F3400017
S2144447C043EA4203D1F81421920C43EA404392044C
S2144447D01343C1F8143110BD48874020C08340209D
S2144447E0F0B545F6CA632D4F2D4CFD5C45F6CC63BB
S2144447F0F95C45F6CB63C5F3801CFE5C45F6CD6399
S214444800F85C45F6CE63FA5CEB0943EA4C0345F69E
S214444810C96C42EA002217F80CC0C2F3090243EA04
S2144448208C03C5F3401C43EA8C23C5F3001C43EABF
S214444830CC23C1F3400C43EA0C3345F6C86C17F856
S2144448400C7043EA4733C6F30017760943EA4753E6
S21444485043EA8653C0F30116800943EA4663C5F328
S214444860400605F0010543EAC66343EA0573D4F8F7
S214444870245105F060452B43C4F8243101F001036C
S21444488042EA832242EAC020C1F30012890940EA80
S214444890423040EA8131A4F82811F0BD48874020D0
S2144448A0C0834020284845F6C86345F6CE6227496B
S2144448B0F0B5C35A45F6CA65845C45F6CD625BBA24
S2144448C0455D825CA709A1F82C3145F6CB6347EADF
S2144448D0820745F6CF62C65C45F6CC63825CC35C11
S2144448E0B009B1F82EC142EA042240EA8500C6F374
S2144448F0810543EA0623C6F3011640EA8520144D93
S214444900C3F309030CEA050C43EA862340EA0C0089
S21444491043EA0733A1F82E01C4F38100C4F301141B
S21444492043EA8053D1F8300100F07F400343C1F896
S2144449303031C2F30903B1F8342143EA84231540E5
S2144449402B43A1F83431F0BD48874020C083402033
S21444495000F0FFFF1D4945F6C8631D48F0B5CB5A25
S21444496045F6CA645BBA0E5DA0F8383145F6CB63AB
S214444970CA5C45F6CD63CD5CC2F3810445F6CC6390
S2144449802F09CB5C44EA870445F6CE6743EA022304
S214444990C95D41EA052144EA8111A0F83A11C3F3FE
S2144449A00901C2F3001343EA41039109C2F34012DA
S2144449B043EAC62343EAC14343EA4253D0F83C2180
S2144449C0920D92051343C0F83C31F0BD4887402011
S2144449D0C0834020184845F6C863184930B5C35AC2
S2144449E05BBAA1F8403145F6CC63C55C45F6CA636C
S2144449F0C45C45F6CB63C35C43EA042245F6CD6308
S214444A00E409C35CB1F8420143EA0523ED09C3F364
S214444A10090343EA85230A4D28400343A1F842315B
S214444A20C2F30903B1F8442143EA84232A401343DA
S214444A30A1F8443130BD00BF48874020C0834020A1
S214444A4000F8FFFF1D4A45F6C8631D4870B5D35AA3
S214444A505BBAA0F8483145F6CA63D45C45F6CC63E5
S214444A60D55C45F6CB63D15C2B09C5F3C00543EA58
S214444A70011145F6CE63D65C45F6CD63D35CDB00C8
S214444A8043EA5612C4F3400343EA450304F00105DF
S214444A90A40843EA850343EAC403B0F84A4104F44D
S214444AA07E442343A0F84A3141EA0233D0F84C21ED
S214444AB0D20DD2051343C0F84C3170BD4887402010
S214444AC0C08340201B4945F6C9631B4830B5CB5CC0
S214444AD080F8503145F6CA63CA5C45F6CD63CD5C72
S214444AE045F6CC63CC5C45F6C863C95C93091B02A7
S214444AF043EA8123C2F3800143EA8143C2F3C001FF
S214444B00C2F3401243EAC143D0F8501143EA025379
S214444B102A0905F00F0543EA4253084A43EA456327
S214444B200A401343C0F85031230943EA041480F87A
S214444B30544130BD48874020C0834020FF0000E0F9
S214444B4030B545F6C863304C3049E35A5BBAA1F8F1
S214444B50183145F6CE63E05C45F6CF63E25C45F635
S214444B60CA63E55C00F0030343EA8503C0F38005AB
S214444B7043EA8523C2F3800543EAC523850943EA0D
S214444B800533B1F81A5105F440452B43C2F3C0052A
S214444B90A1F81A3145F6CB63E35C81F81C31C0F3C7
S214444BA0C0031B0243EA452302F0030543EA852378
S214444BB045F6CC65655D43EA0533C0F30015C0F39E
S214444BC0401043EA0553C2F3001543EA455395099A
S214444BD0120943EA8553D1F81C5102F0020225F427
S214444BE07F05024325F47F452B43C1F81C3145F627
S214444BF0CD63E35C81F81F3191F8203123F0030341
S214444C001A4381F8202130BD48874020C083402085
S214444C10074945F6C863074ACB581BBAC2F8603101
S214444C2045F6CC63CB581BBAC2F86431704700BF14
S214444C3048874020C08340200C4947F664630C48AC
S214444C40CA5C47F66563CB5C43EA022247F6626376
S214444C50CB5C03F00F0343EA0213D0F86821120D2D
S214444C6012051343C0F86831704700BF4887402098
S214444C70C0834020064A47F66263D15C47F66363C6
S214444C80D35C044A43EA0123A2F86C31704700BF60
S214444C9048874020C08340200C4949F6FC530C48C2
S214444CA0CA5C49F6FD53CB5C43EA022249F6FA5302
S214444CB0CB5C03F00F0343EA0213D0F87021120DC5
S214444CC012051343C0F87031704700BF4887402030
S214444CD0C0834020064A49F6FA53D15C49F6FB5352
S214444CE0D35C044A43EA0123A2F87431704700BFF8
S214444CF048874020C083402010B51B4C20890AF0CA
S214444D0085FC1A490AF0D6FC194BA27B1860194B4D
S214444D1060891A600AF07AFC17490AF0CBFC1749F6
S214444D200AF0BEFB0AF018F80DA3D3E9002309F0F5
S214444D30B3FE0AF061FB124B124A1860E37BA0896B
S214444D4003F00F0313600AF061FC0F490AF0B2FC4B
S214444D500AF076FE0D4B186010BD00BFAFF300801E
S214444D60C3F5285C8FC2D53FC0834020CDCCCC3D14
S214444D70981F4020801F40200AD7A33C00C02344ED
S214444D808C1F40207C1F4020ACC52737841F402002
S214444D90104A1149137D03F003000860C3F38300EF
S214444DA00E499B0908600E490B60537D0D49C3F3B9
S214444DB0410003F0010308600B490B6053690B493B
S214444DC0C3F3C7230B60D38A094AC3F3C7031360EC
S214444DD0704700BFC08340206C1F4020681F40209F
S214444DE0641F40205C1F4020601F4020501F40200E
S214444DF0581F4020034B044A1B7C03F001031360F6
S214444E00704700BFC08340204C1F40200B4B0C4AC9
S214444E101B7E03F001011160C3F34001094A11608F
S214444E20C3F38001084A1160C3F3C001074AC3F3C1
S214444E3000131160064A1360704700BFC0834020C9
S214444E40481F4020441F4020401F40203C1F402015
S214444E50381F40200B4B0C4A1B7F03F001011160A6
S214444E60C3F34001094A1160C3F38001084A116044
S214444E70C3F3C001074AC3F300131160064A136024
S214444E80704700BFC0834020341F4020301F40205E
S214444E902C1F4020281F4020241F4020094B0A4A2C
S214444EA093F8203003F001011160C3F34001074A30
S214444EB01160C3F38001064AC3F3C0031160054A78
S214444EC013607047C0834020201F40201C1F402092
S214444ED0181F4020141F402008B5FFF78BFFFFF72C
S214444EE095FFFFF7B7FFBDE80840FFF7D7BF08B503
S214444EF0FFF7F2FFBDE80840FCF7A4BC164A174982
S214444F0092F8243003F003000860C3F38100144988
S214444F100860C3F3011013499B09086012490B60EB
S214444F2092F82530114903F003000860C3F381006A
S214444F300F490860C3F301100E499B0908600E49E7
S214444F400B6092F826300D4A03F00301C3F3810345
S214444F5011600B4A13607047C0834020201A4020DB
S214444F601C1A4020181A4020141A4020101A4020B8
S214444F700C1A4020081A4020041A4020001A4020E8
S214444F80FC19402010B5194C208D0AF03FFB1849F7
S214444F900AF090FB17490AF083FA174B174A186031
S214444FA094F82A30A08D03F00F011B091160144AAF
S214444FB0136094F82B30134A323B13600AF026FBF6
S214444FC011490AF077FB11490AF06AFA104B114A64
S214444FD0186094F82E3003F00F011B0911600E4A36
S214444FE0136094F82F200D4B1A6010BDC0834020E8
S214444FF00AD7A33B0AD72343101F40200C1F402048
S214445000081F4020041F40200AD7A33AF8D323425F
S214445010001F4020FC1E4020F81E4020F41E402066
S21444502010B5194C208E0AF0F1FA18490AF042FBE2
S21444503017490AF035FA174B174A186094F8323075
S214445040A08E03F00F011B091160144A136094F8F4
S2144450503320134B1A600AF0D9FA12490AF02AFB95
S21444506011490AF01DFA114B114A186094F836306B
S21444507003F00F011B0911600E4A136094F83720A1
S2144450800D4B1A6010BD00BFC08340200AD7A33B17
S2144450900AD72343F01E4020EC1E4020E81E402042
S2144450A0E41E40200AD7A33AF8D32342E01E402009
S2144450B0DC1E4020D81E4020D41E402010B5174C7D
S2144450C0208F0AF0A3FA16490AF0F4FA15490AF0B2
S2144450D0E7F9154B154A186094F83A30A08F03F058
S2144450E00F011B091160124A13600AF08FFA114926
S2144450F00AF0E0FA10490AF0D3F9104B104A186047
S21444510094F83E3003F00F011B0911600D4A1360FA
S21444511094F83F200C4B1A6010BD00BFC08340205B
S2144451200AD7A33B0AD72343D01E4020CC1E402098
S214445130C81E40200AD7A33AF8D32342C41E4020B0
S214445140C01E4020BC1E4020B81E402010B53E4C19
S2144451503E4A94F84030B4F8400003F00101C0F3EE
S214445160C7101160C3F34001394A1160C3F382018A
S214445170384AC3F341131160374A13600AF046FABB
S21444518036490AF097FA0AF05BFC354B1860206CF7
S214445190C0F3C7300AF03AFA30490AF08BFA0AF0FC
S2144451A04FFC304B1860B4F84200C0F3C7100AF006
S2144451B02DFA2D490AF074F90AF042FC2B4B94F868
S2144451C0442018602A4B1A6094F84530294A03F064
S2144451D001011160C3F34001274A1160C3F3800103
S2144451E0264A1160C3F3C001254A1160C3F3001177
S2144451F0244A1160C3F34011234A1160C3F380115B
S214445200224ADB091160224A136094F84630214A48
S21444521003F001011160C3F340011F4A1160C3F358
S21444522080011E4A1160C3F3C0011D4A1160C3F3D6
S21444523000111C4A1160C3F340111B4AC3F3801388
S21444524011601A4A136010BDC0834020B41E40202B
S214445250B01E4020AC1E4020A81E40200AD7233C47
S214445260A41E4020A01E4020000020429C1E402039
S214445270981E4020941E4020901E40208C1E4020A5
S214445280881E4020841E4020801E40207C1E4020D5
S214445290781E4020741E4020701E40206C1E402005
S2144452A0681E4020641E4020601E40205C1E402035
S2144452B038B5264D264B95F8484004F00102C4F311
S2144452C002101A60C4F34002224B1A60C4F38002F0
S2144452D0214B1A60C4F3C002204BE4091A600AF05A
S2144452E091F91F4B1F4A18601F4BA86C1C6095F819
S2144452F04930C0F3473003F00F01C3F3001332388C
S21444530011601A4A13600AF081F9194B1860B5F80F
S2144453104A00C0F3471032380AF078F9154B186043
S214445320B5F84C00A0F500400AF070F9124B18602E
S214445330B5F84E000AF06AF910490AF0BBF910496C
S2144453400AF0AEF80F4B186038BD00BFC08340204B
S214445350581E4020541E4020501E40204C1E4020C4
S214445360481E4020401E4020441E40203C1E4020F4
S214445370381E4020341E4020301E40200AD7233C8E
S214445380000048432C1E40207047304B304A10B52E
S21444539093F85940C4F381011170C4F301112D4AA6
S2144453A01170C4F301012C4AA409117093F85820D3
S2144453B02A49C2F381100870C2F3011028490870C4
S2144453C0C2F381002749C2F30102087026490A70D5
S2144453D093F85D202549C2F38100C2F301020870A8
S2144453E023490A7093F85E202249C2F303120A70D6
S2144453F093F85F202049C2F301020A7093F85A20BA
S2144454001E4902F003000860C2F381001C4908608C
S214445410C2F301101B49920908601B490A6093F8BD
S2144454205B201A4902F00300C2F38102086018495F
S21444543093F85C000A700AF0E9F816490AF03AF95B
S214445440154B1860154B1C6010BD00BFC083402030
S214445450281E4020271E4020261E4020251E402071
S214445460241E4020231E4020221E4020211E402071
S214445470201E40204C184020E81D4020181E402086
S214445480141E4020101E40200C1E4020081E4020A3
S21444549045184020CDCCCC3D001E40201C1E40204C
S2144454A0264A274992F8603003F007000860C3F3A1
S2144454B0C00024490860C3F3001023490870C3F3AE
S2144454C040102249C3F38013087021490B70B2F888
S2144454D060302049C3F3C7130B60136E1E49C3F3F1
S2144454E0C7330B60B2F862301C49C3F3C1130B6078
S2144454F092F863301A49C3F341000860C3F3C1000D
S2144455001849C3F34113086017490B6092F8643096
S214445510164A03F003011160C3F38001144A116074
S214445520C3F3C001134A1160C3F30011124AC3F314
S21444553040131160114A1360704700BFC083402077
S214445540E41D4020E01D4020DE1D4020DD1D40209F
S214445550DC1D4020D81D4020D41D4020D01D4020B6
S214445560CC1D4020C81D4020C41D4020C01D4020E6
S214445570BC1D4020B81D4020B41D4020B01D402016
S21444558010B5194C194A94F8683094F86A00C3F375
S2144455908101C3F301131170154A137094F86930EE
S2144455A0144AC3F301011170C3F38101124AC3F3D1
S2144455B081131170114A13700AF024F8104B1860C6
S2144455C094F86B000AF01EF80E4B94F86C201860A2
S2144455D00D4B1A7094F86D200C4B1A7094F86E208C
S2144455E00B4B1A7010BD00BFC0834020A61D402040
S2144455F0951D4020A51D4020941D4020A41D4020FC
S214445600A01D40209C1D4020981D4020971D4020F2
S214445610961D402010B50C4CB4F8720009F0F6FF05
S2144456200A490AF047F80A4B1860B4F8700009F0C3
S214445630EDFF06490AF03EF8064BB4F874201860AD
S214445640054B1A8010BD00BFC0834020CDCCCC3D56
S214445650901D40208C1D40208A1D4020054A064946
S214445660B2F87A3092F87820C3F387030B70034B72
S2144456701A707047C0834020891D4020881D4020F2
S21444568010B5124C124B94F88020B4F881001A607E
S21444569009F0BCFF0F490AF00DF80F4909F000FF66
S2144456A00E4B1860B4F8840009F0B0FF0C490AF0B9
S2144456B001F80C4B0C4A186094F8863003F00F013E
S2144456C01B091160094A136010BD00BFC083402007
S2144456D0841D4020ACC52737ACC5A73E801D40205E
S2144456E0CDCCCC3D7C1D4020781D4020741D4020F0
S2144456F010B5114CB4F8880009F088FF0F4909F03A
S214445700D9FF0F4909F0CCFE0E4B1860B4F88A0056
S21444571009F07CFF094909F0CDFF094909F0C0FEAC
S214445720094B0A4A186094F88C3003F00F011B09A1
S2144457301160074A136010BDC08340200AD7A33CBB
S21444574000C02344701D40206C1D4020681D40202E
S214445750641D4020114A124992F8903003F0030029
S2144457600860C3F381000F490860C3F301100E4973
S2144457709B0908600D490B6092F891300C4903F080
S2144457800100C3F3430308600A490B60D2F8903023
S214445790094AC3F343331360704700BFC0834020B5
S2144457A0601D40205C1D4020581D4020541D402054
S2144457B0501D40204C1D4020481D4020184B1B784F
S2144457C0002B2CD1174A184992F8943003F0030062
S2144457D00860C3F3810015490860C3F301101449F7
S2144457E09B09086013490B6092F89530124903F000
S2144457F003000860C3F3810010490860C3F3011036
S2144458000F499B0908600F490B6092F896300E4A80
S21444581003F00301C3F3810311600C4A136070471D
S2144458203A184020C0834020441D4020401D40205C
S2144458303C1D4020381D4020341D4020301D402053
S2144458402C1D4020281D4020241D4020201D402083
S21444585010B50C4C94F89F0000F01F0000EB80003D
S21444586009F0D4FE084B1860B4F8A00009F0CEFE48
S214445870064909F01FFF064909F012FE054B186059
S21444588010BD00BFC0834020041D4020CDCC4C3DFD
S21444589000C0CC44001D402010B50C4CB4F8A60003
S2144458A009F0B4FE0A4909F005FF0A4909F0F8FD73
S2144458B0094B1860D4F8A800C0F34F00A0F5FF4089
S2144458C07F3809F0A3FE054B186010BDC083402006
S2144458D00AD7A33C00C02344F01C4020E81C4020C8
S2144458E010B50D4CB4F8AE00C0F30D0009F08EFEB2
S2144458F04FF07A5109F0DEFE084B1860B4F8B00059
S214445900C0F30D0009F082FE4FF07A5109F0D2FE42
S214445910034B186010BD00BFC0834020E01C4020ED
S214445920DC1C4020704708B5074BB3F8C400C0F3EE
S214445930090009F06BFE054909F0BCFE044909F06C
S214445940AFFD044B186008BDC0834020CDCCCC3D91
S2144459509A994C42D81C402010B5174CB4F8CA004B
S214445960C0F3090009F052FE144909F0A3FE144B93
S2144459701860B4F8CC00C0F3090009F047FE0F499C
S21444598009F098FE0F4B1860D4F8CC00C0F30930E9
S21444599009F03CFE094909F08DFE0B4B1860B4F83B
S2144459A0D000C0F3090009F031FE044909F082FE34
S2144459B0064B186010BD00BFC0834020CDCCCC3D04
S2144459C0D41C4020D01C4020CC1C4020C81C402066
S2144459D038B5144DB5F8D600800909F017FE1249BB
S2144459E009F068FE114909F05BFDB5F8D840104B44
S2144459F0C4F349041860204609F008FE0D4909F02E
S214445A0059FE0D4B1860D5F8D800C0F3CF2009F0E6
S214445A10FDFD0A4909F04EFE094B1860094B1C600F
S214445A2038BD00BFC0834020CDCC4C3D6666724135
S214445A30C41C40209A99193EC01C40200AD7233CD7
S214445A40BC1C4020501C402010B5164CB4F8DE0058
S214445A50C0F3090009F0DAFD134909F02BFE134B95
S214445A601860B4F8E000C0F3090009F0CFFD0E4911
S214445A7009F020FE0E4B1860D4F8E000C0F3C920AD
S214445A8009F0C4FD084909F015FE0A4B1860B4F83D
S214445A90E200800909F0BAFD034909F00BFE064B03
S214445AA0186010BDC08340209A99193EB81C402007
S214445AB0B41C4020B01C4020AC1C402010B5134CF5
S214445AC0B4F8EA00C0F3C50009F0A0FD104909F097
S214445AD0F1FD104909F0E4FC0F4B1860B4F8EC00F3
S214445AE0C0F30B0009F092FD0C4909F0E3FD0C4BA2
S214445AF01860D4F8EC00C0F30A3009F087FD044976
S214445B0009F0D8FD074B186010BD00BFC083402085
S214445B10CDCCCC3DCDCC4C40A81C40200AD7233C11
S214445B20A41C4020A01C40207047704710B50C4C65
S214445B3094F80B0100F01F0000EB800009F066FDAE
S214445B40084B1860B4F80C0109F060FD064909F0EA
S214445B50B1FD064909F0A4FC054B186010BD00BF12
S214445B60C08340209C1C4020CDCC4C3D00C0CC443F
S214445B70981C402010B50C4CB4F8120109F046FDB0
S214445B800A4909F097FD0A4909F08AFC094B18604E
S214445B90D4F81401C0F34F00A0F5FF407F3809F055
S214445BA035FD054B186010BDC08340200AD7A33C82
S214445BB000C02344941C4020901C4020704708B5E5
S214445BC0074BB3F82801C0F3090009F01FFD054947
S214445BD009F070FD044909F063FC044B186008BDE5
S214445BE0C0834020CDCCCC3D9A994C426C1C40207E
S214445BF010B5174CB4F82E01C0F3090009F006FDA1
S214445C00144909F057FD144B1860B4F83001C0F33A
S214445C10090009F0FBFC0F4909F04CFD0F4B1860D6
S214445C20D4F83001C0F3093009F0F0FC094909F012
S214445C3041FD0B4B1860B4F83401C0F3090009F079
S214445C40E5FC044909F036FD064B186010BD00BF5C
S214445C50C0834020CDCCCC3D681C4020641C4020F2
S214445C60601C40205C1C402010B5134CB4F83A012C
S214445C70800909F0CBFC114909F01CFD104909F0D4
S214445C800FFC104B1860B4F83C01C0F3490009F00F
S214445C90BDFC0D4909F00EFD09F0D2FE0B4B186011
S214445CA0D4F83C01C0F3C72009F0B0FC084909F019
S214445CB001FD084B186010BDC0834020CDCC4C3D40
S214445CC0666672418C1C40209A99193E841C40207A
S214445CD00AD7233C881C402010B50C4CB4F842012B
S214445CE0C0F3090009F092FC094909F0E3FC094BAA
S214445CF01860B4F84401C0F3090009F087FC04496D
S214445D0009F0D8FC044B186010BD00BFC083402087
S214445D109A99193E801C40207C1C402008B5FEF70A
S214445D20EBFFFFF735F8FFF7E9F8FFF70FFAFFF751
S214445D30BFFAFFF72AFBFFF7B3FBFFF721FCFFF799
S214445D4069FCFFF78BFCFFF71DF9FFF769F9FFF7CE
S214445D50B5F9FFF795FCFFF7CBFCFFF7FBFCFFF725
S214445D602DFDFFF7F9FDFFF733FEFFF76DFEFFF756
S214445D703FFFFFF779FFBDE80840FFF7ADBF10B51A
S214445D80124CB4F84A01C0F3C50009F03FFC104970
S214445D9009F090FC0F4909F083FB0F4B1860B4F8E8
S214445DA04C01C0F30B0009F031FC0C4909F082FCAD
S214445DB00B4B1860D4F84C01C0F30A3009F026FCAB
S214445DC0034909F077FC074B186010BDC083402098
S214445DD0CDCCCC3DCDCC4C40781C40200AD7233C7F
S214445DE0741C4020701C402008B5FFF767FEBDE8D1
S214445DF00840FFF7C4BF7047704708B5084BD3F850
S214445E006801C0F30F1009F001FC064909F052FC82
S214445E10054909F045FB09F013FE044B186008BD1C
S214445E20C0834020CDCC4C3D00C0CC449C1B40207D
S214445E3008B5084BB3F86C0109F0E8FB064909F0CD
S214445E4039FC064909F02CFB09F0FAFD044B1860AE
S214445E5008BD00BFC08340200AD7A33C00C02344EB
S214445E60A01B402008B5094BD3F87001C0F30F10AF
S214445E7009F0CCFB064909F01DFC064909F010FB65
S214445E8009F0DEFD044B186008BD00BFC083402007
S214445E90CDCC4C3D00C0CC44901B402008B5084BAC
S214445EA0B3F8740109F0B2FB064909F003FC06494D
S214445EB009F0F6FA09F0C4FD044B186008BD00BFAB
S214445EC0C08340200AD7A33C00C02344901B4020F4
S214445ED008B5FFF7BDFCFFF7DFFCFFF701FDFFF752
S214445EE022FDFFF723FEFFF745FEFFF768FEFFF7A8
S214445EF084FFFFF79DFFFFF7B5FFBDE80840FFF7B7
S214445F00CDBF1A4B186810B5C830194C09F07AFB47
S214445F10184909F083FC08F01FFF0DF025FF09F02F
S214445F204BFA154B1549A4F87801186809F0BAFAE3
S214445F30134909F073FC08F00FFF0DF015FF09F044
S214445F403BFA104BA4F87A011B68A4F87C310E4B3C
S214445F50186808F001FF0DF007FF09F02DFA0B4B07
S214445F6084F87E011B6884F87F3110BD581C40209D
S214445F70C0834020CDCCCC3D541C402000C023449C
S214445F800AD7A33C501C40204C1C4020481C4020B0
S214445F90224B234A1B68234982F88431224B0968E2
S214445FA01B6809029B0201F4407103F480630B43AF
S214445FB01E490968C90201F4C0510B431C490968CB
S214445FC0490301F4C0410B431A490968C90301F463
S214445FD0C0310B43D2F8841121F4FF3121F480718F
S214445FE00B431549C2F88431144B09681B6801F009
S214445FF00701A2F88A31124B1B68A2F88831114B6C
S2144460001B78DB0003F008030B4392F88C1121F055
S2144460100F010B4382F88C31704700BFD81D4020D7
S214446020C0834020381C4020341C4020301C402074
S2144460302C1C4020281C4020E41D4020241C4020CA
S214446040201C4020DE1D4020184B1949186810B506
S21444605009F0E4FB174C08F07FFE0DF085FE09F0CE
S214446060ABF9154B1249A4F89001186809F0D6FB11
S21444607008F072FE0DF078FE09F09EF90F4B0C49BD
S214446080A4F89201186809F0C9FB08F065FE0DF003
S2144460906BFE09F091F90A4BA4F894011B7884F836
S2144460A09731084B1B7884F8963110BD8C1D4020E0
S2144460B0CDCCCC3DC0834020901D4020001E4020C7
S2144460C0891D4020881D4020044B054993F8E8214B
S2144460D0096861F3000283F8E8217047C0834020D2
S2144460E0FC1B4020124B13491A68134B02F0010262
S2144460F01B6803F0010343EA4203104A126802F0A5
S214446100010243EA82030E4A126802F0010243EA9D
S214446110C2030C4A126802F0010243EA021391F8E1
S214446120EC2122F01F02134381F8EC31704700BF84
S214446130F41B4020C0834020F81B4020F01B402026
S214446140EC1B4020E81B4020124B13491A68134BA3
S21444615002F001021B6803F0010343EA4203104ABB
S214446160126802F0010243EA82030E4A126802F001
S214446170010243EAC2030C4A126802F0010243EAEF
S214446180021391F8F02122F01F02134381F8F031F4
S214446190704700BFE01B4020C0834020E41B4020E3
S2144461A0DC1B4020D81B4020D41B40200F4B1049FA
S2144461B01A68104B02F001021B6803F0010343EA1D
S2144461C042030D4A126802F0010243EA82030B4A74
S2144461D0126802F0010243EAC20391F8F42122F065
S2144461E00F02134381F8F431704700BFCC1B4020A4
S2144461F0C0834020D01B4020C81B4020C41B4020E6
S21444620038B51A4B1A4C19681A4B186809F04AF9EB
S214446210194B05461949186809F044F9184909F014
S214446220FDFA08F099FD0DF09FFD09F0C5F8154BF1
S2144462301549A4F8F801186809F034F9134909F027
S214446240EDFA08F089FD0DF08FFD09F0B5F8104918
S214446250A4F8FA01284609F0E1FA08F07DFD0DF0AD
S21444626083FD09F0A9F8A4F8FC0138BD7C1740204A
S214446270C0834020981F4020801740200000484399
S2144462800AD7233C7817402000C023440AD7A33CAF
S214446290CDCCCC3D1C4B1D49186810B509F0BEFA50
S2144462A01B4C08F059FD0DF05FFD09F085F8194BBD
S2144462B0A4F89801186808F04FFD0DF055FD09F054
S2144462C07BF8154B1549A4F89A01186809F0EAF8C2
S2144462D0134909F0A3FA08F03FFD0DF045FD09F017
S2144462E06BF8104B1049A4F89C01186809F0DAF8CA
S2144462F00E4909F093FA08F02FFD0DF035FD09F02C
S2144463005BF8A4F89E0110BD901F4020CDCCCC3D38
S214446310C08340205C1940208018402000C023449D
S2144463200AD7A33C341B4020000048430AD7233CEA
S214446330114B1249186810B509F070FA104C08F061
S2144463400BFD0DF011FD09F037F80E4B0E491B7886
S214446350A4F8A001A4F8A2310C4B186809F0A2F8DE
S2144463600B4909F05BFA08F0F7FC0DF0FDFC09F068
S21444637023F8A4F8A40110BDE4184020CDCCCC3DAD
S214446380C0834020EE18402000C0234468184020B4
S2144463900AD7A33C184B1949186810B509F082F877
S2144463A0174909F03BFA174C08F0D6FC0DF0DCFC14
S2144463B009F002F8144B1549A4F8A801186809F026
S2144463C071F8134909F02AFA08F0C6FC0DF0CCFC23
S2144463D008F0F2FF0F4BA4F8AA011B6884F8AC310E
S2144463E00D4B1A680D4B1B6803F00F0343EA021368
S2144463F084F8AD3110BD00BFF01C402000C02344DB
S2144464000AD7A33CC0834020001D402000C0CC4493
S214446410CDCC4C3D001C4020B41B4020B81B402033
S214446420164B1749186810B509F03CF8154909F099
S214446430F5F9154C08F090FC0DF096FC08F0BCFFFE
S214446440124B1349A4F8B001186809F02BF8114907
S21444645009F0E4F908F080FC0DF086FC08F0ACFF87
S2144464600D4BA4F8B2011A680C4B1B6803F00F03DB
S21444647043EA021384F8B43110BD00BF941C402094
S21444648000C023440AD7A33CC0834020981C402025
S21444649000C0CC44CDCC4C3DA41B4020A81B40207F
S2144464A0174B186810B500F28F20164C09F0AAF85E
S2144464B0154909F0B3F908F04FFC0DF055FC08F007
S2144464C07BFF124BA4F8B801186800F2666009F026
S2144464D099F80F4909F0A2F908F03EFC0DF044FC87
S2144464E008F06AFF0B4BA4F8BA011A680A4B1B68FB
S2144464F003F00F0343EA021384F8BC3110BD00BF17
S214446500A01B4020C08340200AD7A33C9C1B4020AD
S214446510CDCC4C3D941B4020981B4020174B18680C
S21444652010B500F28F20164C09F06CF8154909F0A6
S21444653075F908F011FC0DF017FC08F03DFF124BFE
S214446540A4F8C001186800F2666009F05BF80F49C9
S21444655009F064F908F000FC0DF006FC08F02CFF86
S2144465600B4BA4F8C2011A680A4B1B6803F00F03CE
S21444657043EA021384F8C43110BD00BF901B402088
S214446580C08340200AD7A33C8C1B4020CDCC4C3D36
S214446590841B4020881B40200A4A0B4B126883F811
S2144465A0E0210A4A126883F8E121094A126883F80E
S2144465B0E221084A126883F8E321074A1268C3F8BE
S2144465C0E4217047801B4020C08340207C1B402031
S2144465D0781B4020741B4020701B40204D4B4E4A75
S2144465E01B78012B5BD14D4B4D491B6809689B00BA
S2144465F001F0030103F00C030B434A4909680901FF
S21444660001F030010B43484909688901C9B20B437C
S21444661046490968090201F440710B434449096834
S214446620890201F440610B4342490968090301F4B5
S21444663040510B4340490968890389B20B433F499B
S2144466400968090401F440310B433D49096889044B
S21444665001F440210B43D2F8C811090D09050B4338
S214446660C2F8C831374B1B7803F00301364B1B780E
S21444667003F003031B0143EA81133449097801F00C
S214446680030143EA0123B2F8CA1121F47C710B4397
S214446690A2F8CA312E4B1B8882F8CC317047002BA7
S2144466A033D12C4B2C491B6809689B0001F003012D
S2144466B003F00C030B4329490968090101F0300132
S2144466C00B43274909688901C9B20B432549096820
S2144466D0090201F440710B4323490968890201F415
S2144466E040610B4321490968090301F440510B43B7
S2144466F01F490968890389B20B431E49096809047E
S21444670001F440310B431C49A0E7023B012BA9D8B6
S214446710C7E700BF3A184020C08340201C1A4020D8
S214446720201A4020181A4020141A4020101A4020DC
S2144467300C1A4020081A4020041A4020001A402010
S214446740FC194020031B4020021B4020041B402011
S214446750001B4020401D4020441D40203C1D40203E
S214446760381D4020341D4020301D40202C1D402024
S214446770281D4020241D4020201D4020124B134934
S2144467801B7803F00302124B1B7803F0030343EA1F
S2144467908203104A127802F0030243EA02130E4AB6
S2144467A0127802F0030243EA82130C4A127802F08B
S2144467B0030243EA0223B1F8D02102F47C42134395
S2144467C0A1F8D031704700BF431B4020C08340200F
S2144467D0441B4020421B4020411B4020401B40207D
S2144467E0094B0A491A680A4B02F001021B6803F077
S2144467F0030343EA820391F8DC2122F007021343A1
S21444680081F8DC31704700BF381B4020C0834020ED
S2144468103C1B402038B5344B344D1868C83008F01B
S214446820F1FE334908F0FAFF08F096FA0DF09CFAA8
S214446830304B1C68304B64001B6804F0020403F0C1
S21444684001031C432D4B1B689B0003F004031C43AD
S2144468502B4B1B68DB0003F008031C43294B1B68C7
S2144468601B01DBB21C43284B1B681B0203F440731A
S2144468701C43264B1B689B0203F4E0531C43244BE7
S2144468801B685B0303F4C0431C4308F095FD214B8F
S214446890214903EAC0331C43D5F8D43103F00043FE
S2144468A01C431E4BC5F8D441186808F0FBFD10493C
S2144468B008F0B4FF08F050FA0DF056FA08F07CFDE4
S2144468C0174B1549A5F8D801186808F0EBFD084998
S2144468D008F0A4FF08F040FA0DF046FA08F06CFD04
S2144468E0A5F8DA0138BD00BF0C1B4020C083402009
S2144468F00AD7233C281B40202C1B4020241B402026
S214446900201B40201C1B4020181B4020141B4020EA
S214446910101B40200080FF7F00004843081B402097
S214446920341B4020274B2849186810B508F0BAFD98
S214446930264908F073FF264C08F00EFA0DF014FAB8
S21444694008F03AFD234B2449A4F85402186808F08A
S214446950A9FD224908F062FF08F0FEF90DF004FA9A
S21444696008F02AFD1E4BA4F856021B68A4F85832B9
S2144469701C4B1A681C4B02F003021B6803F001030D
S21444698043EA4203194A126802F0030243EAC20386
S214446990174A126802F0010243EA4213154A126883
S2144469A002F00F0243EA8213134A126802F00F02FF
S2144469B043EA8223B4F85A2202F440421343A4F82A
S2144469C05A3210BD2C1E4020000048430AD7233CB0
S2144469D0C0834020F01C402000C023440AD7A33C78
S2144469E0F41A4020301C4020EC1A4020281C40203A
S2144469F0E01A4020DC1A4020D81A4020244B4FF09E
S214446A008E41244A1B6812681B0102F00F02DBB257
S214446A101343214A1268120202F4706213431F4A57
S214446A201268120302F4805213431D4A126852033A
S214446A3002F4C04213431B4A1268D20302F4C03223
S214446A401343194A1268520410B502F0FF72174CE9
S214446A501343D4F85C2202F07E421343C4F85C32FB
S214446A60134B186808F01EFD08F076F90DF07CF913
S214446A7008F0A2FC0F4BA4F860021A680E4B1B6881
S214446A8003F00F0343EA021384F8623210BD00BFDA
S214446A90D01A4020D41A4020CC1A4020C81A40208D
S214446AA02C1C4020C01A4020D81D4020C0834020C3
S214446AB0301E4020B81A4020BC1A4020114B10B556
S214446AC0186808F049F9104C0DF04EF908F074FCBB
S214446AD00E4B84F864021B6884F865320C4B1B68C2
S214446AE0A4F866320B4B1B68A4F868320A4B1A6843
S214446AF00A4B1B6803F00F0343EA021384F86A3216
S214446B0010BD00BF4C1C4020C0834020481C402081
S214446B10201C4020241C4020A01A4020A41A4020B8
S214446B201C4A936CC3F3473382F89C32B2F84A301B
S214446B30C3F3471382F89D32B2F84230C3F3C71307
S214446B4082F89E3292F85C3082F89F32124B196873
S214446B50124B01F007011B6803F0010343EA4103AB
S214446B600F49097801F0010143EA01130D49096808
S214446B7001F00F0143EA41130B49096801F00F0184
S214446B8043EA4123B2F8A01201F460410B43A2F851
S214446B90A0327047C0834020E41D4020B01D4020F2
S214446BA0DE1D40209C1A4020981A4020174B186837
S214446BB010B500F28F20164C08F024FD154908F055
S214446BC02DFE08F0C9F80DF0CFF808F0F5FB124B8F
S214446BD0A4F83402186800F2666008F013FD0F4902
S214446BE008F01CFE08F0B8F80DF0BEF808F0E4FB18
S214446BF00B4BA4F836021A680A4B1B6803F00F03C3
S214446C0043EA021384F8383210BD00BF941A402079
S214446C10C08340200AD7A33C901A4020CDCC4C3D9C
S214446C20881A40208C1A4020174B186810B500F27A
S214446C308F20164C08F0E6FC154908F0EFFD08F0E6
S214446C408BF80DF091F808F0B7FB124BA4F83C0211
S214446C50186800F2666008F0D5FC0F4908F0DEFDBF
S214446C6008F07AF80DF080F808F0A6FB0B4BA4F871
S214446C703E021A680A4B1B6803F00F0343EA0213EA
S214446C8084F8403210BD00BF841A4020C0834020A0
S214446C900AD7A33C801A4020CDCC4C3D781A4020DD
S214446CA07C1A4020174B186810B500F28F20164CFB
S214446CB008F0A8FC154908F0B1FD08F04DF80DF0B1
S214446CC053F808F079FB124BA4F84402186800F213
S214446CD0666008F097FC0F4908F0A0FD08F03CF801
S214446CE00DF042F808F068FB0B4BA4F846021A680D
S214446CF00A4B1B6803F00F0343EA021384F8483236
S214446D0010BD00BF741A4020C08340200AD7A33C5D
S214446D10701A4020CDCC4C3D681A40206C1A402056
S214446D20174B186810B500F28F20164C08F06AFC12
S214446D30154908F073FD08F00FF80DF015F808F043
S214446D403BFB124BA4F84C02186800F2666008F04D
S214446D5059FC0F4908F062FD07F0FEFF0DF004F8F9
S214446D6008F02AFB0B4BA4F84E021A680A4B1B6821
S214446D7003F00F0343EA021384F8503210BD00BFF9
S214446D80641A4020C08340200AD7A33C601A40209F
S214446D90CDCC4C3D581A40205C1A40204C4B4FF00A
S214446DA084412DE9F04FDFF864A187B01B788AF858
S214446DB0C432484B1B788AF8C532474B186808F0EB
S214446DC071FB4FF0834108F075FC07F0C5FF0CF0EB
S214446DD0CBFF424B8046894618684FF0844108F002
S214446DE061FB4FF0834108F065FC07F0B5FF0CF0FB
S214446DF0BBFF3B4B06460F4693F800B0394B3A4927
S214446E000BF0010B186808F04DFB384908F006FDF6
S214446E1007F0A2FF0CF0A8FF354B364A1B78CDE9A5
S214446E20000110683449059308F03CFB334908F0E8
S214446E30F5FC07F091FF0CF097FF314A1478314A7D
S214446E4004F001041578240305F00105CDE9020198
S214446E504946404608F0B0FAC0F30900AD02394648
S214446E600543BAF8C60200F4784005433046AAF80B
S214446E70C6524FEA8B2508F09FFAC0F3090BDDE9AA
S214446E80000108F099FA204A059B45EA0B0B02EAF2
S214446E90C02203F001034BEA020BDAF8C8224BEA9D
S214446EA0C35302F07F421343DDE90201CAF8C832F5
S214446EB008F082FAC0F30B000443BAF8CC0200F49C
S214446EC060400443AAF8CC4207B0BDE8F08F00BF48
S214446ED03919402038194020341940202C194020B4
S214446EE0281940202419402033336F410AD7233CC5
S214446EF0201940201C194020CDCCCC42CDCC4C3D52
S214446F00181940203019402000F87F00C0834020E4
S214446F10124B1A8DC3F86C22114A1168114A01F0BB
S214446F200F01126802F00F0242EA011293F82B1086
S214446F3042EA0122A3F870229A8DC3F874220A4AC0
S214446F4011680A4A126802F00F0242EA011283F8F4
S214446F507822074A126883F879227047C083402013
S214446F60081F40200C1F4020F81E4020FC1E4020D6
S214446F70F41E4020114B1A8EC3F87C22104A116826
S214446F80104A126802F00F0242EA011283F8802285
S214446F900D4A126883F881229A8EC3F884220B4ADB
S214446FA011680B4A126802F00F0242EA011283F893
S214446FB08822084A126883F889227047C083402092
S214446FC0E81E4020EC1E4020E41E4020D81E4020F0
S214446FD0DC1E4020D41E40200F4B1A8FC3F88C2250
S214446FE00E4A11680E4A126802F00F0242EA011273
S214446FF083F890229A8FC3F894220A4A11680A4A60
S214447000126802F00F0242EA011283F89822074AF5
S214447010126883F899227047C0834020C81E4020D7
S214447020CC1E4020BC1E4020C01E4020B81E40201F
S214447030334B3449F0B51E78334B06F0030691F8CB
S2144470405C201D78314B42EA062205F003051C6895
S2144470502F4B42EA8522240318682E4BA4B2000420
S2144470601B78224300F4702003F003072A4B104396
S2144470701B7803F0030343EA8703284F3F7807F05F
S214447080030743EA0713264F3F7807F0030743EA0C
S2144470908713244F3F7807F0030743EA0723224F1A
S2144470A03F7807F0030743EA8723204F3F7807F0EB
S2144470B0030743EA07331E4F3F68BF03BFB23B4351
S2144470C01C4F43EA06433F7843EA864307F00307E8
S2144470D043EA065343EA865343EA066343EA87632E
S2144470E0D1F8107207F070473B43C1F81032D1F81C
S2144470F014321B0D1B051843C1F81402F0BD00BF23
S214447100201E4020C0834020211E4020B419402029
S214447110B0194020231E4020221E4020241E40201A
S214447120251E4020261E4020281E4020271E402084
S2144471301C1E40204518402008B5FFF7F1FCBDE86A
S2144471400840FFF775BF214B214A70B51C68214B98
S214447150B2F8605004F00F04186892F8603005F4F2
S214447160FF4592F8641000F00F0003F07F032B43B2
S214447170156E05F4FF052B43B2F86250C5F3C115EE
S21444718043EAC55392F86350C5F3410643EA46635F
S214447190C5F3C106C5F3411543EAC66343EA4573DE
S2144471A0D2F8185205F000452B43C2F8183201F0C5
S2144471B03F03B2F81C1243EA841301F4404143EA05
S2144471C080230B43A2F81C3270BD00BFAC1D402088
S2144471D0C0834020A81D40201D4B1E4A1B681268D1
S2144471E09B001D4902F0030203F00C0313431B4AA1
S2144471F01268120102F030021343194A12689201CF
S214447200D2B21343174A1268120202F4407213436E
S214447210154A1268920202F440621343134A1268F3
S214447220120302F440521343114A1268920302F4C2
S214447230703213430F4A1268920402F470121343D6
S214447240D1F83022920D92051343C1F8303270477C
S214447250A0194020A4194020C08340209C194020F7
S2144472609819402094194020901940208C194020A9
S21444727088194020841940201A4B1B49186810B5B9
S21444728008F0CCFA194C07F067FD0CF06DFD08F0D9
S21444729093F8174B1449A4F82002186808F0BEFA6D
S2144472A007F05AFD0CF060FD08F086F8114BA4F880
S2144472B02202188808F0AAF90B4908F0AFFA07F03A
S2144472C04BFD0CF051FD08F077F80B4BA4F8240264
S2144472D01A680A4B1B6803F00F0343EA021384F848
S2144472E0263210BD8C1D4020CDCCCC3DC0834020E2
S2144472F0901D40208A1D4020F01D4020F41D402053
S214447300124A92F8783010B582F82832104BD2F8E8
S21444731028421878B2F87A30C3F38701936FC3F3E0
S21444732009231B0243EA81430A49097801F00F0105
S21444733043EA8163084921400B43C2F8283292F855
S2144473402C3260F3030382F82C3210BDC0834020F5
S2144473507E1940207F194020FF0000C0094B0A498F
S2144473601A680A4B02F007021B6803F0030343EA59
S214447370820391F8A42222F01F02134381F8A43218
S214447380704700BF301C4020C0834020281B40204C
S214447390064B10B5064C186808F052FBB4F8A832F1
S2144473A060F30903A4F8A83210BD00BF4C1C40206B
S2144473B0C0834020094B0A4A1B7812789B0009492F
S2144473C002F0030203F00C03134391F8AC2222F0BC
S2144473D00F02134381F8AC32704700BF7A1940203D
S2144473E07B194020C0834020044B054993F8B022C3
S2144473F0097861F3020283F8B0227047C0834020C4
S21444740079194020044B054993F8B422097861F36E
S214447410030283F8B4227047C08340207819402082
S214447420F8B53D4B3D4D1B783D4985F8B8323D4B4C
S214447430186808F0F3F907F08FFC0CF095FC07F099
S214447440BBFF394A394B03EA40231068D5F8B822C3
S214447450000200F480700343354810400343C5F8E7
S214447460B832344B1B7885F8BC32334B1C68334BEC
S21444747004F003041F68324B07F001071E68314BC3
S21444748044EA870406F00106186808F0BBF84FF093
S214447490814108F00FF908F0D3FA2B4A2B4B44EA03
S2144474A0C606D5F8BC1203EA00231068284A8005AD
S2144474B095F8C04200F4800024F00F04034310689B
S2144474C0244A2643C005126800F4000085F8C062CA
S2144474D01206034302F0407213431F4A1268920690
S2144474E002F0406213431D4A1268120702F08052AB
S2144474F013431B4A1268520702F000521343194AB8
S2144475001268920702F080421343174A0A40134314
S214447510C5F8BC32F8BD00BF58194020C08340208F
S214447520CDCCCC3D901F4020541A402000FEFF0195
S214447530FF0000FE591940202C1A4020281A4020EB
S214447540241A40204C1A4020481A402000FF3F008E
S214447550441A4020301C40203C1A4020381A402010
S214447560341A4020301A4020FF000080084A094B55
S2144475701278094983F8D022084A0978127883F8A1
S214447580D12293F8D22261F3000283F8D2227047C4
S2144475906A194020C0834020681940206919402059
S2144475A0114B12491B6810B5114C84F8F032114B3C
S2144475B01B6884F8F132104B186807F073FF0F49C4
S2144475C008F02CF907F0C8FB0CF0CEFB07F0F4FEED
S2144475D00B4A94F8F4321278A4F8F20262F30003E9
S2144475E084F8F43210BD00BF6419402000C0234420
S2144475F0C0834020601940205C1940200AD7A33C31
S2144476005A194020F8B5204B204D186807F0FAFF69
S2144476104FF0814108F04EF808F012FA1C4B04462D
S2144476201F681C4BC4F30D0407F001071E681A4B71
S21444763044EA8734186844EAC63407F0E3FF4FF058
S214447640814108F037F808F0FBF9144AC0F30D03FB
S214447650A5F8EC421068124A800300F480400343C5
S2144476601068104AC003126800F4FF00D2050343B2
S21444767002F0FF421343D5F8E82202F000421343D7
S214447680C5F8E832F8BD00BF44194020C083402006
S214447690401940203C19402054194020501940209D
S2144476A04C194020481940200D4B0E4A1B780E4971
S2144476B082F8FC320D4B09781B7801F0010182F800
S2144476C0FD320B4B1B785B0003F002030B4392F82E
S2144476D0FE1221F003010B4382F8FE32704700BFCE
S2144476E017194020C0834020151940201619402001
S2144476F0141940200C4B0D4A1B680D4982F8F83289
S2144477000C4B09781B6801F0030182F8F9320A4BE6
S2144477101B789B0003F00C030B430849097843EAA3
S214447720011382F8FA32704710194020C083402073
S2144477300B1940200C1940200A19402009194020F2
S214447740F8B5254B254C1B78254F84F80033254B3C
S2144477501B7884F80133244B1878323007F056FFF0
S214447760014607F09FFE08F06BF9204984F80203AF
S2144477700E781F493F780D781E4907F001071E4BC7
S21444778008781E491A78303009781D4B49001B7812
S21444779001F03E01394394F8037327F03F07394319
S2144477A084F8031303F03F0102F01F0306F00F02B0
S2144477B043EA411343EAC22305F03F0243EAC23395
S2144477C000F03F0243EA4253D4F8042302F07842DE
S2144477D01343C4F80433F8BD08194020C08340203E
S2144477E00519402007194020061940200119402059
S2144477F000194020FF184020031940200419402057
S2144478000219402038B50C4B0C4C5D68284607F0EE
S214447810A3FA0CF0A9FA07F0CFFD0949C4F8E4022C
S214447820284607F0FBFF07F097FA0CF09DFA07F09E
S214447830C3FDC4F8E00238BD20464020C083402043
S214447840000008422DE9F74F374D384E686808F077
S214447850F7F886F80803A86808F0F2F8344986F87A
S2144478600903686907F01EFE324907F0D7FF08F09F
S214447870E7F88346A86908F0E3F82D490446E86922
S21444788007F010FE2B4907F0C9FFCBF3090B08F0AD
S214447890D7F88246286A08F0D3F825498146686AAC
S2144478A007F000FE234907F0B9FF08F0C9F8804600
S2144478B0A86A08F0C5F81E4900F00107E86807F012
S2144478C0F1FD1C4907F0AAFF08F0BAF8C0F3090313
S2144478D02869019308F0B4F8019B00F0010043EADC
S2144478E08023B6F80A0300F4784003431248A6F807
S2144478F00A33A30200EACA2A03F480634FEA4950D3
S21444790043EA0B0300F4001043EA0A03034343EA42
S2144479108853C6F80C3396F8103367F3000386F89A
S214447920103303B0BDE8F08F20464020C08340208B
S21444793066667241CDCC4C3D00F81F00084A094BA0
S2144479401278094983F83823084A0978127883F864
S214447950392393F83A2361F3000283F83A237047B5
S214447960FE184020C0834020FC184020FD184020CC
S214447970114B124A1B68124910B5124C127884F8FF
S2144479802833114B1B6884F8293394F82C3362F35C
S214447990000384F82C330D4B186807F083FD0C491C
S2144479A007F03CFF07F0D8F90CF0DEF907F004FDC9
S2144479B0A4F82A0310BD00BFF8184020EE18402053
S2144479C000C02344C0834020F4184020F0184020D0
S2144479D00AD7A33C284B294910B5294C1B7884F870
S2144479E02033284B186807F019FF07F0B5F90CF058
S2144479F0BBF907F0E1FC244A244B03EA4023106811
S214447A00D4F82023000200F480700343204810403A
S214447A10204A03431268C4F8203312021E4B02F471
S214447A2080721B7884F824331C4B1B685B0203F477
S214447A30C06313431A4A1268D20202F4C052134374
S214447A40184A1268520302F400521343164A126844
S214447A50920302F480421343144A1268D20302F497
S214447A60C0321343D4F8242322F4FF3222F4807223
S214447A701343C4F8243310BDEC184020CDCCCC3D81
S214447A80C0834020901F4020E818402000FEFF019D
S214447A90FF0000FEE0184020ED184020DC1840208F
S214447AA0D8184020D4184020D0184020CC18402065
S214447AB03A4B4FF084412DE9F047394E1B7886F80F
S214447AC01433384B1B7886F81533374B186807F051
S214447AD0E9FC4FF0834107F0EDFD07F0B1FF334B6F
S214447AE00446334993F800A0324B0AF0010A18685A
S214447AF007F0D8FC304907F091FE07F0A1FF2F4B62
S214447B0081462F4993F800802E4B08F001081868E8
S214447B1007F0C8FC2C4907F081FE07F091FF2B4B79
S214447B2005464FF084411F78294BC5F30B0507F0F3
S214447B300107186807F0B6FC4FF0834107F0BAFD1A
S214447B4007F07EFF234BC0F3090245EA0735187851
S214447B50C4F3090300F0010043EA8A2342EA802280
S214447B60B6F8160300F4784002431B4800EAC929D5
S214447B70A6F81623D6F8182343EA090302F07F42F0
S214447B8043EAC8531343C6F81833B6F81C3303F411
S214447B9060431D43A6F81C53BDE8F087C91840202F
S214447BA0C0834020C8184020BC184020B818402045
S214447BB033336F41B41840200AD7233CB0184020D2
S214447BC0CDCCCC42AC184020CDCC4C3DA81840205F
S214447BD0C4184020C018402000F87F002DE9F74F15
S214447BE0374D384E686807F02BFF86F85803A86868
S214447BF007F026FF344986F85903686907F052FCB3
S214447C00324907F00BFE07F01BFF8346A86907F0CE
S214447C1017FF2D490446E86907F044FC2B4907F052
S214447C20FDFDCBF3090B07F00BFF8246286A07F0ED
S214447C3007FF25498146686A07F034FC234907F064
S214447C40EDFD07F0FDFE8046A86A07F0F9FE1E49E2
S214447C5000F00107E86807F025FC1C4907F0DEFD44
S214447C6007F0EEFEC0F309032869019307F0E8FE27
S214447C70019B00F0010043EA8023B6F85A0300F45F
S214447C80784003431248A6F85A33A30200EACA2AA5
S214447C9003F480634FEA495043EA0B0300F40010B0
S214447CA043EA0A03034343EA8853C6F85C3396F828
S214447CB0603367F3000386F8603303B0BDE8F08FA3
S214447CC020464020C083402066667241CDCC4C3D61
S214447CD000F81F000D4B0E4A1B780E4982F83433C9
S214447CE00D4B09781B7801F0010182F835330B4BB4
S214447CF01B785B0003F002030B4392F8361321F023
S214447D0003010B4382F83633704700BFA718402060
S214447D10C0834020A5184020A6184020A418402020
S214447D200C4B0D4A1B680D4982F830330C4B0978CE
S214447D301B6801F0030182F831330A4B1B789B0021
S214447D4003F00C030B430849097843EA011382F80D
S214447D5032337047A0184020C083402098184020F3
S214447D609C1840209718402096184020F8B5254B7C
S214447D70254C1B78254F84F85033254B1B7884F8C4
S214447D805133244B1878323007F040FC014607F054
S214447D9089FB07F055FE204984F852030E781F49A4
S214447DA03F780D781E4907F001071E4B08781E4998
S214447DB01A78303009781D4B49001B7801F03E0193
S214447DC0394394F8537327F03F07394384F85313E1
S214447DD003F03F0102F01F0306F00F0243EA41138B
S214447DE043EAC22305F03F0243EAC23300F03F02AF
S214447DF043EA4253D4F8542302F078421343C4F877
S214447E005433F8BD95184020C08340209218402033
S214447E1094184020931840208E1840208D184020F7
S214447E208C18402090184020911840208F184020ED
S214447E3008B5FFF785FCBDE80840FFF797BF38B59F
S214447E400C4B0D4C5D68284606F086FF0BF08CFF05
S214447E5007F0B2FA0949C4F84C03284607F0DEFC9A
S214447E6006F07AFF0BF080FF07F0A6FAC4F8480342
S214447E7038BD00BF20464020C08340200000084252
S214447E8008B5FEF73EF8FEF783F8FEF7DDF8FEF792
S214447E901BF9FEF727F9FEF757F9FEF787F9FEF7C1
S214447EA0AFF9FEF777FAFEF7BBFAFEF7F9FAFEF7F4
S214447EB035FBFEF771FBFEF791FBFEF75FFCFEF722
S214447EC08FFCFEF7A7FCFEF72DFDFEF797FDFEF7A9
S214447ED0F5FDFEF76BFEFEF7A7FEFEF7E3FEFEF7A4
S214447EE01FFFFFF715F8FFF745F8FFF775F8FFF79C
S214447EF02AF9FFF7C1F9FFF703FAFFF76DF9FFF721
S214447F002DFAFFF745FAFFF755FAFFF76DFAFFF734
S214447F1079FAFEF743FFFFF775FCFFF7C9FDBDE8A6
S214447F200840FFF78CBF114B11491B6810B5114C24
S214447F3084F86433104B1B6884F865330F4B186819
S214447F4007F0B0FA0E4907F069FC06F005FF0BF09F
S214447F500BFF07F031FA0B4A94F868331278A4F80A
S214447F60660362F3000384F8683310BD8818402023
S214447F7000C02344C08340208418402080184020FA
S214447F800AD7A33C7D1840200D4B0E4A1B780E4959
S214447F9082F870330D4B09781B7801F0010182F8A2
S214447FA071330B4B1B785B0003F002030B4392F8D0
S214447FB0721321F003010B4382F87233704700BFFB
S214447FC07C184020C08340207A1840207B184020EC
S214447FD0791840200C4B0D4A1B780D4982F86C33B7
S214447FE00C4B09781B7801F0030182F86D330A4B79
S214447FF01B789B0003F00C030B430849097843EABB
S214448000011382F86E33704778184020C0834020AE
S2144480107618402077184020751840207418402061
S214448020114B12491B6810B5114C84F87433114B2C
S2144480301B6884F87533104B186807F033FA0F49F9
S21444804007F0ECFB06F088FE0BF08EFE07F0B4F962
S2144480500B4A94F878331278A4F8760362F3000354
S21444806084F8783310BD00BF7018402000C0234405
S214448070C08340206C184020681840200AD7A33C90
S214448080641840200D4B0E4A1B780E4982F87C3308
S2144480900D4B09781B7801F0010182F87D330B4BB8
S2144480A01B785B0003F002030B4392F87E1321F027
S2144480B003010B4382F87E33704700BF63184020A9
S2144480C0C083402061184020621840206018402039
S2144480D00C4B0D4A1B680D4982F880330C4B0978CB
S2144480E01B6801F0030182F881330A4B1B789B001E
S2144480F003F00C030B430849097843EA011382F85A
S214448100823370475C184020C08340205518402076
S21444811058184020541840205318402008B5FFF7FC
S21444812025FAFFF73DFAFFF77BF9FFF76BFAFFF7FF
S21444813089FBFFF7B9FAFFF7DDFAFFF7FFFBFFF716
S21444814017FCFFF747FCFFF749FDFFF7C3FDFFF7B2
S214448150E7FDFFF7E8FEFFF717FFFFF73BFFFFF7E4
S2144481605FFFFFF78FFFBDE80840FFF7B1BF074A40
S2144481700020074BD2F87811D2F87C219962DA6253
S214448180044B93E80600FBF74FBC00BFC083402077
S2144481904887402074744600144A154892F885115E
S2144481A092F8843110B4C1F3010480F8283001F009
S2144481B01C03C1F34111234380F82930D2F884319B
S2144481C0C3F3C13492F88C31C3F3C003DB0143EAF2
S2144481D084030B4380F82A30D2F88831C3620020E7
S2144481E0044B10BC93E80600FBF71EBCC08340203B
S2144481F0488740207C7446000B4A00200B4BD2F83C
S21444820090119962B2F8941183F82C1092F8961152
S21444821092F8972183F82D1083F82E20044B93E888
S2144482200600FBF701BC00BFC083402048874020BF
S2144482309C744600064B0020064A93F8E831C3F384
S214448240000382F82830044B93E80600FBF7ECBBA7
S214448250C083402048874020A4744600084B002032
S21444826093F8EC31C3F3000203F01E031343054AAC
S21444827082F82830044B93E80600FBF7D5BB00BFD2
S214448280C083402048874020AC744600084B0020FA
S21444829093F8F031C3F3000203F01E031343054A78
S2144482A082F82830044B93E80600FBF7BDBB00BFBA
S2144482B0C083402048874020B4744600084B0020C2
S2144482C093F8F431C3F3000203F00E031343054A54
S2144482D082F82830044B93E80600FBF7A5BB00BFA2
S2144482E0C083402048874020BC744600064A00208D
S2144482F0064BD2F8F811B2F8FC2199629A85044BE1
S21444830093E80600FBF790BBC08340204887402094
S214448310C474460008B50A4B50200A4AD3F8A8113C
S21444832093F8AC31283211600821137103F08CFEA7
S214448330054B002093E80600BDE80840FBF774BBF5
S214448340C08340204887402044744600094B0020A0
S2144483500949D3F8B02193F8B4318A6203F0F002A5
S214448360C3F30303134381F82F30044B93E806000A
S214448370FBF75ABBC0834020488740204C744600D5
S214448380094B00200949D3F8B82193F8BC318A62D6
S21444839003F0F002C3F30303134381F82F30044B76
S2144483A093E80600FBF740BBC08340204887402044
S2144483B054744600094B00200949D3F8C02193F869
S2144483C0C4318A6203F0F002C3F30303134381F813
S2144483D02F30044B93E80600FBF726BBC0834020AF
S2144483E0488740205C7446000A4A00200A4BD2F86C
S2144483F0E01192F8E421996283F82C2083F82D202A
S21444840083F82E2083F82F20044B93E80600FBF7CE
S2144484100BBB00BFC083402048874020947446006E
S214448420254A264992F8C831C3F3010003F0FC03F9
S214448430034310B481F8283092F8C931C3F30100DD
S21444844003F0FC03034392F8CA0181F82930C0F3D1
S214448450010400F00C0323438409C0F3011081F89F
S2144484602A3092F8CB3103F003039B0143EA84039A
S214448470034381F82B3092F8CC3181F82C3092F8B3
S214448480CD3103F03800C3F30203034381F82D30A3
S21444849092F8CE31C3F38300D2F8CC31C3F383339E
S2144484A043EA0013002081F82F30054B10BC93E8B4
S2144484B00600FBF7B9BA00BFC08340204887402077
S2144484C0647446000B490C4A91F8D031C3F301005A
S2144484D003F0FC030343002082F8283091F8D1319E
S2144484E0C3F3010382F82930044B93E80600FBF7F4
S2144484F09BBA00BFC083402048874020847446000F
S214448500084B002093F8DC3103F00402C3F3010364
S2144485101343054A82F82830044B93E80600FBF7D9
S21444852083BA00BFC0834020488740208C744600EE
S2144485301049114A91F8D431C3F3000003F0FE0306
S214448540034382F8283091F8D53103F07C00C3F316
S21444855001030343002082F82930D1F8D431C3F311
S214448560CF335385D1F8D831D362044B93E8060011
S214448570FBF75ABAC0834020488740206C744600B4
S2144485801B4938B51B4CD1F8543204F5FE52B1F8A9
S2144485905802136041F6C473E05291F85A32C3F35A
S2144485A04100C3F3C1050543C3F30000C3F34013BE
S2144485B040EA850040EA430341F6C670235491F8E6
S2144485C05B32C3F38300B1F85A3241F6C771C3F342
S2144485D0831343EA001313206354082103F09DFEDB
S2144485E0054B012093E80600BDE83840FBF71CBA6B
S2144485F0C083402048874020147546002149224BBA
S21444860091F85C0203F5FE5210B500F0F004C0F396
S21444861003002043107091F85D0200F07004C0F32C
S2144486200300204341F6C174185541F6C274D1F88C
S2144486305C02C0F3C130185541F6C374B1F85E020B
S214448640C0F34700185541F6C470B1F8604291F83B
S21444865062121C5441F6C57000241C5401F0F0000C
S214448660C1F30301014341F6C7701954082114208D
S21444867003F053FE054B012093E80600BDE8104086
S214448680FBF7D2B9C0834020488740201C7546007B
S214448690154B164903F5FE5291F8640210B5107056
S2144486A0002441F6C1701C5441F6C270B1F86642CB
S2144486B01C5241F6C470B1F8684291F86A121C52D2
S2144486C001F0F000C1F30301014341F6C7701954A9
S2144486D00821152003F021FE054B012093E80600EF
S2144486E0BDE81040FBF7A0B948874020C08340202F
S2144486F02475460010B512490020124C01F5FE526E
S214448700D4F89C32136041F6C473C85494F8A1322A
S214448710C3F34300B4F8A032C3F3431343EA00134D
S21444872041F6C7700B540821162003F0F6FD064B9D
S214448730012093E80600BDE81040FBF775B900BF7A
S21444874048874020C08340204475460008B5FFF75C
S21444875071FDFFF783FDFFF799FDFFF7AFFDBDE819
S2144487600840FFF7C7BF08B5FDF73EFBF9F76BF8BF
S214448770FEF7E2FCBDE80840FFF7E8BF08B50E4840
S2144487800E4B00F5FE52D3F8341293F8383211608B
S21444879003F0F001C3F303030B4341F6C77143549C
S2144487A00821502003F0B9FD054B012093E806004C
S2144487B0BDE80840FBF738B948874020C0834020CE
S2144487C0F474460008B50E480E4B00F5FE52D3F836
S2144487D03C1293F84032116003F0F001C3F30303F4
S2144487E00B4341F6C77143540821512003F095FDCD
S2144487F0054B012093E80600BDE80840FBF714B992
S21444880048874020C0834020FC74460008B50E4884
S2144488100E4B00F5FE52D3F8441293F848321160DA
S21444882003F0F001C3F303030B4341F6C77143540B
S2144488300821602003F071FD054B012093E80600F3
S214448840BDE80840FBF7F0B848874020C083402086
S2144488500475460008B50E480E4B00F5FE52D3F894
S2144488604C1293F85032116003F0F001C3F3030343
S2144488700B4341F6C77143540821612003F04DFD74
S214448880054B012093E80600BDE80840FBF7CCB84A
S21444889048874020C08340200C754600194B1A4A2E
S2144488A003F5FE51B2F86C02088092F8701201F09B
S2144488B0F000C1F30301014341F6C270195441F676
S2144488C0C37192F87102585441F6C47092F8741207
S2144488D0195441F6C570195492F8781201F0F00014
S2144488E0C1F30301014341F6C6701954012092F8BE
S2144488F0791241F6C7729954044B93E80600FBF785
S21444890093B800BF48874020C08340202C7546005B
S214448910194B1A4A03F5FE51B2F87C02088092F8C5
S214448920801201F0F000C1F30301014341F6C27026
S214448930195441F6C37192F88102585441F6C470F2
S21444894092F88412195441F6C570195492F8881254
S21444895001F0F000C1F30301014341F6C670195417
S214448960012092F8891241F6C7729954044B93E851
S2144489700600FBF759B800BF48874020C083402014
S21444898034754600174B184A03F5FE51B2F88C026C
S214448990088092F8901201F0F000C1F303010143FD
S2144489A041F6C270195441F6C370D2F89412195461
S2144489B0090A41F6C470195492F8981201F0F0006E
S2144489C0C1F30301014341F6C6701954012092F8DD
S2144489D0991241F6C7729954044B93E80600FBF784
S2144489E023B800BF48874020C08340203C754600DB
S2144489F02848294990F8103201F5FE5270B5C3F361
S214448A00010403F0FC032343137090F81132C3F3BC
S214448A10010403F0FC03234341F6C1740B5541F6AD
S214448A20C27390F812422501A609C4F30114CD542A
S214448A3090F8135205F00303C5F381051B0143EA7E
S214448A408603234341F6C37443EA85130B5541F624
S214448A50C47390F81442CC5441F6C57490F8153259
S214448A6090F816021D01C3F3031300F00F000D55D2
S214448A7043EA001341F6C7700B5408214FF4AE6026
S214448A8003F04BFC054B012093E80600BDE870401C
S214448A90FAF7CABFC083402048874020CC744600BB
S214448AA02D4991F8180238B5C0F3001500F00803B4
S214448AB02A4C43EA4513C0F3020504F5FE522B4301
S214448AC0C0F34015C0F3801043EA851343EAC0134D
S214448AD041F6C1701370B1F81832C3F3C713235468
S214448AE041F6C270D1F81832C3F3C733235491F811
S214448AF01B02C0F3C103C0F34105C0F341101B0180
S214448B0043EA8503B1F81A52C5F3C1152B4343EA29
S214448B10801341F6C370235441F6C47091F81C3256
S214448B209B00235491F81D32C3F38300B1F81C32E2
S214448B3041F6C771C3F3831343EA00134FF4B0609E
S214448B406354082103F0E9FB054B012093E8060033
S214448B50BDE83840FAF768BFC083402048874020C5
S214448B60D47446001849194891F8303200F5FE523C
S214448B7010B5C3F3010403F0FC032343137091F8C8
S214448B80313203F03C04C3F30103234341F6C1747A
S214448B90035591F83232C3F38304D1F8303241F6A8
S214448BA0C771C3F3833343EA04134354082140F2A2
S214448BB0855003F0B2FB064B012093E80600BDE85F
S214448BC01040FAF731BF00BFC0834020488740209A
S214448BD0EC7446001149124B01F5FE52D3F82002BC
S214448BE010B5B3F82442106041F6C47093F82632A8
S214448BF00C5203F0F000C3F30303034341F6C7707B
S214448C000B5408214FF4B26003F087FB054B012058
S214448C1093E80600BDE81040FAF706BF48874020B0
S214448C20C0834020DC7446001749184891F828321F
S214448C3000F5FE5210B5137041F6C174D1F82832CF
S214448C40C3F30923035541F6C274B1F82A32C3F379
S214448C508103035591F82C3203F00F0491F82B321C
S214448C6041F6C771C3F3830343EA0413435408210C
S214448C7040F2955003F051FB054B012093E8060063
S214448C80BDE81040FAF7D0BEC08340204887402055
S214448C90E4744600084B0120084993F8A43203F0D4
S214448CA01C02C3F30103134341F6C3728B54044BB3
S214448CB093E80600FAF7B8BEC083402048874020B1
S214448CC04C754600084B41F6C271B3F8A822074BD0
S214448CD0C2F30120585441F6C37101205A54044B40
S214448CE093E80600FAF7A0BEC08340204887402099
S214448CF054754600054B0120054A93F8AC321B01D7
S214448D001370044B93E80600FAF78EBEC0834020E7
S214448D1008A740205C754600074B41F6C1720749D8
S214448D20012093F8B03203F007039B008B54044BA6
S214448D3093E80600FAF778BEC08340204887402070
S214448D4064754600074B41F6C1720749012093F803
S214448D50B432C3F303038B54044B93E80600FAF788
S214448D6063BE00BFC0834020488740206C754600E1
S214448D700D4843F65872B0F8D01208B549BA0B4BB2
S214448D8099521A4490F8D21243F65A70C9011954AB
S214448D900321322003F058F9054B022093E80600DD
S214448DA0BDE80840FAF740BEC083402048874020CC
S214448DB084754600114B43F65870114AB3F8F012C6
S214448DC049BA10B5115243F65A74B3F8F21293F8EE
S214448DD0F43249BA03F00103115343F65C719B0124
S214448DE0535402440521402002F0B7FF054B0220AD
S214448DF093E80600BDE81040FAF716BEC08340204C
S214448E00488740209C7546003048314A90F8BC322A
S214448E1090F8B81270B543F6587590F8BF4253555B
S214448E2043F65973D15443F65A71D0F8B832C3F363
S214448E304F235BBA5352C4F3801304F0100141EA43
S214448E40C301C4F30103194390F8B93203F0010394
S214448E5041EA4311C4F3810304F0200441EA831138
S214448E6043F65C73D15490F8C012C1F3800601F007
S214448E700803C1F3010143EA06130B4390F8BE12FC
S214448E80D0F8BC022343CC09C1F3801143EA8413CF
S214448E9043F65D741355C0F30D2343F65E74C0F376
S214448EA005409B001055642043EA410343F65F7136
S214448EB053542A44082103F0C7F8064B022093E88B
S214448EC00600BDE87040FAF7AFBD00BFC08340203F
S214448ED048874020747546001F4843F658721F4B17
S214448EE0B0F8EA12C1F3C71170B5995443F65974F1
S214448EF0D0F8E8121A44B0F8E852C1F3C731C5F3C3
S214448F000526195590F8ED4204F08001C4F3801408
S214448F10314343F65A76995543F65B715D54B0F83F
S214448F20EC5290F8E912C5F3052001F040010143E4
S214448F3043F65C7041EAC411195443F65D716A20E5
S214448F405D54062103F080F8054B022093E80600A2
S214448F50BDE87040FAF768BDC0834020488740208B
S214448F609475460038B52C4B43F658702B4AB3F8E4
S214448F70C412B3F8CC5249BA115293F8CA12CC0967
S214448F80C5F3032141EA041193F8CD42C4F3001417
S214448F9041EA441193F8C742C4F3800441EA841179
S214448FA093F8C942C4F3800441EAC41143F65A74A0
S214448FB0115543F65B71B3F8C642555443F65C719B
S214448FC0C4F30905C4F387045454B3F8C812D3F859
S214448FD0C832C1F30904C1F3051141EA851143F6C9
S214448FE05D755155C3F3CB21C3F3C34343EA04131E
S214448FF043F65E74135543F65F73D1540244082116
S214449000702003F021F8064B022093E80600BDE8E2
S2144490103840FAF709BD00BFC08340204887402047
S2144490207C754600284A43F658702849B2F80833F7
S2144490305BBA30B40B5243F65A73B2F80A03B2F82A
S2144490400C53C0F30904C0F38700C854C5F3012089
S21444905092F80B3303F00403034392F80D03C0F372
S214449060800043EAC00392F80E03C0F3401043EA7C
S214449070001392F8100300F0010043EA401343F64D
S2144490805B7043EA841343F65D740B5443F65C7397
S214449090D2F80C03CD54C0F3C923B2F80E23C0F360
S2144490A047309B010855900943EA923343F65E7273
S2144490B08B5443F65F73C8540220054B30BC93E888
S2144490C00600FAF7B1BC00BFC08340204887402062
S2144490D0BC754600104843F65871104A08B5B0F8B7
S2144490E0FC325BBA535290F8FE3203F00100C3F3ED
S2144490F0400343EA400343F65A7013540A444FF479
S2144491004470032102F029FE054B022093E8060032
S214449110BDE80840FAF788BCC08340204887402012
S214449120AC754600134843F65872134BB0F8F81221
S21444913049BA10B599521A4490F8FA1243F65A703E
S214449140C1F301041C54C1F3031443F65B70C1F32A
S21444915081011C5443F65C70195405214FF4547035
S21444916002F0FBFD054B022093E80600BDE81040E4
S214449170FAF75ABCC083402048874020A47546006E
S214449180254943F65872B1F8000338B540BA234B24
S21444919091F8034398521A44D1F8040304F00105A5
S2144491A0C4F34404C0F3C53040EAC51043F65A75C8
S2144491B0585543F65B75B1F80403C0F3451058554B
S2144491C043F65C7591F80403C0F304005855B1F8AF
S2144491D00603C0F3022500F4FC6045EAC40443F6E3
S2144491E05D755C5591F80543C4F3C304204343F6C8
S2144491F05E74185591F8020343F65F71585408217B
S2144492004FF4617002F020FF054B022093E80600FD
S214449210BDE83840FAF708BCC08340204887402061
S214449220B4754600094943F65870094AD1F8E03205
S2144492301BBA13500220D1F8E43243F65C711BBAD1
S2144492405350044B93E80600FAF7EEBBC083402025
S214449250488740208C7546000E4845F6F062B0F8C4
S214449260381308B549BA0C4B99521A4490F83A1335
S21444927045F6F260C1F3000119540321332002F08D
S214449280E3FE064B032093E80600BDE80840FAF7E1
S214449290CBBB00BFC083402048874020EC754600C7
S2144492A0114B45F6F060114AB3F8281349BA10B585
S2144492B0115245F6F264B3F82A1393F82C3349BA9C
S2144492C003F00103115345F6F4619B0153540244E1
S2144492D00521402002F09EFD054B032093E806003E
S2144492E0BDE81040FAF7A0BBC08340204887402022
S2144492F0D47546002248234A90F8201338B590F88F
S214449300243345F6F064135545F6F163D15445F6D7
S214449310F261D0F82033C3F34F235BBA535290F82C
S2144493202513C1F34013C1F380151B0143EAC5035B
S214449330C1F341052B4390F8215305F0010543EA58
S2144493404513C1F3C10501F0010143EA851345F60F
S214449350F4655355D0F824336520C3F3C13343EA48
S214449360811145F6F563D1542244082102F06CFE7F
S214449370054B032093E80600BDE83840FAF754BB93
S214449380C083402048874020CC75460038B52C4BD7
S21444939045F6F0602B4AB3F81413B3F81C5349BA95
S2144493A0115293F81A13CC09C5F3032141EA041168
S2144493B093F81D43C4F3001441EA441193F8174349
S2144493C0C4F3800441EA841193F81943C4F3800437
S2144493D041EAC41145F6F264115545F6F361B3F813
S2144493E01643555445F6F461C4F30905C4F387049B
S2144493F05454B3F81813D3F81833C1F30904C1F31B
S214449400051141EA851145F6F5655155C3F3CB215F
S214449410C3F3C34343EA041345F6F664135545F6CB
S214449420F763D15402440821712002F00DFE064B26
S214449430032093E80600BDE83840FAF7F5BA00BFC3
S214449440C083402048874020C475460008B5FEF7D0
S2144494508EFEFEF7A1FEFEF7CFFEFEF75BFFFEF79D
S21444946075FFFEF7C1FFFEF7DBFFFFF72BF8FFF7AC
S21444947047F8FFF75DF8FEF739FFFFF781F8FFF787
S214449480BDF8FFF705F9FFF79DF9FFF7BFF9FFF7BA
S214449490E1F9FFF773F9FFF701FAFFF739FAFFF737
S2144494A071FAFFF7A5FAFFF7FBFAFFF793FBFFF70E
S2144494B059FBFFF7B9FBFFF755FDBDE80840FFF73A
S2144494C065BF284A45F6F0602749B2F858335BBA78
S2144494D030B40B5245F6F263B2F85A03B2F85C5312
S2144494E0C0F30904C0F38700C854C5F3012092F8BA
S2144494F05B3303F00403034392F85D03C0F3800038
S21444950043EAC00392F85E03C0F3401043EA0013F4
S21444951092F8600300F0010043EA401345F6F36016
S21444952043EA841345F6F5640B5445F6F463D2F8DF
S2144495305C03CD54C0F3C923B2F85E23C0F347306E
S2144495409B010855900943EA923345F6F6628B54DC
S21444955045F6F763C8540320044B30BC93E8060032
S214449560FAF762BAC0834020488740200476460013
S214449570104845F6F061104A08B5B0F834335BBA83
S214449580535290F8363303F00100C3F3400343EAE2
S214449590400345F6F26013540A444FF444700321E2
S2144495A002F038FC054B032093E80600BDE808406B
S2144495B0FAF73ABAC083402048874020E47546000C
S2144495C0134845F6F062134BB0F8301349BA10B559
S2144495D099521A4490F8321345F6F260C1F30104E6
S2144495E01C54C1F3031445F6F360C1F381011C54C3
S2144495F045F6F460195405214FF4547002F00AFC01
S214449600054B032093E80600BDE81040FAF70CBA71
S214449610C083402048874020DC754600254945F6EF
S214449620F062B1F8500338B540BA234B91F853432F
S21444963098521A44D1F8540304F00105C4F3440480
S214449640C0F3C53040EAC51045F6F265585545F6B0
S214449650F365B1F85403C0F34510585545F6F46520
S21444966091F85403C0F304005855B1F85603C0F3B8
S214449670022500F4FC6045EAC40445F6F5655C55ED
S21444968091F85543C4F3C304204345F6F66418558D
S21444969091F8520345F6F7615854082140F2853054
S2144496A002F0D2FC054B032093E80600BDE83840A0
S2144496B0FAF7BAB9C083402048874020FC75460074
S2144496C008B5FFF75DFDBDE80840FFF7A7BF08B53E
S2144496D0F8F7BBF8FEF7ACFBBDE80840FFF7F0BF71
S2144496E0094945F6F060094AD1F848331BBA135085
S2144496F00320D1F84C3345F6F4611BBA5350044B5F
S21444970093E80600FAF790B9C08340204887402083
S214449710F4754600114B47F68860114AB3F8641353
S21444972049BA10B5115247F68A64B3F8661393F8EB
S214449730683349BA03F00103115347F68C619B0121
S214449740535402440521402002F0C2FB054B04203A
S21444975093E80600BDE81040FAF766B9C083402097
S214449760488740200C764600104847F68861104AE1
S21444977008B5B0F870335BBA535290F8723303F0BE
S2144497800100C3F3400343EA400347F68A60135498
S2144497900A444FF44470032102F09AFB054B04201C
S2144497A093E80600BDE80840FAF73EB9C083402077
S2144497B04887402014764600134847F68862134B81
S2144497C0B0F86C1349BA10B599521A4490F86E130F
S2144497D047F68A60C1F301041C54C1F3031447F6E8
S2144497E08B60C1F381011C5447F68C6019540521E3
S2144497F04FF4547002F06CFB054B042093E80600CB
S214449800BDE81040FAF710B9C0834020488740208E
S2144498101C76460008B50A4B49F6226209494020A0
S214449820B3F876335BBA8B520521074A02F0AEFB97
S214449830064B052093E80600BDE80840FAF7F4B85E
S214449840C08340204887402068254120247646002F
S214449850134849F62062134BB0F8801349BA10B542
S21444986099521A4490F8821349F62260C1F30104CF
S2144498701C54C1F3810449F62360C1F303111C54FC
S21444988049F62460195405214FF4547002F07EFBC7
S214449890054B052093E80600BDE81040FAF7C4B827
S2144498A0C08340204887402034764600104849F616
S2144498B02061104A08B5B0F87C335BBA535290F82E
S2144498C07E3303F00100C3F3400343EA400349F602
S2144498D0226013540A444FF44470032102F056FBAA
S2144498E0054B052093E80600BDE80840FAF79CB807
S2144498F0C0834020488740202C76460008B5FFF7B2
S21444990037FAFFF757FAFFF77FFAFFF7E5FAFFF75C
S214449910E1FBFFF707FCFFF79FFCFFF7C1FCFFF7EF
S214449920E9FCFFF725FEFFF74BFEFFF7F3FEFFF7D4
S2144499301BFFFFF741FFFFF76DFFFFF7B7FFBDE8DB
S2144499400840FFF785BF08B5FCF7C2FAF7F763FF90
S214449950FEF7E4FBBDE80840FFF7D0BF704770470A
S21444996070477047064AB2F83032B2F8681003F4CB
S2144499704043C1F30D010B43A2F83032704700BF99
S214449980C0834020044BB3F81221A3F83422B3F822
S2144499900C21A3F836227047C0834020044BB3F80A
S2144499A0A620A3F83C22B3F8A020A3F83E22704792
S2144499B0C083402070477047054BB3F86C21A3F82A
S2144499C04422D3F86821C2F30F12A3F84622704704
S2144499D0C0834020054BB3F87421A3F84C22D3F837
S2144499E07021C2F30F12A3F84E227047C083402062
S2144499F0054BB3F86C21A3F8B821D3F86821C2F319
S214449A000F12A3F8BA217047C0834020054BB3F821
S214449A107421A3F8C021D3F87021C2F30F12A3F81F
S214449A20C2217047C083402008B5FFF7E1FFFFF727
S214449A30EDFFFFF797FFFFF7A5FFFFF7AFFFFFF731
S214449A40BBFFBDE80840FFF7C5BF08B5FCF766F99D
S214449A50F7F7E2FEFEF714FAFFF7E6FFBDE8084024
S214449A60FFF7F4BC70477047704770470B4AD2F80C
S214449A70C831D2F894101B0DC1F313011B050B43D8
S214449A80D2F89810C2F8C83101F47F11D2F8CC311C
S214449A9023F47F130B43C2F8CC317047C083402075
S214449AA008B5F9F761F8BDE80840F8F76DBA7047AD
S214449AB0F7F7AFBEFFF747BFFFF7C7BFFBF717BAC7
S214449AC07047074A1378632B96BF01330023DBB2F3
S214449AD01370044A136801331360FEF744BE00BF94
S214449AE068484120E020402008B5F9F7B9FFBDE8B2
S214449AF0084001F0F7BD08B5FFF7E9FD4CF24053C6
S214449B00044AD058B0FA80F0BDE808404009F9F756
S214449B10A5B800BF6C484120014900201DF024BB75
S214449B20F89A460000201DF023BB0022114610463A
S214449B301DF022BB704700BF044B1A78044B1B78B9
S214449B40134302BF034B02221A7070474318402047
S214449B503F18402044184020064B01221A70064BFA
S214449B601B78934204D1054A13707822044B1A801A
S214449B70704700BF031B40203F184020021B402074
S214449B80001B4020074B08480849094A10B51B7873
S214449B90084C012B18BF0023237003700B701370FE
S214449BA010BD00BF041B40204918402048184020E0
S214449BB0471840204A184020124B134870B519786D
S214449BC0124B012900781C78114B124D1A78124B0F
S214449BD01B780CD1012C0AD1012A08D1012B06D1BD
S214449BE0012804D1002328700C4A137070BD214309
S214449BF000260A432E70134303430CBF0123334607
S214449C00F2E700BF4C184020471840204A1840202E
S214449C1049184020511840204818402050184020E9
S214449C20044B01221A600022034B1A700322034B92
S214449C301A707047E82040204E18402044184020B0
S214449C4008B5FFF79FFFFFF7B7FF044B1B78012BC0
S214449C5003D1BDE80840FFF7E3BF08BD51184020D4
S214449C60054B1B78012B06D1044B1B78012B02BFF6
S214449C70034B00221A7070473F1840204D1840206E
S214449C80441840200D4B0E4A1B7833B90D4B1B78B5
S214449C90012B02BF13880133138000230A490B703B
S214449CA00A490B801188B1F5FA7F05D31380054A1B
S214449CB013700222064B1A70704700BF3E184020AD
S214449CC0F6174020031B4020021B4020001B402068
S214449CD0521840200F4B1B78012B18D10E4B1B7883
S214449CE0012B14D10D4B1B78012B10D10C4B1B7838
S214449CF0012B0CD10B4B1B785A1E534253410A4A34
S214449D0013700123094A1370094A137070470023DD
S214449D10F5E700BF4C1840204A1840204918402018
S214449D2048184020471840205118402050184020DA
S214449D3052184020FFF7A6BF064B1B78042B064B51
S214449D4097BF002201221A70032298BF034B1A7051
S214449D50704700BF08184020041B4020521840207B
S214449D6008B5FFF7B7FF0C480278012A0ED1FFF773
S214449D7089FF0A4B1B78012B07D10278032A04D1AA
S214449D80074A00211160074A137008BD022AF0D121
S214449D90FFF7D2FFEDE700BF52184020501840208E
S214449DA0E8204020441840202DE9F04FC24CBFB074
S214449DB04FF0000A4FF0000BA046D4E91A23D4E92A
S214449DC00267CDE90E2330460022BC4B394605F0E7
S214449DD0A1FA002840F0BB81D4E91245D8E90C2307
S214449DE020462946CDE9002305F08AFA08B9DDE97C
S214449DF0004500224FF08043DDE90E0105F06CFA81
S214449E000022002800F0A68100232046294604F0BC
S214449E10FBFF02460B46D8E98645CDE90223224697
S214449E202B4604F039FE804689468FA3D3E90023A7
S214449E3005F07AFA002800F08F81204629468AA346
S214449E40D3E9002304F02AFECDE90201DFF8688254
S214449E500022DDE90234C8E98634D8E93A34CDE94B
S214449E600034D8E90E4500232046294605F034FA46
S214449E70002800F0838100220023D8E9140105F06D
S214449E803FFA50B100228E4B3046394605F042FA2E
S214449E9018B100230024CDE90034874C94F8583296
S214449EA0002B40F0BA8140F20113A4F85832824B9A
S214449EB00022D3E94045D3E93E892046814B2946D2
S214449EC005F032FA002840F0C78100227E4B204637
S214449ED0294605F00BFA002840F0C18142464B461D
S214449EE02046294604F0D8FD04460D4660A3D3E92F
S214449EF0002305F019FA002840F0B481204629468C
S214449F005DA3D3E9002305F0F1F9002840F0AE81C3
S214449F1042464B462046294604F0C0FD02460B46C0
S214449F20CDE92A2356A3D3E9002304F06DFF8046E7
S214449F30894609F061FF04460D464046494609F005
S214449F40CDFE624B8046894620462946D3E9002307
S214449F5004F05AFF04460D46404649464AA3D3E910
S214449F60002304F051FF0022002304F04DFF024674
S214449F700B462046294604F091FD45A3D3E9002329
S214449F8004F042FF44A3D3E9002304F03DFF00223B
S214449F904F4B04460D4605F0C7F9002840F06A8149
S214449FA0002200232046294605F0A0F908B10024E3
S214449FB00025414B20462946D3E93C8942464B4638
S214449FC004F06AFD04460D4635A3D3E9002305F0A4
S214449FD0ABF9002840F051812046294632A3D3E904
S214449FE0002305F083F9002840F04B8122462B4697
S214449FF04046494604F052FD02460B462E4CCDE9F7
S21444A00038232BA3D3E9002304F0FEFE0022314B71
S21444A010CDE90401C4E9A0ABDDE9000105F05CF933
S21444A020031E4FF00002394618BF012330460C93F6
S21444A030294B05F065F9051E4FF000024FF08043AA
S21444A04018BF0125DDE9020105F05AF90C9B0028EA
S21444A0500CBF2846681C184404F06CFED4E9A223BE
S21444A06004F01CFD002239E0FCA9F1D24D62703F99
S21444A070FCA9F1D24D62603FFCA9F1D24D6260BFAB
S21444A080399D52A246DF913F407EFCF8F14B7B401F
S21444A090E3A59BC420B0D23F578C22C76075B53F1A
S21444A0A0FCA9F1D24D62903F7B14AE47E17AC4BF1F
S21444A0B09A9999999999E93FF00D422000004940B0
S21444A0C00000594000002440000024C09878460010
S21444A0D000004E4000000840000034407C4B05F031
S21444A0E019F90022D4E98E89002800F0058100235E
S21444A0F04046494605F0F0F808B1C4E994AB754EBD
S21444A1000023754C0022C6E98E340023734CC6E9FE
S21444A1109034D6E99445724B2046294605F0E6F835
S21444A12060B120462946DDE90423C6E9922358A3B4
S21444A130D3E9002304F0B2FCC6E994010023664C3C
S21444A140C6E9A0344FF0000ADFF890B103E1544664
S21444A1505D464EE6604B58E64FA3D3E9002340469F
S21444A160494605F0C3F800283FF470AE2046294619
S21444A1704BA3D3E9002304F08FFC65E6DDE9000138
S21444A18005F0F2F803283FF688AEDFE800F002193F
S21444A1901D1900220023D8E9140105F0B1F800285F
S21444A1A03FF47BAE00224C4B2046294605F094F8FB
S21444A1B078BB00224A4B2046294605F08DF840BB22
S21444A1C000224FF080431AE000220023D8E914010D
S21444A1D005F096F800283FF460AE0022414B304626
S21444A1E0394605F097F800283FF457AE00223A4B1C
S21444A1F02046294605F070F840B90022384B2046E0
S21444A200294605F069F800283FF447AECDE90045F5
S21444A21043E600234FF080443DE694F85932012B40
S21444A220D4E900010BD100222F4B05F05FF818B19A
S21444A230022384F859323AE6C4E9A2AB37E61AA3B5
S21444A240D3E9002305F070F808B10123F1E70022B2
S21444A250214BC4E9A2232AE60024244D3EE60024EA
S21444A260234D3BE612A5D5E9004551E612A5D5E9AE
S21444A27000454DE600241F4D9BE611A5D5E9004553
S21444A280B4E611A5D5E90045B0E600BFAFF30080BB
S21444A2907B14AE47E17A743FFCA9F1D24D6280BF8D
S21444A2A0FCA9F1D24D62803F0000000000C062402D
S21444A2B0FCA9F1D24D62603FFCA9F1D24D6260BF69
S21444A2C0FCA9F1D24D62903F7B14AE47E17AC4BFFD
S21444A2D000001040F00D42200000F03F00408F4048
S21444A2E00000084000005940000049C000002440D7
S21444A2F0000024C000004E40BF4B4046494604F090
S21444A300EBFF002800F03D87D4E99223D4E91001FE
S21444A31005F000F8002800F02A87D4E99067AAA33D
S21444A320D3E900233046394604F06EFD02460B4618
S21444A3303046394604F0B0FB06460F46A4A3D3E99C
S21444A340002304F0D3FF002840F00787C4E9906751
S21444A350AA4BD3E990ABA9490022A94BD1E94201C3
S21444A36004F052FD0022A74B04F04EFD00220446A2
S21444A3700D46A14BDDE9000104F0AEFF0C9B00281E
S21444A3804FF000022046294608BF1E469E4B18BF83
S21444A3904FF0FF3604F0C8FF002840F0F88600224D
S21444A3A000232046294604F0A1FF08B100240025D6
S21444A3B0304604F0BFFC22462B4604F025FD8F4B66
S21444A3C004460D46D3E9886732463B4604F064FBB0
S21444A3D000228E4B8046894604F0A6FF00220028C1
S21444A3E000F0D986894B3046394604F057FB04467C
S21444A3F00D46824B002220462946C3E98845824BB7
S21444A40004F092FF002840F0D6860022002320461F
S21444A410294604F06BFF08B10024002500224FF0C3
S21444A4208043DDE90E0104F057FF002800F0C7869C
S21444A43072490022764BD1E9140104F0E5FC064645
S21444A4400F4665A3D3E9002304F06EFF002840F0CE
S21444A450BE86002200233046394604F047FF08B142
S21444A46000260027DFF894810022634BD8E91E01BA
S21444A47004F032FF002288B95F4BD8E9220104F089
S21444A4802BFF002800F0A88600225B4BD8E9240165
S21444A49004F022FF002800F09F8600220023DFF805
S21444A4A05C81C8E99823C8E9A845DDE90434D8E9BD
S21444A4B00401C8E99C34DDE92A34C8E9B467C8E92C
S21444A4C0A434C8E9A6ABD8E9442304F0E7FA44A385
S21444A4D0D3E9002304F098FC04460D4642A3D3E98E
S21444A4E00023D8E9460104F08FFC02460B4620467A
S21444A4F0294604F0D3FA3EA3D3E9002304F0AEFD84
S21444A500D8E94823CDE92201D8E9060104F0C6FA81
S21444A51033A3D3E9002304F077FC04460D4632A364
S21444A520D3E90023D8E94A0104F06EFC02460B4600
S21444A5302046294604F0B2FA2DA3D3E9002304F0BA
S21444A5408DFDD8E94C23CDE91001D8E9080104F083
S21444A550A5FA23A3D3E9002304F056FC04460D468B
S21444A56021A3D3E90023D8E94E0104F04DFC02466A
S21444A5700B462046294604F091FA1DA3D3E900234E
S21444A58004F06CFDDDE91023CDE9120110461946AE
S21444A59004F03AFC04460D46DDE9122310461946FB
S21444A5A004F032FC02460B462046294604F076FA6E
S21444A5B009F068FC0022002304460D4604F08CFE95
S21444A5C028E000BFAFF300809A9999999999A93FDA
S21444A5D07B14AE47E17A843F000000000070974049
S21444A5E0FCA9F1D24D62603FFEF2469F2892AF3FEF
S21444A5F01F94D22C39CFB03F0000F03FF00D4220DC
S21444A6000000B03F000054C000408F4000000840A7
S21444A6100000594048B922462B46DDE9220104F0A1
S21444A6201DFD09F0D1F904460D4620462946D8E9D1
S21444A6304023CDE92423BCA3D3E9002304F0E4FB60
S21444A64002460B46DDE9240104F026FAD8E90A342A
S21444A650CDE92C01CDE92634DDE92601D8E952239B
S21444A66004F01CFAB2A3D3E9002304F0CDFB04465D
S21444A6700D46B1A3D3E90023D8E9540104F0C4FB42
S21444A68002460B462046294604F008FAACA3D3E912
S21444A690002304F0E3FC00220023CDE92E01DDE98B
S21444A6A0000104F019FE0646002840F09985002271
S21444A6B04FF08043DDE9000104F00EFE58B9C24B6A
S21444A6C00022DDE9000104F007FE0C9B00280CBFC5
S21444A6D01E464FF0FF360022BC4BDDE9020104F073
S21444A6E093FB99A3D3E9002304F0B8FC98A3D3E9D9
S21444A6F0002304F089FB0022B54B04F085FB96A3A7
S21444A700D3E9002304F0AAFC04460D46304604F080
S21444A71011FB02460B462046294604F075FB0246CA
S21444A7200B46CDE90823AB4BD3E98A4522462B4654
S21444A73004F0B2F906460F4689A3D3E9002304F091
S21444A740F3FD002800F04F852046294684A3D3E92C
S21444A750002304F0A3F9CDE908019E4CDDE9082363
S21444A760DDE90801C4E98A23D4E9562304F096F9BE
S21444A7706FA3D3E9002304F047FB06460F467AA3AB
S21444A780D3E90023D4E9580104F03EFB02460B46C5
S21444A7903046394604F082F975A3D3E9002304F021
S21444A7A05DFC02460B46CDE90423D4E95A2304F063
S21444A7B073F90022854B04F027FBD4E95C2304F0AC
S21444A7C06BF902460B46CDE91423D4E95E2304F024
S21444A7D063F900227D4B04F017FBD4E9602304F0B0
S21444A7E05BF902460B46CDE91623D4E9622304F00E
S21444A7F053F90022754B04F007FBD4E9642304F0B4
S21444A8004BF95DA3D3E90023CDE93001DDE904012A
S21444A81004F0FAFA06460F4659A3D3E90023DDE9C5
S21444A820140104F0F1FA32463B4604F037F9804608
S21444A830894655A3D3E90023DDE9160104F0E4FA7A
S21444A84002460B464046494604F028F9DDE93023E3
S21444A85004F024F94EA3D3E9002304F0D5FAD4E94E
S21444A8606623CDE918011046194604F017F9DDE9C8
S21444A870182304F013F9D4E92A2304F00FF946A365
S21444A880D3E9002304F0C0FA8046894644A3D3E9BA
S21444A8900023D4E9680104F0B7FA02460B46404662
S21444A8A0494604F0FBF8804689463FA3D3E9002393
S21444A8B0D4E92E0104F0A8FA02460B46404649461F
S21444A8C004F0EAF83AA3D3E9002304F0C7FB0246AF
S21444A8D00B46CDE91A23D4E96A2304F0DFF814A31F
S21444A8E0D3E9002304F090FA8046894632A3D3E99C
S21444A8F00023D4E96C0104F087FA02460B4640462E
S21444A900494604F0CBF82EA3D3E9002304F0A6FB73
S21444A910D4E90023CDE93201DDE9040104F0BCF8B2
S21444A920002259E0AFF30080F8C1631ADCA54C401E
S21444A930FCA9F1D24D62603FFEF2469F2892AF3F9B
S21444A9401F94D22C39CFB03F000000000020AC400A
S21444A9505C8FC2F528DC2740B46155D0CC38FB3F29
S21444A9609A9999999999D93FB428207983A6BA3F58
S21444A97054434F56A8ACBB3F9A99999999996340CA
S21444A9809A99999999996A40CDCCCCCCCCCC3540FF
S21444A990E3F36EFB79D0E33E277845D92444D93F88
S21444A9A0FB50D7647BD71C403043BB3975F1044019
S21444A9B06D0D4BFEC9AF1840EBF33CDE4AA2813F17
S21444A9C0E9C8B5C771D3893F0000F03F00408F40C7
S21444A9D000004E40F00D4220C34B04460D4604F0A2
S21444A9E0A3FC002840F0128420462946A2A3D3E9BB
S21444A9F0002304F07BFC002840F01B840022BB4B61
S21444AA002046294604F090FC002800F003840022E7
S21444AA10B64B2046294604F03FF880468946B44C57
S21444AA20DDE90401D4E96E2304F036F80022B14B84
S21444AA3004F0EAF9D4E9702304F02EF802460B46F3
S21444AA40CDE91C23D4E9722304F026F80022A94B4E
S21444AA5004F0DAF9D4E9742304F01EF802460B46EF
S21444AA60CDE91E23D4E9762304F016F80022A14B40
S21444AA7004F0CAF9D4E9782304F00EF880A3D3E9A5
S21444AA800023CDE93401DDE91C0104F0BDF932466A
S21444AA903B4604F003F806460F467BA3D3E900235F
S21444AAA0DDE91E0104F0B0F902460B46304639464D
S21444AAB003F0F4FFDDE9342303F0F0FF74A3D3E995
S21444AAC0002304F0A1F9D4E98C2303F0E5FF024601
S21444AAD00B46CDE93A23D4E97A2303F0DFFF6EA38D
S21444AAE0D3E9002304F090F906460F466CA3D3E955
S21444AAF00023D4E97C0104F087F902460B4630462D
S21444AB00394603F0CBFF68A3D3E9002304F0A6FA42
S21444AB10D4E97E23CDE90A011046194603F0BEFF68
S21444AB20DDE90A2303F0BAFFD4E9322303F0B6FF83
S21444AB305FA3D3E9002304F067F906460F465EA3F5
S21444AB40D3E90023D4E9800104F05EF902460B46BB
S21444AB503046394603F0A2FF06460F4658A3D3E9CB
S21444AB600023D4E9360104F04FF902460B4630463A
S21444AB70394603F091FF54A3D3E9002304F06EFA58
S21444AB8000225D4BD4E91445CDE9200120462946F0
S21444AB9004F0ACFB002840F07D830022564B204650
S21444ABA0294603F079FF4AA3D3E9002304F02CF99D
S21444ABB00022524B06460F4604F0ACFB08B1002672
S21444ABC04E4F45A3D3E90023DDE9200104F01CF9E8
S21444ABD000224B4B83468A4604F088FB06900028A6
S21444ABE040F05B830022474B5846514604F09CFB9A
S21444ABF0002840F057830AF1004A4046494638A3A5
S21444AC00D3E9002304F000F9DDE9322303F046FFDC
S21444AC108046894632463B465846514604F0F4F848
S21444AC2042464B4603F03AFF02460B46CDE906231E
S21444AC300022354B04F078FB0022002840F037838E
S21444AC40324BDDE9060104F051FB18B100222F4BCC
S21444AC50CDE90623264ED6E92223DDE90E01CDE9C9
S21444AC60362300224FF0804304F036FB002207468A
S21444AC70002800F01E834BE00000000000409FC008
S21444AC809A99999999996A40CDCCCCCCCCCC3540FC
S21444AC90E3F36EFB79D0E33EFCA9F1D24D62603F0C
S21444ACA05ED817C2038C9E3F6F216A9B4B52A13FCE
S21444ACB02ED7D19C0A49373F7119ABB745FF1F4081
S21444ACC0ECBC164D8E930F401988C921F3361040BC
S21444ACD09A9999999999C93FCDCCCCCCCCCCEC3F98
S21444ACE03B08AA2A23DCA63F00409F400000494078
S21444ACF0F00D422000408F40000014400000F03F1A
S21444AD0000003EC000003E4000005440000054C0D6
S21444AD10AB4BD6E91E0104F0DFFA88B90022A84BF3
S21444AD20DDE9360104F0D8FA002800F0EA82002271
S21444AD30A34BD6E9240104F0CFFA002800F0E182C0
S21444AD402046294600269AA3D3E9002304F086F930
S21444AD5000229C4B04F0E8FA002800F0D3829A4F75
S21444AD60DFF87482D8E92023CDE90C23DDE90C0111
S21444AD700022934B04F0B0FA002840F0C5823246D5
S21444AD803B46C8E99E23DDE90023C8E9B667C8E91F
S21444AD90AE23DDE9020122462B4603F07DFE002267
S21444ADA08A4B8B4ECDE93C012046294604F02CF8CC
S21444ADB002460B460020874903F06EFE0022844B71
S21444ADC00C46054604F092FA002808BF28467AA3A3
S21444ADD0D3E9002316BF00202146314604F014F878
S21444ADE0CDE902017C49D1E982ABD1E9160152464C
S21444ADF05B4603F051FE002280468946744B284643
S21444AE00214604F073FA002840F0818204F100449D
S21444AE1042464B46DDE9020104F068FA002840F059
S21444AE2079822846214664A3D3E9002303F0ECFF45
S21444AE3006460F4602460B464046494604F056FA36
S21444AE4008B946464F463246634E3B4650465946F8
S21444AE504FF0000803F022FE82468B46DFF86091EE
S21444AE60D6E91C23CDE90E23DDE90E010022544B1E
S21444AE7004F032FA88B942464B46D6E9260104F035
S21444AE802BFA002800F0498242464B46D6E9280170
S21444AE9004F022FA002800F04082002200234E49A3
S21444AEA0C1E99A23D1E98423C1E9B2ABD1E91801B7
S21444AEB0CDE9282303F0F0FD06460F4602460B462E
S21444AEC0DDE9020104F012FA88B9284621463AA37D
S21444AED0D3E9002303F098FF02460B46CDE902234C
S21444AEE032463B4604F020FA08B9CDE90267DDE96C
S21444AEF00223DDE9280103F0D1FD374C02460B4618
S21444AF00C4E9AA2300220023CDE90201C4E9B02300
S21444AF10DDE90C0100222A4B04F0DEF968B9002270
S21444AF20274BDDE90E0104F0D7F930B90022244B53
S21444AF30D4E91E0104F0D0F908B1C4E9B08900226E
S21444AF401F4BDDE9360104F0C7F9002800F0E8811C
S21444AF50214BC3E9B089DFF880800022DDE9003464
S21444AF60D8E95067C8E93A34DDE9383430463946DA
S21444AF70C8E93C34DDE92A34C8E93E34174B03F0CB
S21444AF8043FF04460D460022154BDDE92C0103F031
S21444AF903BFF02460B462046294603F07FFD024609
S21444AFA00B46DDE92E0103F077FD1BE0AFF300808E
S21444AFB0CDCCCCCCCCCC0C40FCA9F1D24D62603F7D
S21444AFC00000F03F0000E03F000054C000001A407C
S21444AFD00080614000007940F00D4220000014409B
S21444AFE00000594096A3D3E9002303F00DFFDDE9A2
S21444AFF0242303F053FD00229B4BC8E94001D8E9C3
S21444B000420103F001FFDDE93C2303F047FDD8E9A4
S21444B0100423C8E94201C8E94423DDE92234DDE9D2
S21444B0202C01C8E94634D8E90623C8E94823DDE9B3
S21444B0301034C8E94A34D8E90823C8E94C23DDE982
S21444B0401234C8E94E347EA3D3E9002303F0DCFE71
S21444B05032463B4603F022FDDDE92634C8E950017A
S21444B060C8E95234DDE92E34C8E95434DDE90834FD
S21444B070C8E95634DDE90434C8E95834C8E95A34D2
S21444B080DDE91434C8E95C34C8E95E34DDE91634D5
S21444B090C8E96034C8E96234DDE93034C8E9643468
S21444B0A0DDE91834C8E96634D8E92C23C8E92A23EC
S21444B0B0DDE91834C8E92C34DDE91A34C8E96834C3
S21444B0C0D8E93023C8E92E23DDE91A34C8E93034F8
S21444B0D0C8E96A34DDE93234C8E96C34DDE906345B
S21444B0E0C8E98C34DDE90434C8E96E34DDE91C343F
S21444B0F0C8E97034C8E97234DDE91E34C8E982AB65
S21444B100C8E97434C8E97634DDE93434C8E97834B7
S21444B110DDE93A34C8E97A34DDE90A34C8E97C34EE
S21444B120C8E97E34D8E93423C8E93223DDE90A3451
S21444B130C8E93434DDE92034C8E98034D8E9382312
S21444B140C8E93623DDE92034C8E93834DDE9023479
S21444B150C8E984343FB0BDE8F08FC4E990ABC4E995
S21444B1608EABC4E992ABC4E994ABFFF7F1B80022C6
S21444B1703E4BC4E9902300223D4BC4E9A023FEF78E
S21444B180E1BF4FF0000A4FF0000BFFF7E4B800248D
S21444B190364DFFF70DB9374B4046494604F0A6F8FE
S21444B1A000283FF426A90022334B3046394603F0A4
S21444B1B073FCFFF71CB900242C4DFFF72FB9224629
S21444B1C02B465046594603F069FCFFF738B91EA78C
S21444B1D0D7E90067FFF746B932463B46FFF75FB903
S21444B1E00026FFF778BA1AA3D3E900233046394637
S21444B1F004F07CF800283FF4B0AA2046294616A35B
S21444B200D3E9002303F048FCFFF7A5BA00241B4DFE
S21444B210FFF7FDBB00221A4B2046294604F07AF875
S21444B22090BB0022174B2046294603F037FCFFF715
S21444B230F4BB0BA5D5E90045F3E700BFAFF30080A8
S21444B240FCA9F1D24D62603F0000000000709740B8
S21444B2509A9999999999E9BF9A9999999999E93FA7
S21444B2600000000000409FC00000EE3F00408F40BA
S21444B2700000F03F000008C00000084000409F4027
S21444B280000049C0000049404FF000084FF0000954
S21444B290FFF7C5BB0026002793E44FF0000BDFF80A
S21444B2A0B8A0AAE4DDF818B0DFF8B0A0A5E4264BB1
S21444B2B0CEE40023DDE9000104F00EF80646E0B9CA
S21444B2C000224FF08043DDE9000104F005F8B0B9F0
S21444B2D01E4B0022DDE9000103F0FEFF00280C9B14
S21444B2E018BF4FF0FF33184603F024FDDDE906236C
S21444B2F003F08AFD06460F4632E53846F4E7304604
S21444B300F2E7002600272BE50022002339E5002536
S21444B3100F4C7DE5DDE9026795E552465B46BEE5A2
S21444B3200C4C0022094BD4E9260103F0D5FF002833
S21444B3303FF411AE0022054BD4E9280103F0CCFFBC
S21444B34000287FF405AE06E6000054400000F03FB7
S21444B350008061C0F00D422000003E4000003EC028
S21444B360704700BF38B55A4B5A4C186803F0F4FC83
S21444B370594B1D78C4E90001284603F0CBFC574BD3
S21444B380C4E91A01186803F0E7FC554BC4E91401F4
S21444B390186803F0E1FC534BC4E90401186803F051
S21444B3A0DBFC514BC4E90601186803F0D5FC4F4B4F
S21444B3B0C4E90801186803F0CFFC4D4BC4E90A0100
S21444B3C0186803F0A7FC4B4BC4E91C01186803F04B
S21444B3D0A1FC494BC4E91E01186803F09BFC474B8B
S21444B3E0C4E92001186803F095FC454BC4E92201E2
S21444B3F0186803F08FFC434BC4E92401186803F033
S21444B40089FC414BC4E92601186803F083FCC4E96F
S21444B4102801002D2CD13D4B186803F09DFC3C4B75
S21444B420C4E90201186803F075FC0022394BC4E9EC
S21444B4301223394BC4E90C01186803F06BFC374BF4
S21444B440C4E90E01186803F087FC354BC4E91601BD
S21444B450186803F081FCC4E91801324B1B78002BB2
S21444B46032D1314B186803F077FCC4E9100138BD7B
S21444B470012D22D12D4B186803F06EFC2C4BC4E9E9
S21444B4800201186803F046FC2A4BC4E90C0118680C
S21444B49003F040FC284BC4E91201186803F03AFC58
S21444B4A0264BC4E90E01186803F056FC002200231C
S21444B4B0C4E91601C4E91823CFE7022DCDD10022F2
S21444B4C00023C4E90C23C8E700200021CDE700BFD1
S21444B4D0301E4020F00D42203A1840204C1C40209C
S21444B4E0E01E4020001F4020C41E4020D01E4020A6
S21444B4F0381F4020201F40204C1F4020181F40204B
S21444B500141F4020401F40203C1F40207C1D4020EC
S21444B510841D402000004440541D4020701D40209F
S21444B5206C1D4020401840202C1E4020981F402070
S21444B530801F4020501F4020681F40208C1F402002
S21444B5402DE9F74F534CDFF89491DFF894A1DFF8D8
S21444B55074B1D4E9000103F04FFF4F4B074618601F
S21444B560D4E9060103F048FFC9F80000D4E9040111
S21444B57003F042FF494B1860D4E9020103F03CFF54
S21444B5800646CAF80000CBF80000D4E9120103F0DE
S21444B59033FF434A434B804610601860D4E9160193
S21444B5A003F00AFF404905460860D4E9180103F051
S21444B5B003FF3E490870D4E91E0103F01DFF3C49D1
S21444B5C00860D4E91C0103F017FF3A490860D4E93F
S21444B5D01A0103F011FF38490860304637490968B4
S21444B5E0019104F023FA2E4A2E4BCDF80090914652
S21444B5F01C46019968B1CAF80010CBF80010304ECA
S21444B6004046314604F012FAB8B1C9F800602660E4
S21444B6101AE001F1004B3046594604F0E9F928B1E6
S21444B620CAF800B0274BC3F800B0E8E7594630469E
S21444B63004F0DEF90028E2D0F4E7234E40463146D3
S21444B64004F0D6F90028E0D1204B1B786BB9204B88
S21444B65025F0020519681F4C012D0AD1384603F01F
S21444B66021FF206003B0BDE8F08F012B03D11A4BB5
S21444B670EEE72160F6E7022B02D1164B1F60F1E796
S21444B680032BEFD10023009A1360134B1A68114B17
S21444B6901A60E7E750104220881F40209017402049
S21444B6A08018402068184020301C402084174020D2
S21444B6B0801740207C174020781740208817402069
S21444B6C000004843F0184020000048C33A18402081
S21444B6D07C1D4020901F4020981F4020341B402053
S21444B6E05C194020F8B5174B174C1E78174D66B1B9
S21444B6F0012E19D000210020F6F7E6F8002101209B
S21444B700F6F7E2F800232B700CE02678002EF1D1F1
S21444B71000213046F6F7D8F80D490120F6F7D4F85C
S21444B72001232E702370F8BD2F78002FE2D10849EC
S21444B7303846F6F7C9F800213046F6F7C5F82E70B5
S21444B7402770F0E73A184020C4174020C517402019
S21444B7500000C8422D4A2E49106810B550B90B68EF
S21444B760012B07D12B4803602B4803602B4803600A
S21444B7702B4803602B4B502018602B4B2B481860EB
S21444B7802B4B1B6813602B4B1B780B602A4B1C6897
S21444B79074B92A4B0021186804F020F988B1284B64
S21444B7A007221A600122274B1C60274B1A6008E0C8
S21444B7B0012C07D10223224A1360224A1360224AEC
S21444B7C0136010BD022C0FD11C4B0021186804F0E6
S21444B7D005F90028F5D01A4B03221A600022194BAB
S21444B7E01A60194B1C60ECE7032CEAD1134B00217A
S21444B7F0186804F0F3F80028E3D0114B04221A60CA
S21444B8000122104B1A6002220F4BCFE7141B402034
S21444B810101B4020201B4020241B4020281B402077
S21444B8202C1B40200C1B4020081B4020000048C214
S21444B830A0194020DE1D4020301C40204C1C4020D7
S21444B8401C1B4020181B40203C1B402000000000CE
S21444B85038B5174B00211C68204604F0C9F808B1D7
S21444B86004F10044134D20462C6003F075FA0CA3F3
S21444B870D3E9002303F0F2FB0BA3D3E9002303F040
S21444B880C3FA00220C4B03F0BFFA0C4B002203F021
S21444B890E5FB03F0B1FD0A4B6860186038BD00BF95
S21444B8A05C8FC2F528DC2740B4A766033D39FB3FCE
S21444B8B0301E4020F420402000004E4000408F4080
S21444B8C04C1C4020264B1B68012B264B0FD0264A87
S21444B8D01288012A0BD0254A1068012807D0244A2A
S21444B8E01268012A03D0234A1278012A0CD1022274
S21444B8F01A601B68204A1370204B1B78013B012BAF
S21444B9002CD80323137070471D4A11681D4A012919
S21444B910126807D1196803291BD1002AE8D0012AE6
S21444B920E7D118E0012A06D1186803280ED1002969
S21444B930DFD10122DCE719B9196809B90322D7E730
S21444B940002AD6D11A68012AD3D1F7E70029F3D0C2
S21444B950CFE7012AF4D10028EBD0CAE7704700BFEE
S21444B960601F40202C1C4020E0174020501D4020E3
S21444B970701F4020841740203A1840200218402068
S21444B980601D40206C1F402008B5FEF77BF9144B21
S21444B9901B886BB9134B144A1B681268134307D1B0
S21444B9A0124A1360124A1360124A1360124A136012
S21444B9B00023124A01211360114A1360114A13608E
S21444B9C0114A1360114A1360114A1360114A1360F6
S21444B9D0114A1360114A1160114A136008BD00BF32
S21444B9E0E0174020601F4020501D4020441D40204A
S21444B9F0401D40201C1A4020201A4020341C402061
S21444BA00E01A40203C1D4020381D4020341D402074
S21444BA10301D40202C1D4020281D4020241D402041
S21444BA20201D402008B5FEF797F8044B1B68012BF1
S21444BA301EBF034B00221A6008BD00BF501D4020A5
S21444BA40E01A402008B5FEF787F8064B1B68012B22
S21444BA501EBF054B00221A60044B1A68044B1A603A
S21444BA6008BD00BF601F4020341C4020501F4020AB
S21444BA70481C4020F8B5134A0223134F1360134E54
S21444BA80134A3B60136033600123124D124C2B6003
S21444BA902360FEF7F7F8114B1B8893B9104B114AF5
S21444BAA01B6812681343104A1268134309D10F4B9C
S21444BAB01B7833B903223B6033602B6023600C4B06
S21444BAC01A60F8BD3C1B4020441D4020401D4020C9
S21444BAD0301C4020341C4020E01A4020E017402010
S21444BAE0601F4020501D4020701F40208417402077
S21444BAF02C1C402008B5174B186803F0A1FF164BC2
S21444BB00164A186001231360154A1360154A1360D9
S21444BB10154A1168154A1160154A16491370164A93
S21444BB201370164A1370164A1370164A1370164A40
S21444BB30137000220A7015490A7015490B7015498E
S21444BB400B7015490B7015490B70154B1A70154B35
S21444BB501A7008BD341B40204C1A4020481A402016
S21444BB60381A4020D4184020301C4020DC1840208E
S21444BB7068194020A5184020FC1840205A19402037
S21444BB80EE1840201519402014194020A4184020CF
S21444BB907D184020791840207A18402064184020A8
S21444BBA0601840206118402000230A4A152113706B
S21444BBB0094A1370094A11700621094A1370094A42
S21444BBC01370094A1170094A13701822084B1A70E8
S21444BBD0704700BF0619402005194020041940202C
S21444BBE00319402002194020011940200019402022
S21444BBF0FF18402008B5FFF77DFFFFF7D5FFFFF796
S21444BC0061FEFFF7AFFBFEF7CFF8FFF799FC0D4B4D
S21444BC101B781BB9BDE80840FFF704BF012B03D1CE
S21444BC20BDE80840FFF70EBF022B03D1BDE808402D
S21444BC30FFF720BF032B03D1BDE80840FFF7A4BE9F
S21444BC4008BD00BF3A184020074B19221A60052247
S21444BC50064B1A600F22064B1A600222054B1A60E6
S21444BC60054B064A1A607047801B40207C1B4020C8
S21444BC70781B4020741B4020701B4020EFAB030011
S21444BC8008B5074B186803F0BDFC064B0649186018
S21444BC9003F0B8FE10B1054B03221A7008BD00BF6E
S21444BCA0D81D40202C1840200000F0413018402079
S21444BCB0034B044A9B6FC3F309231370704700BFBA
S21444BCC0C083402008184020084B1B78013B022BB9
S21444BCD00AD80023064A00211370064A1160064A11
S21444BCE013700322054B1A60704700BF02184020A9
S21444BCF001184020341B4020001840202C1C4020B3
S21444BD00044B054A1B781370013B012B01D8FFF7FF
S21444BD10DBBF7047E41D402002184020FE28D4BFF5
S21444BD2001300020704770B50022FF23064ED4B27F
S21444BD30551C8C4202D3D843C0B270BD025D5340FA
S21444BD402A46F35CF3E700BFA87846000721013093
S21444BD5008B5FFF7E8FFC0B208BDB0F5447F38B574
S21444BD60144617D1244D204695F8FC32FF2B14BFB9
S21444BD7001330023DBB285F8FC3253701F4A13703C
S21444BD80FFF7E4FF1E4BC0B285F8FD022070187022
S21444BD90012038BD402818D0B0F5547FF8D1164D50
S21444BDA0204695F8F832FF2B14BF01330023DAB24D
S21444BDB085F8F8226270134A1360FFF7C7FFC0B2D3
S21444BDC0114B85F8F902207014E00B4D204695F887
S21444BDD0F032FF2B14BF01330023DAB285F8F02289
S21444BDE062700A4A1360FFF7B1FF094BC0B285F888
S21444BDF0F10220701860CBE7C0834020171940201A
S21444BE0016194020101940200C194020641940206F
S21444BE1060194020402838B5144616D1254D204692
S21444BE2095F82833FF2B14BF01330023DAB285F884
S21444BE3028236270204A1360FFF788FF1F4BC0B266
S21444BE4085F829032070186005E0B0F5547F04D0C7
S21444BE50B0F5447F17D0012038BD164D204695F8DE
S21444BE603033FF2B14BF01330023DAB285F8302376
S21444BE706270134A1360FFF769FFC0B2114B85F82E
S21444BE8031032070DFE70B4D204695F83433FF2B03
S21444BE9014BF01330023DBB285F8343353700A4AA7
S21444BEA01370FFF753FF094BC0B285F83503207073
S21444BEB01870D0E7C0834020F8184020F41840207B
S21444BEC0A01840209C184020A7184020A6184020C0
S21444BED0402838B5144617D1254D204695F82833C2
S21444BEE0FF2B14BF01330023DAB285F86423627053
S21444BEF0204A1360FFF72AFF1F4BC0B285F865033C
S21444BF0020701860012038BDB0F5547F18D0B0F5C5
S21444BF10447FF7D1164D204695F87033FF2B14BF57
S21444BF2001330023DBB285F870335370134A137021
S21444BF30FFF70CFFC0B2124B85F87103207014E073
S21444BF400B4D204695F86C33FF2B14BF013300236A
S21444BF50DBB285F86C3353700A4A1370FFF7F6FE6B
S21444BF60094BC0B285F86D0320701870CAE700BF4D
S21444BF70C083402088184020841840207C184020E5
S21444BF807B1840207818402077184020402838B541
S21444BF90144616D1254D204695F87433FF2B14BF0E
S21444BFA001330023DAB285F874236270204A1360A2
S21444BFB0FFF7CCFE1F4BC0B285F87503207018609F
S21444BFC005E0B0F5547F04D0B0F5447F17D0012087
S21444BFD038BD164D204695F88033FF2B14BF0133E9
S21444BFE00023DAB285F880236270134A1360FFF7A1
S21444BFF0ADFEC0B2114B85F881032070DFE70B4DD0
S21444C000204695F87C33FF2B14BF01330023DBB264
S21444C01085F87C3353700A4A1370FFF797FE094B32
S21444C020C0B285F87D0320701870D0E7C0834020E6
S21444C030701840206C1840205C1840205818402047
S21444C0406318402062184020502870B505461446B0
S21444C05016D18C4A92F8AC31FF2B14BF013300231F
S21444C060D9B282F8AC11884A2171136040F2853304
S21444C0709D4200F0DD80162D00F0F080012070BD5A
S21444C080642826D065283BD032284FD0702863D009
S21444C090712877D0332800F08C806A2800F09F807F
S21444C0A0B0F5617FE2D1774D204695F80033FF2BFB
S21444C0B014BF01330023DBB285F800335370734A50
S21444C0C01370FFF743FEC0B2714B85F8010320702E
S21444C0D06DE06C4E204696F8B832FF2B14BF013301
S21444C0E00023DBB286F8B83253706A4A1370FFF7FF
S21444C0F02DFE694BC0B286F8BC0220701870B5E7B6
S21444C100604E204696F82033FF2B14BF013300239D
S21444C110DBB286F820335370604A1370FFF716FE7E
S21444C120C0B25F4B86F824032070E7E7554E20469E
S21444C13096F8D032FF2B14BF01330023DBB286F8C7
S21444C140D0325370574A1370FFF700FEC0B2564BB6
S21444C15086F8D1022070D1E74A4E204696F8C4327B
S21444C160FF2B14BF01330023DBB286F8C43253706E
S21444C1704E4A1370FFF7EAFDC0B24D4B86F8C5022F
S21444C1802070BBE73F4D204695F81433FF2B14BF71
S21444C19001330023DBB285F814335370454A1370D9
S21444C1A0FFF7D4FD444BC0B285F8150320701870D1
S21444C1B064E7344D204695F83833FF2B14BF0133DB
S21444C1C00023DBB285F8383353703C4A1370FFF7CC
S21444C1D0BDFDC0B23A4B85F839032070E7E7294DD8
S21444C1E02046D5F8E832D5F8E822C3F3C733FF2B08
S21444C1F014BF01330023DBB263F3D632C5F8E8221A
S21444C2006370D5F8E8322F4AC3F3C7331360FFF799
S21444C2109DFDB5F8EA32C0B22B4A60F3CE13A5F8BA
S21444C220EA322070B5F8EA32C3F3C713136025E741
S21444C230144D2046254A95F85033FF2B14BF01333E
S21444C2400023DBB285F8503363701370FFF77EFD2E
S21444C250C0B21F4B85F851032070A8E70949B1F8CE
S21444C260A022C2F34313013303F00F0363F34812CF
S21444C270A1F8A0226370B1F8A032164AC3F3431360
S21444C280D4E700BFC0834020001C4020081940204B
S21444C290071940205819402059194020EC184020CE
S21444C2A0ED1840206A194020691940203919402069
S21444C2B038194020C9184020C8184020FE1840208D
S21444C2C0FD1840204C19402048194020951840201D
S21444C2D0941840209C1A40200F28D4BF01300020D8
S21444C2E0704770B50022FF23074ED4B2551C8C42CB
S21444C2F005D3DB4383EA131303F00F0070BD025DDE
S21444C30053402A46F35CF0E7A879460007210130FB
S21444C31008B5FFF7E6FFC0B208BDB0F5AE6F70B51E
S21444C320054614461AD1C04D204695F815221309E1
S21444C330013363F3071203F00F0385F81522BB4A53
S21444C3401360FFF7E3FF95F8163260F3030300F03B
S21444C3500F0085F81632B64B1860C0E0B0F5B06FE3
S21444C3601DD0B0F5B26F35D1AF4D204695F8262294
S21444C37002F00F03013363F3030203F00F0385F85F
S21444C3802622AC4A1360FFF7C1FF95F8263260F3C5
S21444C390071300F00F0085F82632A74BDCE7A24DC2
S21444C3A02046B5F81C22C2F38313013363F3891283
S21444C3B003F00F03A5F81C22A04A1360FFF7A6FF5C
S21444C3C095F81D3260F3850300F00F0085F81D32A2
S21444C3D09B4BC1E740F29553984222D040F2855396
S21444C3E0984258D050287CD0512835D18E4D20467E
S21444C3F095F8402202F00F03013363F3030203F07F
S21444C4000F0385F840228F4A1360FFF77FFF95F8A5
S21444C410403260F3071300F00F0085F840328A4B31
S21444C4209AE7814E204696F82B22C2F383030133C3
S21444C43003F00F0363F3850286F82B22834A1370B6
S21444C440FFF764FF96F82C3200F00F0060F3030306
S21444C45086F82C327E4B1870602D5DD0612D35D118
S21444C460714D204695F8502202F00F03013363F3D2
S21444C470030203F00F0385F85022764A1360FFF751
S21444C48045FF95F8503260F3071300F00F0085F827
S21444C4905032714B60E7644E2046D6F83022C2F3E1
S21444C4A08333013363F3913203F00F03C6F830222B
S21444C4B06A4A1360FFF72AFF96F8323260F3850320
S21444C4C000F00F0086F83232654B1860132D3ED0CC
S21444C4D0142D57D0152D70D0162D00F089800120CC
S21444C4E070BD514D204695F8382202F00F030133B3
S21444C4F063F3030203F00F0385F83822594A1360A6
S21444C500FFF704FF95F8383260F3071300F00F0086
S21444C51085F83832544B1FE7434D204695F8482259
S21444C52002F00F03013363F3030203F00F0385F8AD
S21444C53048224E4A1360FFF7E9FE95F8483260F306
S21444C540071300F00F0085F84832494B04E7364D90
S21444C5502046B5F85A22C2F38313013363F3891293
S21444C56003F00F03A5F85A22424A1360FFF7CEFEA3
S21444C57095F85B3260F3850300F00F0085F85B3274
S21444C5803D4BE9E6284D204695F8622202F00F031B
S21444C590013363F3030203F00F0385F86222374A3C
S21444C5A01360FFF7B3FE95F8623260F3071300F0AA
S21444C5B00F0085F86232324BCEE61B4D204695F886
S21444C5C06A2202F00F03013363F3030203F00F03FE
S21444C5D085F86A222B4A1360FFF798FE95F86A326C
S21444C5E060F3071300F00F0085F86A32264BB3E673
S21444C5F00D4D2046B5F8A022C2F34313013363F32E
S21444C600481203F00F03A5F8A022204A1360FFF750
S21444C6107DFE95F8A13260F3440300F00F0085F8E0
S21444C620A1321B4B98E600BFC0834020B41940207B
S21444C630B0194020F41D4020F01D4020AC1D402081
S21444C640A81D40207C1A4020781A40207F1940209C
S21444C6507E1940205C1A4020581A402088194020F1
S21444C660841940208C1A4020881A40206C1A402096
S21444C670681A4020DC1A4020D81A4020BC1A4020B1
S21444C680B81A4020A41A4020A01A40209C1A4020E1
S21444C690981A402038B53D4B1A783D4B1B781343C7
S21444C6A040D13C4B1B78013B18BF01233A4A1370D8
S21444C6B03A4B1A683A4B1B6813433A4B14BF012251
S21444C6C000221A70384B1A78384B1B781343384B71
S21444C6D014BF012200221A70364B374A1B78013B9E
S21444C6E018BF01231370354B354A1B78003B18BFDF
S21444C6F001231370334B344A1B78003B18BF012385
S21444C7001370324B1C789CB9314D2B78012B0BD1CE
S21444C710304B1C70304B1C70FFF796FABDE838401F
S21444C720FFF7AEBA0123C1E7022B1FD12C7038BDE8
S21444C730012CFCD1264B1B78012B05D1254A1370BE
S21444C740BDE83840FDF7F8B9022B03D1BDE83840C0
S21444C750FDF776BA032BEAD1FFF74CFAFFF7D0FA87
S21444C760FEF7F8FFBDE83840FFF772B8032B02D156
S21444C770FFF79EFADAE7002BD9D1184A0121116057
S21444C780174A1360BDE83840FDF7EABAA61D4020B4
S21444C790A51D4020DC1D402043184020501E40204C
S21444C7A04C1E402040184020951D4020941D40209B
S21444C7B041184020DD1D402042184020DE1D402008
S21444C7C03F184020E81D40203E1840204518402091
S21444C7D044184020041B4020521840203C1B402054
S21444C7E0301C40207047704730B53D4C85B03D48BE
S21444C7F0237801A90193019B1B020193019A637854
S21444C80013440193019B1B020193019AA37813449A
S21444C8100193019B1B020193019AE378134401930D
S21444C82023790293029B1B020293029A6379134470
S21444C8300293029B1B020293029AA3791344029327
S21444C840029B1B020293029AE37913440293237ACF
S21444C8500193019B1B020193019A637A134401934B
S21444C860019B1B020193019AA37A13440193019BF3
S21444C8701B020193019AE37A13440193237B0293A8
S21444C880029B1B020293029A637B13440293029B0D
S21444C8901B020293029AA37B13440293029B1B023D
S21444C8A00293029AE37B1344029342F21273019377
S21444C8B042F21373029300F0B0FB04F1100004F14B
S21444C8C0080104F11802082314F8015B013B00F840
S21444C8D0015B11F8015B02F8015BF5D105B030BD90
S21444C8E0D4104220808080000C4A0823002102F1A4
S21444C8F0280030B402F1080502F12004013B02F896
S21444C900011B05F8011B13F0FF0304F8011B00F894
S21444C910011BF3D130BCFFF767BF00BFD4104220E1
S21444C9204F4BF0B51B688BB002934E4B1A6803927C
S21444C9305A6804929B68059342F21273029A9A428A
S21444C94000F08980484800F013FBFFF7CDFF002332
S21444C95046480AAA50F8231002EB83020133082BF8
S21444C96042F8201CF5D1002340480AAA50F8231068
S21444C97002EB83020133082B42F8201CF5D10299BE
S21444C9800025039A049B0598394C0090394826465E
S21444C99000F0EEFA029B38481B0E2370029B1B0CD9
S21444C9A06370029B1B0AA370029BE370039B1B0EDF
S21444C9B02371039B1B0C6371039B1B0AA371039B8C
S21444C9C0E371049B1B0E2372049B1B0C6372049B33
S21444C9D01B0AA372049BE372059B1B0E2373059BE1
S21444C9E01B0C6373059B1B0AA373059BE37300F040
S21444C9F0B6FA013516F8010B00F0DAFA082DF8D12C
S21444CA001E4D002600F0CBFA1D482F4600F0A7FA2C
S21444CA10013617F8010B00F0CBFA082EF8D100F0D7
S21444CA20BEFA184B002203F1080703F1100003F185
S21444CA3018019446013214F8016B15F801EB082AE4
S21444CA4003F8016B07F801EB00F8016B01F801CB22
S21444CA50F0D10BB0F0BD0C4800F08AFA77E700BF7F
S21444CA6080808000848080000A8046001080800099
S21444CA70D41042202E8046004B804600DC104220D4
S21444CA8055804600E410422020804600194A08217A
S21444CA901948F0B592F8A53100F1100C00F10805DC
S21444CAA000F11807012B9CBF002382F8D4310023E1
S21444CAB010F8014B01391CF8016B17F801EBB4422E
S21444CAC02E7818BF013344EA060418BFDBB2764515
S21444CAD005F8014B1CBF0133DBB211F0FF01E7D16F
S21444CAE033B1B2F8BE301BB9BDE8F040FFF77CBEA8
S21444CAF0F0BD00BF10114220D41042201FB5144B85
S21444CB0001A953F820305A1E073312F8010F9A42EF
S21444CB1001F8010BF9D19DF804300024502B8DF810
S21444CB200C4007D0432B0CD0422B0DD0552B08BFBE
S21444CB304FF440040DF1050000F04CFA204404B0D4
S21444CB4010BD4FF48004F5E74FF40004F2E700BF4D
S21444CB50FC2040202DE9F04F5C4D8DB082462B687A
S21444CB6005F1080806AC09A963F07C4340462E4606
S21444CB70A9462B604246082316F8017B013B04F87D
S21444CB80017B9BB210F8017B01F8017B002BF3D1AB
S21444CB90BAF10A0F0BD141464C4C0823FF20013B07
S21444CBA004F8010B01F8010B9BB2002BF7D1484B5C
S21444CBB0C8240021013C03F8011BA4B2002CF9D17F
S21444CBC026464449DFF808B104F1080380279BB29F
S21444CBD000932B781F4203D198F800301F4248D068
S21444CBE051F824300DF10C0C581E073310F801EFA1
S21444CBF098420CF801EBF9D14FF000038DF814304D
S21444CC009DF80C30502B59D0432B59D0422B5AD038
S21444CC10552B34D14FF440030DF10D00019300F031
S21444CC20D9F9019B95F800C0184498F800302A4A70
S21444CC303B404FEA102E274918BF082317EA0C0F2B
S21444CC404FEA104C18BF43F001030BF806C006F138
S21444CC50010C1FFA8CFC0BF80CE006F1020C1FFAD0
S21444CC608CFC0BF80C00F01C043680B2B6B20BF801
S21444CC7000300134009B7F08A4B2A342A9D10135F9
S21444CC8008F1010895429FD1BAF10A0F0FD19DF8D9
S21444CC901A30BDF8182089F80230A9F800209DF80B
S21444CCA02630BDF8242089F80A30A9F80820084B15
S21444CCB0002230469A550DB0BDE8F08F0023ABE70E
S21444CCC04FF48003A8E74FF40003A5E7D4104220AE
S21444CCD032224020FC204020DC104220F0B50D4C8F
S21444CCE00822002004F1080514F8016B082380216B
S21444CCF00E4202D12F78394201D0013080B2013B36
S21444CD0049089BB2002BF3D1013A013592B2002A6E
S21444CD10EAD1F0BDD41042202DE9F04FDFF8B480BC
S21444CD20002685B08346A8F1080A3446284B022ECE
S21444CD304FF080094FF0000234BF082703272744EA
S21444CD40BFB29AF8001019EA010F04D198F80010FF
S21444CD5019EA010F2DD053F8241001AD481E0731AF
S21444CD6010F801CF814205F801CBF9D19DF80410A3
S21444CD708DF80C20502914D0432914D0422915D0BC
S21444CD8055291CD14FF440050DF1050000F022F959
S21444CD9005440F4B00225D450BD1E0B205B0BDE81B
S21444CDA0F08F0025F0E74FF48005EDE74FF40005DB
S21444CDB0EAE701344FEA5909A4B2A742C1D1013681
S21444CDC008F101080AF1010A082EB0D1FF20E5E770
S21444CDD0FC204020DC1042202DE9FF470024074673
S21444CDE0204EA146022C4FF0000834BF4FF0080AEC
S21444CDF04FF0030A336801A95A1E073312F8010F8D
S21444CE009A4201F8010BF9D19DF804308DF80C9044
S21444CE10502B0DD0432B15D0422B16D0552B17D064
S21444CE2001340436082CDDD1FF2004B0BDE8F08779
S21444CE3000250DF1050000F0CDF80544BD420AD1A9
S21444CE40E0B2F2E74FF48005F3E74FF40005F0E76D
S21444CE504FF44005EDE708F101081FFA88F39A45B8
S21444CE60C8D8DDE7FC2040202DE9F04FDFF8C49019
S21444CE70002585B08346A9F108082C462B4A022D86
S21444CE804FF0800A4FF0000134BF08270327274499
S21444CE90BFB298F800001AEA000F04D199F80000CF
S21444CEA01AEA000F32D052F824000DF1040C461E44
S21444CEB0073016F801EFB0420CF801EBF9D19DF8B3
S21444CEC004008DF80C10502818D0432818D0422857
S21444CED019D0552820D14FF440060DF1050000F036
S21444CEE079F80644124B00215E45104A0ED1595536
S21444CEF0E0B21D44297205B0BDE8F08F0026ECE789
S21444CF004FF48006E9E74FF40006E6E701344FEABB
S21444CF105A0AA4B2A742BCD1013509F1010908F165
S21444CF200108082DABD1FF20E5E700BFFC204020D8
S21444CF30D4104220DC1042207047092894BF303079
S21444CF403730C0B2704707B501220DF107018DF89E
S21444CF500700002013F0CCFB03B05DF804FB10B5CB
S21444CF60441E14F8010F00B910BDFFF7ECFFF8E7B4
S21444CF700FB400B5C3B044AA02A852F8041B0192E9
S21444CF8004F06AFC002302A88DF805318DF80631BA
S21444CF90FFF7E5FF43B05DF804EB04B070470D209F
S21444CFA008B5FFF7D0FF0A20BDE80840FFF7CBBF1F
S21444CFB010B504460009FFF7C0FFFFF7C4FF04F0AE
S21444CFC00F00FFF7BAFFFFF7BEFF2C20BDE8104066
S21444CFD0FFF7B9BF002330B51A46441E184614F866
S21444CFE0011F392908D82F290AD95D1C01F00F03DF
S21444CFF003EB00102B4606E0A1F14105052D06D9AA
S21444D00000B943B108220132072AE8D930BD5D1C75
S21444D010A1F13703ECE71D46EAE70020704700001D
S21444D020034A92F89E30013382F89E30704700BF20
S21444D0301011422010B52A4C94F89A30642B94BFB1
S21444D0400133002384F89A3094F8C63043B1013B48
S21444D050DBB284F8C6301BB984F8C53084F88A310C
S21444D06094F8C73053B1013BDBB284F8C7302BB9D0
S21444D07094F88A21032A08BF84F88A31B4F8E43144
S21444D0805BB1013B9BB2A4F8E43133B9012284F886
S21444D090CF3184F8C13184F8A52194F8C2310133E4
S21444D0A084F8C231FFF7F2FC94F8A13123B1002092
S21444D0B084F8A10101F01FFCB4F8BE3073B1013B03
S21444D0C09BB2A4F8BE304BB984F88A3184F8C53094
S21444D0D084F8A33184F8C13184F8DC3110BD00BF34
S21444D0E010114220034A92F89830013382F898305F
S21444D0F0704700BF1011422070470323002010B52C
S21444D100064CA4F8EC3104F154020823E16CF5F71C
S21444D1102FFC002384F8953010BD00BF1011422028
S21444D120024B0022C3E91522704700BF101142206B
S21444D13030B5224B002201244FF4FB604FF4FA61D1
S21444D140082583F8A541A3F89820A3F8B420C3F88B
S21444D150D420A3F8CA20A3F8CC2083F88121A3F8CE
S21444D160822183F88C2183F89C21C3F8A02183F87C
S21444D170D62183F8DB2183F8DC21A3F8E42183F865
S21444D180EA21A3F8C220C3F8C420D864196083F8FF
S21444D1909450A3F8C621C3F8D02183F8D421C3E918
S21444D1A072424FF40C14C3E92E22C3E96122C3F839
S21444D1B0C04183F8C421C3E92B1030BD101142206E
S21444D1C0144B002293F88D1183F88A21E1B9032287
S21444D1D0A3F8861183F8542093F8882142F040023D
S21444D1E083F8552093F89C21012A01BF7F2283F8B7
S21444D1F05520002283F89C21B3F8862152BAA3F81E
S21444D200562000229A65704746F60362A3F85420D7
S21444D210E8E700BF10114220054B3022A3F8542003
S21444D2200A2283F856200D2283F8C720704700BF91
S21444D23010114220034B012283F8C5200B2283F8A9
S21444D240C62070471011422008B5FFF783FC033010
S21444D250284B81B2284AC0B207291DD85921C3F8A1
S21444D260982183F8540083F8551093F89E1183F858
S21444D2705610FF2183F85710117883F858105178C8
S21444D28083F859109178D27883F85A1083F85B2043
S21444D2900422A3F8CA2008BDA3F8CC10090AC3F890
S21444D2A0982141F0100183F8550083F85410592111
S21444D2B083F8561093F89E1183F85710FF2183F88D
S21444D2C05810117883F859105178927883F85A1088
S21444D2D083F85B200322A3F8CA20012283F8C520E2
S21444D2E0022283F88A21212283F88C21222283F881
S21444D2F08821D0E71011422032224020024B0022DF
S21444D30083F85420704700BF1011422038B5CB1C18
S21444D31040F6FF749BB2A34228BF2346174C1D0A0F
S21444D32084F855306223A4F8CC1045F0100584F8F0
S21444D330580084F85630030A84F85450022163F0A7
S21444D3400F03C4F8982184F857300123A4F8CA3050
S21444D3501378A4F8CA1084F85930537884F85A30AD
S21444D3600323A4F8CA30937884F85B30FFF762FF4F
S21444D370212384F88A1184F88C3138BD1011422058
S21444D380F0B5C84C87B094F8C2310133DAB21B0604
S21444D3904ABF002384F8C22184F8C231B4F8C631A7
S21444D3A013B1013BA4F8C63194F8A03123B100234D
S21444D3B084F8A031FFF798FA94F88A51012D40F08A
S21444D3C0288194F888312E2B3DD146F60362A4F882
S21444D3D054206289A4F8562094F88D210D2A0BD146
S21444D3E0002384F88A31012384F8953040F2F513FB
S21444D3F0A4F8BE3007B0F0BD0E2AF4D194F88911D3
S21444D400A9480491A9490391B4F8CA10CDE9012169
S21444D41094F8C52029460092B4F88421FFF7A8FD65
S21444D42094F88931012B03D1002001F064FAD7E740
S21444D430022B03D1002001F079FAD1E7FF2BCFD19C
S21444D44084F8CB51CCE7222BCAD1B4F88431B3F557
S21444D450A06F6BD1964D0022964915F8010B1346E2
S21444D46001321F2892B204D9322A01F8010BF4D1B2
S21444D4701346E2182C213A2082F8E4105A1C422122
S21444D48014FA82F282F8E4109A1C4F2114FA82F2BB
S21444D49082F8E410DA1C14FA82F282F8E4101A1DB8
S21444D4A0542114FA82F282F8E4105A1D562114FAD2
S21444D4B082F282F8E410991DDA1D14FA81F192B2D0
S21444D4C081F8E4007C49087842281FD022444E2143
S21444D4D082F8E41003F10802302114FA82F282F84A
S21444D4E0E41003F10A010933202289B214FA83F3C3
S21444D4F083F8E4206318002201314FF4A06083F8D7
S21444D500E42089B26B4AFFF701FF6CE70B466B4D8C
S21444D5101878114601321F2892B2EBD901332144C0
S21444D520AB4281F8E400F3D11146E3E7644EB4F825
S21444D530862106EB4316B4F886C14FEA122E378985
S21444D540D0B29CFA9CFCF268FB1C99B2DBB2072969
S21444D5502FD984F85530C1F30321622384F857E069
S21444D56041F0100184F8580084F85630002384F8BB
S21444D57054100221A4F8CA30C4F89821A4F8CC70F8
S21444D5801378A4F8CA5084F859305378A4F8CA10CB
S21444D59084F85A30937884F85B300323A4F8CA306E
S21444D5A0FFF748FE322384F88A1184F8C6302123D4
S21444D5B074E0622184F85430A4F856C0013384F8E9
S21444D5C055100021C4F89821DBB2A4F8CA10A4F878
S21444D5D0CC701078A4F8CA5084F85800507884F870
S21444D5E059000220A4F8CA00907884F85A00032010
S21444D5F0A4F8CA00D27884F85B200422A4F8CA208F
S21444D600DAB2082A3FF4ECAEE218013382F854103A
S21444D610F6E7022D7FF4EEAE94F8C530002B7FF487
S21444D620E9AE94F88831222B7FF4DDAE94F8C4300A
S21444D630012B06D9023BDBB284F8C430002B7FF4BE
S21444D640D9AE94F8C330072194F88C212E27B4F829
S21444D650CC50D4F89861134884F8C43084F85420E5
S21444D660B4F8CA3001390130AB4238BF16F803C0AB
S21444D67003F101032CBF80F8547080F854C09BB269
S21444D68011F0FF01A4F8CA30EAD19D4202F1010329
S21444D690DBB298BF84F88A112F2B88D884F88C3153
S21444D6A0A1E600BF101142204E834600A812422035
S21444D6B000014400F411422020104000391040007C
S21444D6C0A87A4600FFF75CBE38B51B4C6389A4F8BD
S21444D6D09E31FFF713FE94F89E5105F0F703022B94
S21444D6E005D10123002584F89D31284638BD012DF7
S21444D6F00FD145F6061384F85650A4F8543094F8DF
S21444D7009F3184F85730FFF7E9FA40BAA4F8580036
S21444D710EBE7032D12BF47F6027345F6021384F86F
S21444D72056504FF001051BBFA4F854301223A4F8FA
S21444D730543084F85630D8E71011422008B5FFF725
S21444D740DDFD0B4B4CF20252A3F854209A7A012A80
S21444D75083F8562004D1002283F8D421012008BD42
S21444D760022A01D10122F7E77F2283F85520F5E704
S21444D77010114220064B47F60372A3F854200122A8
S21444D78083F8560083F8571083F89C21704700BFEF
S21444D79010114220074B93F8D621132A09D093F848
S21444D7A0A521032A1FBF7F2283F8D621012283F8AE
S21444D7B09C21704710114220002310B56B4C84F80E
S21444D7C0D63194F8CE30222B07D194F8D531032B9A
S21444D7D009D0132384F8D63105E0202B14D194F8CD
S21444D7E0D531022BF5D894F8D63163B147F6037297
S21444D7F084F857300123A4F8542094F8CE2084F8B3
S21444D8009C3184F8562010BD102B0BD194F8D5319A
S21444D810022BDED1A37A03F07F03013B022BE2D92D
S21444D8201223D7E7852B12D1A37A013B012B84BF61
S21444D830122384F8D63194F8D531022B02D0132320
S21444D84084F8D63194F8D601FFF7A4FFCBE7272B0C
S21444D85005D194F8D53103F0FB03022BB8E7192B16
S21444D86018D194F8D531012BB3D0A27A0A2AF4D031
S21444D870032AF2D0022AAAD0042A08D1062BA8D119
S21444D880A37B012BAFD0FF2BADD03123A2E7012AD7
S21444D890C6D19CE7282B1DD194F8D511A27A03292A
S21444D8A002F07F0305D0002BC9D0032BC7D0022932
S21444D8B002D0591E0129C2D912F07C0F01D012237E
S21444D8C0BEE7E27A013A022ABCD90BB1032BB9D19E
S21444D8D03123B5E7142B1CD194F8D531042B7FF4AF
S21444D8E078AFE07AA37A00EB0323207B00EB032097
S21444D8F06FF07F439842C4F8D0013FF474AF1C4B9A
S21444D90098423FF470AFFFF767FAFF287FF46BAF97
S21444D910BBE73E2B11D194F8D531022B7FF459AF97
S21444D920A37A13F07F0F4FF4FA7318BF1222A4F8A9
S21444D930E43118BF84F8D62155E7312B09D194F841
S21444D940D531062B3FF645AFA37A013B022B9CD834
S21444D95049E72E2B05D194F8D531022B7FF639AF03
S21444D96041E70F2B3FF63FAF112333E71011422018
S21444D970FF0040004FF287139842134B0ED10A29FA
S21444D9800AD1002283F8D62193F8D621003A18BF4C
S21444D990012283F8DB2170471322F3E74FF28B1200
S21444D9A0904201D10429EBE74FF29512904201D1FF
S21444D9B00329E5E74FF293129042F9D04FF28C12C6
S21444D9C09042DED10729DBE7101142200B4B02467A
S21444D9D093F90A00997A0028B3BF01F07F02012028
S21444D9E083F855200020B8BF9A724FF00102A8BFB2
S21444D9F083F8540083F8A521704700BF10114220D5
S21444DA00274B014610B593F90A009A7A0028BBBF03
S21444DA1002F07F02002001209A729A7A541E022C49
S21444DA2031D8062483F85510022A4FF0000183F8B3
S21444DA3054404FF4997483F85620A3F858404FF056
S21444DA40F40483F8571083F85A404FF4FA7483F872
S21444DA50A521A3F8E44112D1124A1278422A06D1EB
S21444DA6002F5800202F6DF7212784F2A03D00122B2
S21444DA7083F89C2103E00122084683F8CA21002249
S21444DA8083F8CF2110BD47F60372A3F8542093F8C9
S21444DA90CE2083F85620122283F85720E7E700BFAB
S21444DAA0101142202010400010B5214CA37AE07A91
S21444DAB000EB032080B2B0F5754FA4F886010BD175
S21444DAC04FF4A063A4F884310123002084F88A31FB
S21444DAD0222384F8883111E0B0F5704F12D300F059
S21444DAE0A9FD4FF6FF73984209D10223012084F81A
S21444DAF05430637A43F0400384F8553010BDA4F89C
S21444DB008401E1E740F2DF73D4F8E001C01A47F637
S21444DB100373A4F8543018BF012094F8CE3084F828
S21444DB205630312384F85730012384F89C31E5E796
S21444DB30101142202DE9F0414E4C2E23A27AE07A71
S21444DB4084F88831130900EB0220217B0E2B84F8DD
S21444DB508D3180B284F88911A4F886010DD1012351
S21444DB60002084F88A3194F8DB31012B71D1424A83
S21444DB70626584F89C31BDE8F081B0F5704F13D3EC
S21444DB8000F0C3FD0F230246A4F8840184F88D31C7
S21444DB904FF6FF73984204D0384E06EB4013D969CB
S21444DBA021B9032384F8DB310120DCE794F8CF1154
S21444DBB0012901D00223F5E7002084F89C0194F85B
S21444DBC0DB010028F0D19B6894F8D5010333DBB21F
S21444DBD0984207D013232A4884F8DB1184F8D631B8
S21444DBE0FFF7C6F9B4F884310027DFF89C80042593
S21444DBF006EB4313A4F8CA70DA689B68C4F8942109
S21444DC00A4F8CC30B4F8CA3018F8011BD4F89421E0
S21444DC10D154B4F8CA30B4F8CC2001339BB29A42FB
S21444DC20A4F8CA30C0D90020FFF7CAFA94F89C3149
S21444DC3084F8DB7143B9B4F8843106EB4313DB69EB
S21444DC40012B08BF84F8A131013D15F0FF05D9D159
S21444DC50AAE7022B03D10B4B6365012389E7032B09
S21444DC6001BF03F1445303F5391303F57C5363654D
S21444DC7081E700BF10114220037F2E13A87A460086
S21444DC809F834600037F2E331C114220204B0146BF
S21444DC9030B593F90A009A7A0028BBBF02F07F0297
S21444DCA0002001209A72DA7A02F0FD04012C22D177
S21444DCB09A7A02F0FD05012D11D183F8DC5193F8D0
S21444DCC0A521012A4FF0020283F854201AD87F2255
S21444DCD05A7222229A72002283F8DC2130BD12B98D
S21444DCE083F8DC21EBE7022A06BF002083F8DC41F8
S21444DCF083F89C41E3E7022A1FBF7F225A7212220E
S21444DD009A72DCE79A7A83F8551083F85620E5E74A
S21444DD1010114220704770477047704750B1232314
S21444DD200549013B00284FEA40009BB2B8BF484033
S21444DD30002BF6D1704700BF69696C6CF8B56C4B24
S21444DD40064693F8A5211C46012A0BD847F60372CB
S21444DD50A3F854205A7A83F856207F2283F8572013
S21444DD6001253DE0997A01F0FB05012D4AD10623B1
S21444DD7084F8550084F8561084F8543094F8CF311B
S21444DD80012B2FD101292DD10023A4F8A631A4F8C4
S21444DD90A83194F8A661012994F8A72194F8A831EB
S21444DDA018BF022184F8582002EB062294F8A901F1
S21444DDB084F8593003EB022384F85A0000EB03201E
S21444DDC084F85760FFF7AAFF030E84F8A631030CC5
S21444DDD040BA84F8A7310123A4F8A80184F8C131D5
S21444DDE02846F8BD94F8C23103F1110284F8A631EE
S21444DDF084F8A72103F12202343384F8A82184F856
S21444DE00A931C6E7022DABD193F8C121012A4FF0C0
S21444DE10000210D083F8C12147F603720125A3F807
S21444DE20542093F8CE2083F89C5183F8562024221D
S21444DE3083F85720D4E783F8C121DA7A93F8A631D9
S21444DE409A420AD1227B94F8A7319A4205D1B4F873
S21444DE50A821B4F80D309A421DD047F6037306291C
S21444DE60A4F8543094F8CE3084F856304FF0350346
S21444DE7084F857304FF0010384F89C317FF470AF38
S21444DE801C4B1B78422B08D001231B4884F89C313A
S21444DE90FFF76EF801E00629F2D094F89C51002D65
S21444DEA07FF45EAFA37A022784F8556084F8563030
S21444DEB084F85470FFF721F9A37A062B0ED1012378
S21444DEC00E4884F8CF7184F8CA31FFF748F80B48F7
S21444DED0FFF745F80948FFF742F881E794F8A5317B
S21444DEE0023B012B9CBF012384F8CF3178E700BF67
S21444DEF01011422020104000B3834600118446008F
S21444DF00114B002293F89C1183F8D621012904BFB3
S21444DF107F2183F89C2193F8CE2008BF83F85510C0
S21444DF20312A0DD193F8D511062903D9132283F843
S21444DF30D62103E0997A01390229F8D8012070479E
S21444DF40342AFBD11222F2E71011422070B5674CF6
S21444DF500025637A264694F8DD2184F8CE30237A69
S21444DF6084F89C519A4284F8D53101D800200FE0B9
S21444DF70013B062BFAD8FFF71FFC94F89C31012B83
S21444DF800FD1D4F8E02140F2DF739A4201D0012049
S21444DF9070BD94F8D631113B012BF8D884F89C51C7
S21444DFA0E4E7627A94F8CE30102A43F0400003D176
S21444DFB0BDE87040FFF724BD202A03D1BDE8704079
S21444DFC0FFF704BD852A03D1BDE87040FFF7B6BB12
S21444DFD02A2B0AD1E37A84F8C33146F60223A4F8FE
S21444DFE05430A37A84F85630D1E7222B04D16220E9
S21444DFF0BDE87040FFF758BD2E2B04D16E20BDE817
S21444E0007040FFF797BD282B04D16820BDE87040C8
S21444E010FFF73CBE2F2B0ED146F60673344AA4F8BF
S21444E02054300623013B12F8011B13F0FF0382F819
S21444E0304B10F7D1ABE7142B15D1FFF75FF9D4F8A3
S21444E040D0016FF07F43984202D02A4B984207D1C2
S21444E050012386F8A03145F20143A6F8543096E7EA
S21444E060FEF702FFF7E7272B04D16720BDE8704090
S21444E070FFF764BE192B03D1BDE87040FFF724BBFD
S21444E080312B0BD11C4A0723013B12F8011B13F01A
S21444E090FF0382F8DA10F7D1712079E7112B0FD1FC
S21444E0A045F20213A4F85430A37A84F85630FFF7A6
S21444E0B024F81248FEF753FF1148FEF750FF66E770
S21444E0C03E2B0FD194F90A10A37A0029FFF64EAFDF
S21444E0D0022142F0400284F8563084F8541084F802
S21444E0E0552054E7FEF79CFF40E700BF101142203E
S21444E0F01A114220FF00400019114220BD834600F9
S21444E100D283460038B5424C0F2384F88D312546D9
S21444E110237A217B03F00F02637AE07A03EB02232F
S21444E12004F1E40201EB0020C4F8942142F2030215
S21444E13080B2A4F8CC30A4F88A2194F8CE202F2AB2
S21444E14023D1033B2E22A4F87A019BB284F888217B
S21444E15004F22F12A4F88601A4F8CC3084F879315E
S21444E160A37BC4F8942184F831310423627BA4F859
S21444E170CA30E37B84F87C2184F82F1184F830215C
S21444E18084F83231FFF748F814E0A4F8860100F02A
S21444E19051FA4FF6FF7398420ED147F60372312375
S21444E1A0A5F8542095F8CE2085F8D63185F8562023
S21444E1B085F85730012038BD164B03EB4013DA6917
S21444E1C0002AEAD02E22A4F8840184F88821032267
S21444E1D084F88A21DA689B68C4F89421A4F8CC3081
S21444E1E00123A4F8CA30637B1370B4F8CA30D4F859
S21444E1F09421591CA4F8CA10A17BD154B4F8CA304F
S21444E200D4F89421591CA4F8CA10E17BD154B9E738
S21444E21010114220A87A460008B51A4B0022197AF3
S21444E22083F88D2101F00F00597AA3F8842101EB7D
S21444E23000219A7AC82983F888211A7B88BFC82186
S21444E24083F8E520A3F8CC10D97A02EB01205A7B58
S21444E25083F8E41083F8E6209A7BA3F8860142F21A
S21444E260030083F8E720DA7BA3F88A0183F8E820E2
S21444E27005220548A3F8CA20C3F89401FEF7CCFF4C
S21444E280012008BD1011422032224020184B0022A3
S21444E290987A83F8D62183F89C21A0F12E0283F83D
S21444E2A0CE00D1B208291DD840F24912CA40D24302
S21444E2B012F0010216D12E2883F8DB2114D193F8EC
S21444E2C0A521012A02D993F8CF216AB97E2283F880
S21444E2D0D62102F17E2202F5381285325A65012291
S21444E2E083F89C21012070470020FFF70BBF00BF36
S21444E2F010114220002340F2F51210B5884C84F8E1
S21444E300983084F89C31A4F8BE204FF4FA72C4E9DD
S21444E31015332368A4F8E421B3F5FA6F17D1431EE6
S21444E32004F10802073013F8011F984202F8011B53
S21444E330F9D14FF4FA63C4F8E031227A12F0F003CC
S21444E3402BD1FFF703FE002840F08B804CE040F2D0
S21444E350DF72934220D1037813F0F00F1CD1427839
S21444E360A2F11003DBB2182B11D9852A01D03E2A1C
S21444E37012D140F2DF736B4AC4F8E031431E0730D3
S21444E38013F8011F834202F8011BF9D1D5E7664A08
S21444E39022FA03F3DB07ECD410BD102B02D1FFF7AF
S21444E3A075FFD0E7202B40F08F8094F8CE302E3B7C
S21444E3B0D9B206295CD84923CB40DB4313F001038A
S21444E3C056D194F88A1103290ED194F8DD11072901
S21444E3D010D8B4F8CA3001391944B4F8CC3099424C
S21444E3E002D2002384F88A31002384F89C3184F8CE
S21444E3F09830D1E794F88B11914205D14B4884F874
S21444E4008A31FEF7ACFDEFE784F88B210D2284F8C1
S21444E410C72094F8DB2132B9E218D4F89411507A24
S21444E420B4F8CA208854B4F8CA20B4F8CC100132E0
S21444E43092B29142A4F8CA2042D894F8DB31012B18
S21444E4401AD147F60372A4F8542094F8CE2084F8E0
S21444E4505620132284F8572084F89C31002384F8ED
S21444E460DB3194F89C31012B04BF7F2384F855306C
S21444E470012384F89530B7E7022B0CD147F6037393
S21444E480A4F8543094F8CE3084F85630332384F8C5
S21444E49057300123E0E70020FEF792FEB4F88421CB
S21444E4A0234B94F89C1103EB42132248DA69012A61
S21444E4B008BF84F8A12194F8A131FEF759FDCDE7B1
S21444E4C00133072BA5D18FE7302B8DD194F8DD315E
S21444E4D0022B86D9312A03D10B2384F8C63083E72E
S21444E4E094F8C5305BB9322A09D146F20323A4F81E
S21444E4F05430B4F886315BBAA4F856304CE7A37A65
S21444E5000021312A03F1030384F8C51084F8C610A9
S21444E510DBB284F8C33084F8C4303FF662AF63E7B6
S21444E520101142201811422013020401E2834600CF
S21444E530A87A4600FA8346000A4810B5FEF718FD46
S21444E54072B64FF0005308491022084C0848C3E9F5
S21444E5500012FEF70DFDFBF7E8FA2046FEF708FD2D
S21444E560FBE700BF0C8446007154CA3D3384460022
S21444E5701984460038B52C4B93F8C8211C4632B94A
S21444E580FEF7D6FD2948BDE83840FEF7E8BC93F8C8
S21444E5909820002A3FD0002293F89D1183F89820B3
S21444E5A081B193F89E0183F89D21FEF74DFE012329
S21444E5B084F8953040F2F513A4F8BE30BDE83840F0
S21444E5C0FEF79BBD93F89550002DF3D1184A137867
S21444E5D00133DBB2022B01D8137038BD1570FEF739
S21444E5E0CFFE94F8993094F8C22101330132DBB25D
S21444E5F084F8C221042B84F899300CD984F89950B5
S21444E600FEF718FDB4F89C30C72B96BF0133A4F828
S21444E6109C50A4F89C3094F8CA2194F8CB31134308
S21444E620DBD0FFF789FF00BF10114220428446002A
S21444E630F82140204FF22803984218D84FF20F038F
S21444E640984259D9A0F57040113817280DD8DFE8FC
S21444E65000F056292B2D2F3131333537393B3D3F8A
S21444E6604143454547494B4D4F51042070474FF26F
S21444E6709313984245D00CD84FF28713984242D011
S21444E6804FF288124FF6FF73904214BF184601208B
S21444E69070474FF295124FF6FF73904214BF1846D8
S21444E6A002207047062070470720704708207047AE
S21444E6B0092070470A2070470B2070470C2070478B
S21444E6C00D2070470E2070470F207047102070476B
S21444E6D0112070471220704713207047142070474B
S21444E6E0152070471620704717207047182070472B
S21444E6F0192070471A2070474FF6FF707047052060
S21444E70070470320704700207047FFF793BF1C28CC
S21444E7100146F0B585B037D83F4B420103EB40166F
S21444E7209C584FF6FF739C422ED0F369012B2BD195
S21444E730756804F50004B368AD082246009337486C
S21444E7402B46FEF715FCD6E903639A1E012A1DD80C
S21444E750002315E036F82310023389B20291029959
S21444E760090402915088029901440291918889B221
S21444E7700391039909040391D188039A0A440392A6
S21444E7809D4206EB8302E5D805B0F0BD043B012B61
S21444E7903FD90027BD4206EB8701F5D916F8273046
S21444E7A0204602370834DBB20293029B1B060293D0
S21444E7B04A78029B03EB024302938A78029B03EB5C
S21444E7C002230293CB78029A134402930B79DBB26A
S21444E7D00393039B1B0603934A79039B03EB024371
S21444E7E003938A79039B03EB02230393CB7902A911
S21444E7F0039A13440393FEF710FCCBE756F8231012
S21444E80002330291526803929D4206EB8302F5D886
S21444E810BAE70023F8E700BFA87A46004D844600CE
S21444E8201C28014630B403D92C4830BCFEF7A0BBA4
S21444E83042012B4B03EB40109B584FF6FF7293421A
S21444E8401FD0C269012A1CD10169072919D08268E0
S21444E85003F50003C468881E012814D852080234FD
S21444E860002191420DD253F8040B050C24F8025CA7
S21444E8704D1C954205D2023180B28A4224F8040BDC
S21444E880EFD830BC70470439012925D822F003025A
S21444E89022449442F5D053F8041B44F8041BF8E78A
S21444E8A05858050E25704D1CAA42EAD9C0F30745B0
S21444E8B065708D1CAA42E4D9C0F30725A570CD1C0B
S21444E8C0AA42DED90431C0B204348A4204F8010CA8
S21444E8D0D7D99142E4D3D4E70021FAE76E844600C0
S21444E8E0A87A460010B50024A0B20134FFF798FF7A
S21444E8F01D2CF9D110BD1FB50024A0B20134FFF77A
S21444E90006FF1D2CF9D1074B02A902934FF47C73E2
S21444E9100393054B01930198FEF77FFB002004B058
S21444E92010BD00BF55EFCDAB1000800008B508B948
S21444E930FFF7D8FF002008BD124B00B51B688BB00C
S21444E9400293114B1A6803925A6804929B68059383
S21444E9500299039A049B059800900C48FEF708FB1E
S21444E960039BB3F57C7F06D10948FEF701FB0120E3
S21444E9700BB05DF804FB0748FEF7FAFA4FF0FF3099
S21444E980F6E700BF10008000140080007E84460036
S21444E99096844600A184460008B5FFF7CDFF0128BB
S21444E9A005D1FFF79FFFBDE80840FDF7B9BFFFF765
S21444E9B0C3FF0128F5D00020FFF79DFFFFF7BCFFFB
S21444E9C0F1E700BF10F8012B11F8013B012A28BFDC
S21444E9D09A42F7D0D01A7047034613F8012B002A00
S21444E9E0FBD1181A013870470000000000000000F0
S21444E9F001F0FF01102A2BDB10F0070F08D010F8A7
S21444EA00013B013A8B422DD010F0070F42B3F6D1AA
S21444EA10F0B441EA012141EA014122F007047FF0C3
S21444EA2000070023F0E80256083C85EA010586EA1A
S21444EA30010685FA47F5A3FA87F586FA47F6A5FA56
S21444EA4087F68EB9EED1F0BC01F0FF0102F0070262
S21444EA5032B110F8013B013A83EA010313B1F8D10D
S21444EA600020704701387047002D06BF35460338EE
S21444EA70073815F0010F07D1013015F4807F02BF27
S21444EA80013015F4C03F0130F0BC0138704700BF78
S21444EA9081F0004102E000BF83F0004330B54FEA06
S21444EAA041044FEA430594EA050F08BF90EA020F73
S21444EAB01FBF54EA000C55EA020C7FEA645C7FEA06
S21444EAC0655C00F0E2804FEA5454D4EB5555B8BF29
S21444EAD06D420CDD2C4480EA020281EA030382EA9A
S21444EAE0000083EA010180EA020281EA0303362D2C
S21444EAF088BF30BD11F0004F4FEA01314FF4801CFF
S21444EB004CEA113102D0404261EB410113F0004F10
S21444EB104FEA03334CEA133302D0524263EB4303C7
S21444EB2094EA050F00F0A780A4F10104D5F1200E65
S21444EB300DDB02FA0EFC22FA05F2801841F10001C0
S21444EB4003FA0EF2801843FA05F359410EE0A5F194
S21444EB5020050EF1200E012A03FA0EFC28BF4CF0C5
S21444EB60020C43FA05F3C01851EBE37101F000457B
S21444EB7007D54FF0000EDCF1000C7EEB00006EEB88
S21444EB800101B1F5801F1BD3B1F5001F0CD3490812
S21444EB905FEA30004FEA3C0C04F101044FEA445269
S21444EBA012F5800F80F09A80BCF1004F08BF5FEAF0
S21444EBB0500C50F1000041EB045141EA050130BDD0
S21444EBC05FEA4C0C404141EB0101013C28BFB1F5E2
S21444EBD0801FE9D291F0000F04BF01460020B1FA2D
S21444EBE081F308BF2033A3F10B03B3F120020CDA00
S21444EBF00C3208DD02F1140CC2F10C0201FA0CF0DE
S21444EC0021FA02F10CE002F11402D8BFC2F1200C42
S21444EC1001FA02F120FA0CFCDCBF41EA0C019040F8
S21444EC20E41AA2BF01EB0451294330BD6FEA040441
S21444EC301F3C1CDA0C340EDC04F11404C4F120022C
S21444EC4020FA04F001FA02F340EA030021FA04F33E
S21444EC5045EA030130BDC4F10C04C4F1200220FA95
S21444EC6002F001FA04F340EA0300294630BD21FAD3
S21444EC7004F0294630BD94F0000F83F4801306BF99
S21444EC8081F480110134013D4EE77FEA645C18BF8D
S21444EC907FEA655C29D094EA050F08BF90EA020F24
S21444ECA005D054EA000C04BF1946104630BD91EA1C
S21444ECB0030F1EBF0021002030BD5FEA545C05D11F
S21444ECC04000494128BF41F0004130BD14F580045E
S21444ECD03CBF01F5801130BD01F0004545F0FE41D2
S21444ECE041F470014FF0000030BD7FEA645C1ABF07
S21444ECF0194610467FEA655C1CBF0B46024650EA3E
S21444ED00013406BF52EA033591EA030F41F4002169
S21444ED1030BD00BF90F0000F04BF0021704730B5EF
S21444ED204FF4806404F132044FF000054FF00001C4
S21444ED3050E700BF90F0000F04BF0021704730B585
S21444ED404FF4806404F1320410F0004548BF40425A
S21444ED504FF000013EE700BF42004FEAE2014FEAAF
S21444ED6031014FEA02701FBF12F07F4393F07F4F8A
S21444ED7081F06051704732F07F4208BF704793F08D
S21444ED807F4F04BF41F40021704730B54FF46074A0
S21444ED9001F0004521F000411CE700BF50EA0102A3
S21444EDA008BF704730B54FF000050AE050EA01024C
S21444EDB008BF704730B511F0004502D5404261EBBC
S21444EDC041014FF4806404F132045FEA915C3FF4FD
S21444EDD0D8AE4FF003025FEADC0C18BF03325FEA9A
S21444EDE0DC0C18BF033202EBDC02C2F1200300FA4B
S21444EDF003FC20FA02F001FA03FE40EA0E0021FA70
S21444EE0002F11444BDE600BF70B54FF0FF0C4CF45D
S21444EE10E06C1CEA11541DBF1CEA135594EA0C0F0F
S21444EE2095EA0C0F00F0DEF82C4481EA030621EA4A
S21444EE304C5123EA4C5350EA013518BF52EA033585
S21444EE4041F4801143F4801338D0A0FB02CE4FF037
S21444EE500005E1FB02E506F00042E0FB03E54FF067
S21444EE600006E1FB03569CF0000F18BF4EF0010E5F
S21444EE70A4F1FF04B6F5007F64F5407404D25FEA5B
S21444EE804E0E6D4146EB060642EAC62141EA55510E
S21444EE904FEAC52040EA5E504FEACE2EB4F1FD0C50
S21444EEA088BFBCF5E06F1ED8BEF1004F08BF5FEACE
S21444EEB0500E50F1000041EB045170BD06F0004680
S21444EEC046EA010140EA020081EA0301B4EB5C042D
S21444EED0C2BFD4EB0C0541EA045170BD41F4801125
S21444EEE04FF0000E013C00F3AB8014F1360FDEBF4A
S21444EEF0002001F0004170BDC4F10004203C35DA26
S21444EF000C341BDC04F11404C4F1200500FA05F3A8
S21444EF1020FA04F001FA05F240EA020001F0004249
S21444EF2021F0004110EBD37021FA04F642EB0601BF
S21444EF305EEA430E08BF20EAD37070BDC4F10C04E9
S21444EF40C4F1200500FA04F320FA05F001FA04F2AD
S21444EF5040EA020001F0004110EBD37041F1000199
S21444EF605EEA430E08BF20EAD37070BDC4F12005A4
S21444EF7000FA05F24EEA020E20FA04F301FA05F20C
S21444EF8043EA020321FA04F001F0004121FA04F2B4
S21444EF9020EA020000EBD3705EEA430E08BF20EA84
S21444EFA0D37070BD94F0000F0FD101F000464000BE
S21444EFB041EB010111F4801F08BF013CF7D041EA40
S21444EFC0060195F0000F18BF704703F00046520044
S21444EFD043EB030313F4801F08BF013DF7D043EA15
S21444EFE00603704794EA0C0F0CEA135518BF95EACB
S21444EFF00C0F0CD050EA410618BF52EA4306D1D152
S21444F00081EA030101F000414FF0000070BD50EA70
S21444F010410606BF1046194652EA430619D094EAFA
S21444F0200C0F02D150EA013613D195EA0C0F05D1E4
S21444F03052EA03361CBF104619460AD181EA030138
S21444F04001F0004141F0FE4141F470014FF00000F0
S21444F05070BD41F0FE4141F4780170BD70B54FF08B
S21444F060FF0C4CF4E06C1CEA11541DBF1CEA13550B
S21444F07094EA0C0F95EA0C0F00F0A7F8A4EB0504ED
S21444F08081EA030E52EA03354FEA013100F08880E4
S21444F0904FEA03334FF0805545EA131343EA1263AD
S21444F0A04FEA022245EA111545EA10654FEA002662
S21444F0B00EF000419D4208BF964244F1FD0404F51B
S21444F0C0407402D25B084FEA3202B61A65EB030577
S21444F0D05B084FEA32024FF480104FF4002CB6EB34
S21444F0E0020E75EB030E22BFB61A754640EA0C00B4
S21444F0F05B084FEA3202B6EB020E75EB030E22BFF4
S21444F100B61A754640EA5C005B084FEA3202B6EB34
S21444F110020E75EB030E22BFB61A754640EA9C00F3
S21444F1205B084FEA3202B6EB020E75EB030E22BFC3
S21444F130B61A754640EADC0055EA060E18D04FEA81
S21444F140051545EA16754FEA06164FEAC30343EA21
S21444F15052734FEAC2025FEA1C1CC0D111F4801FEE
S21444F1600BD141EA00014FF000004FF0004CB6E7E7
S21444F17011F4801F04BF01430020B4F1FD0C88BF86
S21444F180BCF5E06F3FF6AFAEB5EB030C04BFB6EB91
S21444F190020C5FEA500C50F1000041EB045170BD84
S21444F1A00EF0004E4EEA113114EB5C04C2BFD4EBB1
S21444F1B00C0541EA045170BD41F480114FF0000E35
S21444F1C0013C90E645EA060E8DE60CEA135594EAB1
S21444F1D00C0F08BF95EA0C0F3FF43BAF94EA0C0FB4
S21444F1E00AD150EA01347FF434AF95EA0C0F7FF429
S21444F1F025AF104619462CE795EA0C0F06D152EA7D
S21444F20003353FF4FDAE1046194622E750EA410660
S21444F21018BF52EA43067FF4C5AE50EA41047FF471
S21444F2200DAF52EA43057FF4EBAE12E74FF0FF3CD6
S21444F23006E000BF4FF0010C02E000BF4FF0010CA7
S21444F2404DF804CD4FEA410C7FEA6C5C4FEA430C20
S21444F25018BF7FEA6C5C1BD001B050EA410C0CBF6F
S21444F26052EA430C91EA030F02BF90EA020F0020D1
S21444F270704710F1000F91EA030F58BF994208BF38
S21444F28090422CBFD8176FEAE37040F001007047F5
S21444F2904FEA410C7FEA6C5C02D150EA013C07D14C
S21444F2A04FEA430C7FEA6C5CD6D152EA033CD3D097
S21444F2B05DF8040B704700BF8446104662468C4691
S21444F2C01946634600E000BF01B5FFF7B7FF0028C4
S21444F2D048BF10F1000F01BD4DF808EDFFF7F4FFED
S21444F2E00CBF012000205DF808FB00BF4DF808ED78
S21444F2F0FFF7EAFF34BF012000205DF808FB00BF9B
S21444F3004DF808EDFFF7E0FF94BF012000205DF8BC
S21444F31008FB00BF4DF808EDFFF7CEFF94BF012071
S21444F32000205DF808FB00BF4DF808EDFFF7C4FF6A
S21444F33034BF012000205DF808FB00BF4FEA410CB3
S21444F3407FEA6C5C02D150EA013C0AD14FEA430C96
S21444F3507FEA6C5C02D152EA033C02D14FF00000D3
S21444F36070474FF0010070474FEA410212F5001211
S21444F37015D211D56FF47873B3EB625212D94FEAB3
S21444F380C12343F0004343EA505311F0004F23FA9D
S21444F39002F018BF404270474FF00000704750EAF2
S21444F3A0013005D111F0004008BF6FF000407047AF
S21444F3B04FF00000704700BF4A0011D212F5001209
S21444F3C011D20DD56FF47873B3EB62520ED44FEA74
S21444F3D0C12343F0004343EA505323FA02F07047F4
S21444F3E04FF00000704750EA013002D14FF0FF3032
S21444F3F070474FF0000070474FEA4102B2F1E043D5
S21444F40024BFB3F5001CDCF1FE5C0DD901F0004CC2
S21444F4104FEAC0024CEA5070B2F1004F40EB830012
S21444F42008BF20F00100704711F0804F21D113F13E
S21444F4303872BCBF01F00040704741F480114FEA77
S21444F4405252C2F11802C2F1200C10FA0CF320FA00
S21444F45002F018BF40F001004FEAC1234FEAD3231D
S21444F46003FA0CFC40EA0C0023FA02F34FEA430387
S21444F470CCE77FEA625307D150EA01331EBF4FF010
S21444F480FE4040F44000704701F0004040F0FE402B
S21444F49040F40000704700BF80F0004002E000BF28
S21444F4A081F0004142001FBF5FEA410392EA030F26
S21444F4B07FEA226C7FEA236C6AD04FEA1262D2EB70
S21444F4C01363C1BFD218414048404140B8BF5B4275
S21444F4D0192B88BF704710F0004F40F4000020F00E
S21444F4E07F4018BF404211F0004F41F4000121F024
S21444F4F07F4118BF494292EA030F3FD0A2F101026E
S21444F50041FA03FC10EB0C00C3F1200301FA03F1AB
S21444F51000F0004302D5494260EB4000B0F5000FCE
S21444F52013D3B0F1807F06D340084FEA310102F18D
S21444F5300102FE2A51D2B1F1004F40EBC25008BF3F
S21444F54020F0010040EA03007047490040EB000009
S21444F550013A28BFB0F5000FEDD2B0FA80FCACF10A
S21444F560080CB2EB0C0200FA0CF0AABF00EBC25037
S21444F57052421843BCBFD0401843704792F0000F25
S21444F58081F4000106BF80F400000132013BB5E778
S21444F5904FEA41037FEA226C18BF7FEA236C21D0EE
S21444F5A092EA030F04D092F0000F08BF0846704753
S21444F5B090EA010F1CBF0020704712F07F4F04D121
S21444F5C0400028BF40F00040704712F100723CBF34
S21444F5D000F50000704700F0004343F0FE4040F45E
S21444F5E0000070477FEA226216BF08467FEA23631C
S21444F5F00146420206BF5FEA412390EA010F40F407
S21444F600800070474FF0000304E000BF10F0004352
S21444F61048BF40425FEA000C08BF704743F0964339
S21444F62001464FF000001CE050EA010208BF704754
S21444F6304FF000030AE000BF50EA010208BF7047DB
S21444F64011F0004302D5404261EB41015FEA010CF0
S21444F65002BF84460146002043F0B64308BFA3F1E8
S21444F6608053A3F50003BCFA8CF2083AA3EBC253CA
S21444F67010DB01FA02FC634400FA02FCC2F12002E9
S21444F680BCF1004F20FA02F243EB020008BF20F020
S21444F6900100704702F1200201FA02FCC2F1200286
S21444F6A050EA4C0021FA02F243EB020008BF20EA7B
S21444F6B0DC7070474FF0FF0C1CEAD0521EBF1CEAA9
S21444F6C0D15392EA0C0F93EA0C0F6FD01A4480EA97
S21444F6D0010C400218BF5FEA41211ED04FF0006380
S21444F6E043EA501043EA5111A0FB01310CF00040AC
S21444F6F0B1F5000F3EBF490041EAD3715B0040EAD2
S21444F700010062F17F02FD2A1DD8B3F1004F40EBA1
S21444F710C25008BF20F00100704790F0000F0CF074
S21444F720004C08BF49024CEA502040EA51207F3A38
S21444F730C2BFD2F1FF0340EAC250704740F4000013
S21444F7404FF00003013A5DDC12F1190FDCBF00F004
S21444F75000407047C2F10002410021FA02F1C2F1B2
S21444F760200200FA02FC5FEA310040F1000053EA4E
S21444F7704C0308BF20EADC70704792F0000F00F09C
S21444F780004C02BF400010F4000F013AF9D040EAA2
S21444F7900C0093F0000F01F0004C02BF490011F436
S21444F7A0000F013BF9D041EA0C018FE70CEAD15334
S21444F7B092EA0C0F18BF93EA0C0F0AD030F0004CB4
S21444F7C018BF31F0004CD8D180EA010000F0004068
S21444F7D0704790F0000F17BF90F0004F084691F026
S21444F7E0000F91F0004F14D092EA0C0F01D1420260
S21444F7F00FD193EA0C0F03D14B0218BF084608D129
S21444F80080EA010000F0004040F0FE4040F4000072
S21444F810704740F0FE4040F4400070474FF0FF0C05
S21444F8201CEAD0521EBF1CEAD15392EA0C0F93EA4C
S21444F8300C0F69D0A2EB030280EA010C49024FEA9E
S21444F840402037D04FF0805343EA111143EA101357
S21444F8500CF000408B4238BF5B0042F17D024FF40F
S21444F860000C8B4224BF5B1A40EA0C00B3EB510FEA
S21444F87024BFA3EB510340EA5C00B3EB910F24BFD3
S21444F880A3EB910340EA9C00B3EBD10F24BFA3EB58
S21444F890D10340EADC001B0118BF5FEA1C1CE0D120
S21444F8A0FD2A3FF650AF8B4240EBC25008BF20F0D3
S21444F8B0010070470CF0004C4CEA50207F32C2BF27
S21444F8C0D2F1FF0340EAC250704740F400004FF0C4
S21444F8D00003013A37E792F0000F00F0004C02BFF5
S21444F8E0400010F4000F013AF9D040EA0C0093F0BF
S21444F8F0000F01F0004C02BF490011F4000F013B19
S21444F900F9D041EA0C0195E70CEAD15392EA0C0F80
S21444F91008D142027FF47DAF93EA0C0F7FF470AFB8
S21444F920084676E793EA0C0F04D14B023FF44CAFFB
S21444F93008466EE730F0004C18BF31F0004CCAD190
S21444F94030F000427FF45CAF31F000437FF43CAFCC
S21444F9505FE700BF4FF0FF3C06E000BF4FF0010CEE
S21444F96002E000BF4FF0010C4DF804CD4FEA4002D0
S21444F9704FEA41037FEA226C18BF7FEA236C11D01A
S21444F98001B052EA530C18BF90EA010F58BFB2EBCD
S21444F990030088BFC81738BF6FEAE17018BF40F04D
S21444F9A0010070477FEA226C02D15FEA402C05D101
S21444F9B07FEA236CE4D15FEA412CE1D05DF8040B86
S21444F9C0704700BF844608466146FFE70FB5FFF719
S21444F9D0C9FF002848BF10F1000F0FBD4DF808EDD1
S21444F9E0FFF7F4FF0CBF012000205DF808FB00BFC2
S21444F9F04DF808EDFFF7EAFF34BF012000205DF81C
S21444FA0008FB00BF4DF808EDFFF7E0FF94BF012068
S21444FA1000205DF808FB00BF4DF808EDFFF7D2FF65
S21444FA2094BF012000205DF808FB00BF4DF808EDA8
S21444FA30FFF7C8FF34BF012000205DF808FB00BF75
S21444FA4042000ED2B2F1FE4F0BD34FF09E03B3EBFF
S21444FA50126209D44FEA002343F0004323FA02F02B
S21444FA6070474FF00000704712F1610F01D1420217
S21444FA7002D14FF0FF3070474FF00000704700BF90
S21444FA8053B94AB9002908BF00281CBF4FF0FF31BC
S21444FA904FF0FF3000F0A6B9ADF1080C6DE904CE86
S21444FAA000F03EF8DDF804E0DDE9022304B07047D8
S21444FAB038B505460C462846214600220023FFF763
S21444FAC015FC28B928462146BDE8384000F00AB857
S21444FAD0284604F1004100F005F8404261EB41013C
S21444FAE038BD00BFD0B50C4B002206460F46FFF784
S21444FAF08BF9FFF761FC0446FFF70CF9074B00222D
S21444FB00FFF782F902460B4630463946FEF7C4FFF5
S21444FB10FFF752FC2146D0BD0000F03D0000F04106
S21444FB202DE9F047089D0E4604468C46002B40F0CF
S21444FB3081808A42174645D9B2FA82F24AB1C2F166
S21444FB40200106FA02F320FA01F1974041EA030C39
S21444FB5094404FEA174E230CBCFBFEF6B9B20EFB9C
S21444FB6016CC43EA0C4306FB01F0984209D9FB182D
S21444FB7006F1FF3C80F01581984240F21281023E25
S21444FB803B441B1AA4B2B3FBFEF00EFB103344EA0C
S21444FB90034400FB01F1A14209D93C1900F1FF33AB
S21444FBA080F00181A14240F2FE8002383C44641A4F
S21444FBB040EA064000211DB1D4400023C5E9004375
S21444FBC0BDE8F08702B9FFDEB2FA82F2002A4FD1CE
S21444FBD0CB1B4FEA174E1FFA87F80121B3FBFEFCF6
S21444FBE0260C0EFB1C3346EA034608FB0CF3B342D2
S21444FBF007D9BE190CF1FF3002D2B34200F2EB80B3
S21444FC008446F61AA3B2B6FBFEF00EFB106643EA31
S21444FC10064408FB00F8A04507D93C1900F1FF3319
S21444FC2002D2A04500F2D2801846A4EB080440EA6B
S21444FC300C40C0E78B4208D9002D00F0AF8000216D
S21444FC40C5E900060846BDE8F087B3FA83F1002903
S21444FC5049D1B34202D3824200F2BB80841A66EB97
S21444FC60030301209C46002DAAD0C5E9004CA7E713
S21444FC70C2F120039740D8409140DE404FEA174EE9
S21444FC8008434FEA104CB6FBFEF11FFA87F80EFB0A
S21444FC9011664CEA064601FB08F3B34204FA02F442
S21444FCA009D9BE1901F1FF3C80F08E80B34240F280
S21444FCB08B8002393E44F31A86B2B3FBFEF00EFB49
S21444FCC0103346EA034600FB08F3B34207D9BE198D
S21444FCD000F1FF3C74D2B34272D902383E44F31A60
S21444FCE040EA01417AE7C1F1200703FA01F422FA17
S21444FCF007F31C4320FA07F906FA01F34FEA144CBB
S21444FD00FE4049EA03094FEA1943B6FBFCFE1FFAD4
S21444FD1084F80CFB1E6643EA06460EFB08FAB24518
S21444FD2002FA01F200FA01F308D9A6190EF1FF30DF
S21444FD3048D2B24546D9AEF1020E2644A6EB0A0690
S21444FD401FFA89F9B6FBFCF00CFB106649EA064636
S21444FD5000FB08F8B04507D9A61900F1FF3C2DD2A0
S21444FD60B0452BD90238264440EA0E40A6EB080696
S21444FD70A0FB02894E45C446CE4618D315D075B36B
S21444FD80B3EB0C0266EB0E0606FA07F722FA01F30B
S21444FD90CE401F43C5E90076002111E72946284690
S21444FDA00EE76646EDE6184601E74345E7D2B8EB6C
S21444FDB0020C69EB04040138A646E0E76046D3E744
S21444FDC060468CE78646B9E7614674E702383C44A9
S21444FDD02BE7084647E7ACF1020C3E4411E72946B8
S21444FDE0EEE600BF704700BF2DE9F04788B0002B11
S21444FDF01F461446B8BF03F10043129A109DDDF81F
S21444FE004CA0B6BF1F4600232D231370149B23F02B
S21444FE102008B8F1460F05D0B8F1450F00D101359A
S21444FE20022300E0032307AA049206AACDE902A20D
S21444FE30CDE9003522463B4601F0A6FDB8F1470F12
S21444FE40064602D1119BDB0722D5B8F1460F06EBD6
S21444FE50050910D13378302B0AD1002200232046DE
S21444FE603946FFF739FA18B9C5F10105CAF8005002
S21444FE70DAF8003099440022002320463946FFF73A
S21444FE802BFA08B1CDF81C903022079B4B4507D37C
S21444FE90079B159A9B1B3046136008B0BDE8F08755
S21444FEA0591C07911A70F0E7F7B503460029B8BF06
S21444FEB0494203F8022BB4BF2D222B220929427053
S21444FEC02ADD0DF10704A4460A27A6460A4691FBF6
S21444FED0F7F607FB16153035632A04F1FF340EF89F
S21444FEE0015C3146F1DC3031AEF1020504F8011C08
S21444FEF0441C294661450AD30DF10902A2EB0E02C1
S21444FF00654588BF00221344181A03B0F0BD11F8A3
S21444FF10012B04F8012FEDE7302330318370C17094
S21444FF20031DF1E72DE9F04F91B00C46DDF86880EB
S21444FF3016461F46054602F04DFE036809931846CA
S21444FF40FEF74AFD00230E93D8F800300A90073394
S21444FF5023F0070303F1080294F81890D4F800B08D
S21444FF60C8F80020D3E90023C4E91223D4E9128A4E
S21444FF702AF000430B930B999C4B4FF0FF324046BC
S21444FF80FFF7DCF970BB994B0B994FF0FF324046B4
S21444FF90FFF7B6F930BB0022002340465146FFF730
S21444FFA0A5F910B12D2384F84330914B9148B9F10B
S21444FFB0470F94BF98468046032323612BF00403DF
S21444FFC023604FF0000A009733460FAA214628467E
S21444FFD000F0D2F9013040F08F804FF0FF3011B07E
S21444FFE0BDE8F08F4246534640465146FFF7A6F9D1
S21444FFF040B1BAF1000FBCBF2D2384F843307E488D
S2144500007E4BD4E763685A1C09F0DF0142D10623CC
S2144500106360002206920EAACDE904920DAA4BF41F
S214450020806303920DF13302CDE9013223606368A4
S21445003000934246534628460B91FFF7D5FE0B994B
S214450040472980460D9908D1C81C02DB636899424A
S21445005040DDA9F102095FFA89F9B9F1650F1FD8A4
S21445006001394A4604F150000D91FFF71DFF0E9ADF
S2144500701318012A8246236102DC2268D20701D57D
S214450080013323619DF83330002B9CD02D2384F813
S214450090433098E74729BCD1002BBAD10123B7E7AF
S2144500A0B9F1660F18D1002963680BDD216113B9D4
S2144500B02268D00702D501330B442361A1654FF072
S2144500C0000ADFE713B92268D20701D50233F4E701
S2144500D00123F2E74FF067090E9B994205DB23683B
S2144500E02161D807EAD54B1CE7E70029D4BFC1F103
S2144500F0020201221344E0E723685A0507D4236920
S214450100424631462846B84701302BD165E7B9F116
S214450110650F40F2DC80D4E9120100220023FFF788
S214450120DBF8002833D0364A012331462846B847FF
S21445013001303FF452AFDDE90D239A4202DB2368D6
S214450140D8070FD5DDE9092331462846B84701309B
S2144501503FF443AF4FF0000804F11A090E9B013BEC
S214450160434509DC23689B0700F10181E0680F9B46
S2144501709842B8BF184632E701234A4631462846D4
S214450180B84701303FF429AF08F10108E6E70D9B73
S214450190002B37DC1A4A012331462846B84701303A
S2144501A03FF41BAFDDE90D23134302D12368D9077E
S2144501B0D8D5DDE9092331462846B84701303FF40E
S2144501C00CAF4FF0000904F11A0A0D9B5B424B45F4
S2144501D001DC0E9B94E70123524631462846B84734
S2144501E001303FF4FAAE09F10109EEE7FFFFEF7F74
S2144501F0AE844600B2844600BA844600B6844600BD
S214450200BE8446000E9AA36D9A42A8BF1A46002A97
S214450210914637DC4FF0000B29EAE97904F11A02DA
S214450220D4F858A0AAEB09035B4533DCDDE90D237A
S2144502309A423BDB2368DA0738D40E9A0D99A2EB2F
S2144502400A03A2EB01099945A8BF9946B9F1000FE3
S21445025034DC4FF0000829EAE97904F11A0ADDE9A9
S2144502600D239B1AA3EB090343457FF77BAF012379
S214450270524631462846B84701303FF4AEAE08F1FF
S2144502800108ECE71346314642462846B847013052
S214450290C0D1A2E60123314628460B92B847013025
S2144502A03FF49BAE0B9A0BF1010BB9E7DDE9092349
S2144502B031462846B8470130BFD18EE64B4608EB57
S2144502C00A0231462846B8470130C2D185E60E9A1D
S2144502D0012A01DCDB0737D501234246314628464D
S2144502E0B84701303FF479AEDDE909233146284663
S2144502F0B84701303FF471AED4E91201002200231D
S214450300FEF7EAFFD8B90E9B08F10102013B3146DC
S2144503102846B84701300ED15FE601234A463146A6
S2144503202846B84701303FF458AE08F101080E9B01
S214450330013B4345F1DC534604F15002E1E64FF0FC
S214450340000804F11A09F2E701234246DFE70123D4
S2144503504A4631462846B84701303FF43EAE08F196
S2144503600108E3680F995B1A4345F0DCFEE64FF05B
S214450370000804F11909F4E72DE9F04716469946B1
S2144503808A680B69DDF820809342B8BF1346336010
S21445039091F8432007460C460AB10133336023687B
S2144503A0990642BF336802333360256815F0060563
S2144503B006D104F1190AE36832689B1AAB4226DC7B
S2144503C094F84320131E226818BF012392062BD4A7
S2144503D004F1430249463846C04701301ED02368DB
S2144503E0E568326803F00603042B08BFAD1AA36818
S2144503F022690CBF25EAE57500259342C4BF9B1AC2
S214450400ED1800261A34B5421AD1002008E001231B
S214450410524649463846C047013003D14FF0FF3073
S214450420BDE8F0870135C6E7E1185A1C302081F84B
S2144504304300224494F8451082F843100233C7E738
S2144504400123224649463846C0470130E6D00136A4
S214450450D9E700002DE9FF470C469146277E0C99C3
S214450460782F80469A4604F1430207D8622F0AD869
S214450470002F00F0D880582F00F0A38004F14206E4
S21445048084F842703AE0A7F16303152BF6D801A02D
S21445049050F823F0ED044500010545007D04450070
S2144504A07D0445007D0445007D0445000105450065
S2144504B07D0445007D0445007D0445007D044500DA
S2144504C00D06450031054500EF0545007D04450010
S2144504D07D0445002F0645007D0445003105450051
S2144504E07D0445007D044500F70545000B681A1D4B
S2144504F01B680A6004F1420684F842300123A3E0F3
S214450500256808682E0600F104030AD505680B60C1
S214450510002D03DA2D236D4284F843305E480A23C6
S21445052019E015F0400F05680B6018BF2DB2EFE7D0
S2144505300B682568181D0860280601D51D6802E069
S2144505406906FBD51D8854486F2F0CBF08230A2320
S214450550002184F843106668A660002EA2BF216875
S21445056021F0040121600DB9002E4DD01646B5FB8D
S214450570F3F103FB1157C75D06F8017D2F46BB42D5
S2144505800D46F4D9082B0BD12368DF0708D5236918
S21445059061689942DEBF302306F8013C06F1FF3616
S2144505A0921B2261CDF800A04B4603AA2146404641
S2144505B0FFF7E2FE01304CD14FF0FF3004B0BDE806
S2144505C0F087354884F8457023680E681F0656F848
S2144505D0045B0E6014D5D90744BF43F0200323605F
S2144505E01DB9236823F0200323601023B0E7236852
S2144505F043F0200323607823284884F84530E3E712
S2144506005E0648BFADB2E6E71646BBE70B6826680A
S21445061060691D1D0D6035061B6801D5186002E032
S2144506207106FBD51880002323611646BAE70B688A
S2144506301A1D0A601E68626800213046FEF7D8F922
S21445064008B1801B606063682361002384F84330EB
S214450650A8E72369324649464046D0470130ABD0E5
S21445066023689B0713D4E068039B9842B8BF184697
S214450670A4E70123324649464046D04701309BD041
S2144506800135E36803995B1AAB42F2DCEBE70025DC
S21445069004F11906F5E700BFC0844600D18446003C
S2144506A02DE9F04F87B0174603938B685A1EB2F56F
S2144506B0AE7F83BF6FF4AE755B190293002386BF8A
S2144506C040F25D138B6002930B688B46002543F41E
S2144506D0F0634BF81C3BCDE9045580460C465E4618
S2144506E0AA46A9460195A26852B13B681B784E2B8F
S2144506F064D8402B3CD8A3F12B01C8B20E283AD972
S214450700B9F1000F03D0236823F4807323600AF100
S214450710FF3ABAF1010F00F213815E4500F20581FA
S2144507200125284607B0BDE8F08FA3F161020D2AE2
S214450730E6D801A151F822F07708450001074500A3
S2144507400107450001074500D7084500AF084500A5
S2144507500107450001074500850845000107450096
S2144507600107450001074500010745003D084500CE
S214450770A3F14102DBE70E29C2D801A050F821F0CB
S2144507802F084500010745002F084500C3084500CA
S21445079001074500DD0745001908450019084500CD
S2144507A01908450019084500190845001908450067
S2144507B01908450019084500190845006E2B09D843
S2144507C0602BB2D8542B77D0592B99D1072D97D17A
S2144507D0082529E0742B6FD0792BF6E72168C805E4
S2144507E01AD5029B21F08001216009F101091BB150
S2144507F0013B01320293A260A368013BA3602369D3
S214450800013323617B68013B002B7B6040F384808A
S2144508103B6801333B6066E71AEB050F7FF470AF24
S214450820226822F4C072226006F8013BE4E722689B
S21445083010067FF565AF22F08002F4E7BAF1000FA7
S2144508400ED1B9F1000F0ED1226802F4E061B1F580
S214450850E06F08D122F4F06222604FF0010AE3E728
S214450860BAF1020F55D0012D02D0042D7FF448AFC2
S2144508700135EDB2D8E7BAF1010F7FF441AF4FF03D
S214450880020AD1E77DB9B9F1000F7FF43CAF226883
S21445089002F4E061B1F5E06F7FF439AF22F4F0621F
S2144508A022600125C0E7032DE2D0052DDEE7022DA7
S2144508B07FF426AF0325B7E7062D7FF421AF07253E
S2144508C0B2E7226891057FF51BAF22F420722260BD
S2144508D0CDF80490A8E7226802F4A061B1F5806FD0
S2144508E006D050057FF50CAFB9F1000F3FF40FAFBA
S2144508F0910558BF019922F4F06258BFA9EB010152
S21445090042F4C07258BFCDE9041622604FF0000984
S2144509108AE74FF0030A87E7D4F8803139464046E0
S214450920984700283FF4DFAEEAE6D4F87C3116F85F
S214450930011D3A46404698472369013B2361ECE64C
S2144509406B1E062B25D8022D36D85E457FF6E8AEBB
S214450950D4F87C3116F8011D3A4640469847236937
S214450960013B2361F1E70298D4F87C3110F8011D6C
S21445097002903A46404698472369013B23610AF16F
S214450980FF3A5FFA8AFABAF1020FECD1033DEDB2AF
S214450990761B2368DA052FD55B0510D55E457FF6B1
S2144509A0BFAED4F87C3116F8011D3A464046984706
S2144509B02369013B2361F1E7AA460296DFE716F86D
S2144509C0011C2369652903F1FF3306F1FF352361D1
S2144509D00CD045290AD0D4F87C313A46404698474B
S2144509E0236916F8021C013BB51E2361D4F87C31F9
S2144509F03A46404698472E46256815F0100559D183
S214450A003570236803F4C063B3F5806F1CD1019B32
S214450A104B45A3EB090224D100225946404600F037
S214450A2083FED4F800C0039B1CF0020F1B680646E5
S214450A300F4621D003991A1D0A601B68C3E9006753
S214450A40E3680133E3606CE6049B002BE4D005992C
S214450A500A232A460131404600F0E6FE049B059EE1
S214450A60C21A04F26F139E4228BF04F5B7761249A0
S214450A70304600F029F8CFE71CF0040F03F1040ECA
S214450A8003D00399C1F800E0D7E7039AC2F800E01F
S214450A90D3F8008002460B46FEF750FC28B10748BF
S214450AA000F00EF8C8F80000CAE730463946FEF7AB
S214450AB0A3FCF7E7002534E6E2844600CC7F4600F3
S214450AC0004870470000C07F0EB400B59AB01BAB17
S214450AD0019005906FF00041094806910391094938
S214450AE053F8042B04910068009301A902F0E4FD35
S214450AF0019B00221A701AB05DF804EB03B07047EC
S214450B000C2340200802FFFF2DE9F0410F46904692
S214450B1002F084FB04460D46B8F1000F11D0C7F32A
S214450B200A53C3F16B03002B0BDD1B0503F17F5501
S214450B30002405F5401522462B46FEF765F9044682
S214450B400D4620462946BDE8F0810000000000001D
S214450B502DE9F04FA1B09B4600231C939E4B179260
S214450B601F68824638460E46FDF736FF4FF00008AA
S214450B7004464FF000091B961B9B1A782B2A4CD02F
S214450B803AD80D2A33D8082A33D8002A3DD0002330
S214450B900C931B9D2B78302B40F0A9806B7803F087
S214450BA0DF03582B66D10C9B01931CAB00938B4AF5
S214450BB0CDF808B01DAB1BA9504601F01FFD10F03F
S214450BC00706044605D0062E29D1013500231B9578
S214450BD00C93179B002B40F08E850C9BD3B1424659
S214450BE009F100431046194621B0BDE8F08F202A8A
S214450BF0CDD101331B93BFE72D2AC8D101220C92D4
S214450C005A1C1B925B78002BC3D1179B1B96002B57
S214450C1040F06F8542464B46E4E70022EFE71C9AD4
S214450C203AB135211EA802F0F0FB1C99504602F059
S214450C3031F8013E042E06D8DFE806F00A031417FD
S214450C400A00DDE91E892107C3D549F00049C0E7FA
S214450C50DDE91E831D9A23F4801302F2334243EAEC
S214450C600259F0E7DFF87891EDE76FF000494FF06D
S214450C70FF38E8E71B9B5A1C1B925B78302BF9D054
S214450C80002BA6D0012307931B9B08930023CDE991
S214450C9005339B460A221B980578A5F13003D9B241
S214450CA0092926D92246394602F01CFE002832D0AC
S214450CB000202B465C4604900246652B01D0452B0A
S214450CC013D11CB9079B03439FD000241B9E731C5E
S214450CD01B9373782B2B78D02D2B7BD00027A3F135
S214450CE03001092940F282801B9600259EE00023AC
S214450CF0C9E7BBF1080FD5BF0699059902FB013335
S214450D0002FB013300F10100D4BF069305930BF1B6
S214450D10010B1B90BFE71B9B1A191B921B5DBBF172
S214450D20000F36D004905C46A3F13002092A12D94A
S214450D300122C2E71B9B5A1C1B925B780130302B65
S214450D40F8D0A3F13102082A00F2DA841B9A0490FF
S214450D50002008920446303B00F1010213D0049966
S214450D6011440491224605190A21954213D12218A9
S214450D70082A04F1010404441BDC06990A2202FBF6
S214450D800133069300221B9B591C1B915B7810462A
S214450D90CAE75846D3E7082A04DC069F4F4306971A
S214450DA00132E2E7571C102FDEBF059F4F430597DC
S214450DB0F6E7102CDFBF05990A2202FB013305939F
S214450DC0E0E70023049301227CE70027B31C1B932E
S214450DD0B37884E70127F9E748864600E884460065
S214450DE00000F07F1B9B591C1B915B78302BF9D07C
S214450DF0A3F1310108293FF678AFA3F1300C1B9BD0
S214450E0009934FF00A0E1B9B591C1B915B78A3F167
S214450E103005092D35D9099D491B082944F61F6516
S214450E2002DC6545A8BF654607B16D42002C4CD12E
S214450E30079901437FF4CDAE002A7FF4E6AE692BD1
S214450E4026D023DC492B23D04E2B7FF4DEAE9C499F
S214450E501BA801F00FFE00283FF4D7AE1B9B1B785E
S214450E60282B2CD197491EAA1BA801F017FE05284A
S214450E7025D11F9BDDF8788043F0FF4949F4E0090A
S214450E80A7E60EFB0C3CACF1300CBCE76E2BDCE762
S214450E908D491BA801F0EEFD00283FF4B6AE1B9B1E
S214450EA08A49013B1BA81B9301F0E4FD10B91B9B27
S214450EB001331B93DFF824924FF0000889E68448F7
S214450EC002F00AFD8046894683E6049B0698EB1A9F
S214450ED0BBF1000F08BFA346102C07932646A8BFB4
S214450EE01026FDF717FF092C8046894613DD794BFA
S214450EF003EBC60353E91223FDF786FF80460598A4
S214450F008946FDF707FF02460B4640464946FDF72C
S214450F10C5FD804689460F2C36DC079B002B3FF4E3
S214450F2058AE22DD162B09DC6A4C04EBC304D4E923
S214450F30000142464B46FDF767FFC3E7079AC4F1F3
S214450F402503934220DB634DC4F10F0405EBC40132
S214450F5042464B46D1E90001FDF756FF079B1C1B51
S214450F6005EBC405D5E90023E5E7079B16330BDB00
S214450F70049B584A5D1B02EBC505D5E90023404650
S214450F804946FEF76BF89DE7079BA61B1E44002EB9
S214450F9071DD16F00F030AD04E4901EBC3014246F8
S214450FA04B46D1E90001FDF72FFF8046894636F0CE
S214450FB00F0650D0B6F59A7F27DD4FF0000BCDF8DB
S214450FC010B0CDF820B0CDF818B02223DFF80C913C
S214450FD0CAF800304FF00008089B002B3FF4F9ADE7
S214450FE01C99504601F056FE0699504601F052FEB1
S214450FF00499504601F04EFE0899504601F04AFEC7
S2144510005946504601F046FEE3E500233611404674
S21445101049461F46012E21DC0BB1804689462E4B9C
S214451020A9F1547903EBC70742464B46D7E9000179
S214451030FDF7EAFE294B0A460B4029498B42804676
S214451040BBD8A1F580118B4286BFDFF898904FF04C
S214451050FF3802F15479002305937EE0F20707D561
S2144510601D4B03EBC703D3E90023FDF7CDFE012354
S21445107001377610CEE7EED0764216F00F020AD04C
S214451080144B03EBC20340464946D3E90023FDF71C
S214451090E5FF804689463611DDD01F2E24DD4FF00C
S2144510A0000BCDF810B0CDF820B0CDF818B02223FF
S2144510B04FF000084FF00009CAF800308CE700BF33
S2144510C0BB844600FC844600B38446003C86460006
S2144510D0CC7F460088864600608646000000F07F46
S2144510E00000A07CFFFFEF7F16F0100318BF6A23B1
S2144510F0B34F0593404649460023F20704D5D7E942
S2144511000023FDF781FE0123761007F10807F4D189
S2144511100BB180468946059BBBB1C9F30A53C3F15B
S2144511206B03002B494610DD1F2B40F32881342BDB
S214451130DEBF203B4FF0FF3202FA03F34FF00008C4
S214451140CCBF4FF05C7903EA0109002200234046F4
S2144511504946FEF7C1F80028A1D1069B0093089999
S21445116023465A46504601F0EAFD089000283FF4CB
S21445117024AF049B5D1B079B002BB4BF2B46002367
S2144511800E93079B4FF0000B23EAE3731693CDF8B7
S21445119010B0089B5046596801F048FD0690002857
S2144511A03FF413AF089B1A69023203F10C01920013
S2144511B00C3001F02DFD1EAB01931DAB009342464E
S2144511C04B465046CDE90A8902F0A2F81C90002805
S2144511D03FF4FBAE0121504601F03DFE0490034628
S2144511E000283FF4F2AE1D9D1E9A002DABBF0E9B08
S2144511F0169B169C0E9EACBFEE185C1B059BED1A07
S2144512001544704B013D9D42C2F1360280F2C980BD
S2144512105B1B1F2BA2EB03024FF0010700F3B680C2
S21445122007FA03F30F930025B718059BBE421444EF
S2144512301C443346A8BF3B46A342A8BF2346002BC3
S214451240C2BFFF1AE41AF61A0E9B002B17DD049947
S2144512501A46504601F0A4FE049000283FF4B5AE69
S21445126001461C9A504601F0FFFD099000283FF4C0
S214451270ACAE1C99504601F00DFD099B1C93002F02
S21445128000F39380079B002B08DD169A0699504677
S21445129001F086FE069000283FF497AE002C08DD48
S2144512A006992246504601F0C9FE069000283FF4AE
S2144512B08CAE002E08DD04993246504601F0BEFE3F
S2144512C0049000283FF481AE069A1C99504601F0DA
S2144512D02FFF834600283FF478AE0024C368049960
S2144512E0C4600D9301F009FFA04271DA0D9B53EAE5
S2144512F0080340F09780C9F31303002B40F0928013
S21445130029F000431B0D1B05B3F1D66F40F28A80CA
S214451310DBF8143023B9DBF81030012B40F382801C
S21445132059460122504601F089FE0499834601F04C
S214451330E4FE002876DD0599234A4B46002900F051
S214451340928002EA0901B1F1D66F00F38C80B1F1C3
S2144513505C7F7FF7ACAE1D4A0023CDE9143240468C
S214451360DDE914234946FDF74FFD0B46034308BF09
S21445137022238046894608BFCAF8003030E64FF03B
S214451380FF3202FA03F303EA0808DEE6C5F17F45B5
S21445139005F57F0505F57B45E23507FA05F50F9713
S2144513A042E7012300250F933EE71C993A465046EF
S2144513B001F044FE1C9000287FF464AF05E600BFAC
S2144513C01085460002FCFFFF0000F07F0000503904
S2144513D0CDF8249066D10D9AC9F313035AB39C4AA7
S2144513E093422CD1059B404603B39A4A4B461A4036
S2144513F0B2F1D46F4FF0FF311BD8120DC2F16B031B
S21445140001FA03F398421AD1934B099A9A4202D1AC
S21445141001303FF4DAAD8F4B099A1A4002F5801930
S2144514204FF00008059B002B95D1D9E54FF0FF33CB
S214451430E8E70B46E6E753EA08033FF47CAFE5B139
S214451440099B1D42EED00D9B059A40464946C3B1C1
S214451450FFF75AFB02460B46DDE90A01FDF71EFB80
S21445146080468946DEE71340A3F580136FEA135995
S2144514706FEA09594FF0FF38D4E70F9B13EA080F78
S214451480E0E7FFF741FB02460B46DDE90A01FDF7BB
S21445149003FB0022002380468946FDF71DFF0028F2
S2144514A0C0D004E60499584601F081FF00224FF06B
S2144514B0804306460F46FDF723FF002875D00D9B53
S2144514C0002B47D0654F0026644D099B23F000430B
S2144514D01B0D1B050F930F9A614B9A4240F0C8802F
S2144514E0DDE90A23CDE91423099BA3F15479404647
S2144514F0494601F093FE02460B4630463946FDF70F
S21445150083FC42464B46FDF7C9FA0B465149554AB8
S2144515101940914280465ED90B9B02F15472934224
S21445152003D10A9B01333FF450ADDFF82C914FF0C1
S214451530FF381C99504601F0ADFB0699504601F020
S214451540A9FB0499504601F0A5FB5946504601F0C3
S214451550A1FB1EE6B8F1000F19D1099BC3F313038F
S214451560E3B93E4B002230463946FDF7BFFEC8B9C3
S2144515703D4B002230463946FDF746FC04460D46AF
S21445158005F1004318941993DDE918679DE7B8F10E
S214451590010F03D1099B002B3FF489AD334F00263D
S2144515A0002491E70D9C304DEAE72F4B002230464C
S2144515B03946FDF729FC0D9B04460D4633B901F126
S2144515C0004310901193DDE910677EE702460B460F
S2144515D0CDE91023F7E703F15479059B002BA8D1F5
S2144515E029F000430F9A1B0D1B059A42A1D12046B0
S2144515F02946FEF75DFAFDF7D9FB02460B4620461F
S2144516002946FDF749FA0D9AC9F3130343EA080339
S214451610134304460D4666D009A3D3E90023FDF7D8
S21445162065FE00287FF4DCAC07A3D3E900232046FB
S2144516302946FDF779FE00283FF47BAFD0E400BF8E
S2144516409535A094FFFFDF3F35E5AF350000E03F19
S214451650FFFF0F000000F07FFFFFEF7F0000F03F29
S2144516600000E07FFFFF9F7C0000E03F0000F0BFEA
S214451670059B13B30F9BB3F1D46F1ED826A3D3E9AE
S214451680002320462946FDF73BFE90B129462046D5
S214451690FDF792FE012838BF0120FDF73BFB0D9B69
S2144516A004460D46D3B901F1004312901393DDE984
S2144516B012670F9A07F1D6639F1ADDE90A0101F012
S2144516C0ADFD02460B4630463946FDF79DFBDDE946
S2144516D00A23FDF7E3F9804689467EE702460B4630
S2144516E0CDE91223E3E70EA3D3E90023FDF7FEFD7C
S2144516F0A1E700230C93179A1B9B1360FFF76DBA5F
S214451700652B3FF45EAB452B3FF45BAB0122FFF701
S2144517108FBB00BFAFF300800000C0FFFFFFDF4177
S2144517209535A094FFFFCF3F014BFFF711BA00BF99
S214451730742340202DE9F0473A4E86468C4660464F
S2144517401CF8014BA55D15F00805F8D12D2C33D1B5
S2144517509CF800404FF0010800F1020C002B5CD0CD
S214451760102B0CD1302C0AD19CF8000000F0DF007D
S21445177058284DD19CF8014010230CF1020C08F175
S2144517800047013F0026B7FBF3F9304603FB197ABD
S214451790A4F13005092D18D82C46A34224DD751C26
S2144517A007D081451DD301D1A2451ADB00FB034076
S2144517B001261CF8014BEBE72B2C08BF9CF8004094
S2144517C0A84608BF00F1020CC8E7A4F14105192D4B
S2144517D001D8373CE1E7A4F16105192D04D8573CFB
S2144517E0DBE74FF0FF36E4E7731C06D12223CEF83D
S2144517F00030384642B9BDE8F087B8F1000F00D052
S2144518004042002AF7D00EB10CF1FF311160F2E7E5
S2144518103024002BB3D10823B1E7302CA4D00A23BB
S214451820ADE700BF39854600FFF784BF00B59BB0DE
S214451830019105916FF00041069103910549049188
S21445184001A901F039FF019B00221A701BB05DF813
S21445185004FB00BF0802FFFF13460A46014602483E
S2144518600068FFF7E3BF00BF0C2340202DE9F74F84
S21445187003690C69A3420746C0F28180013C01F129
S214451880140800F1140505EB8403019358F8243039
S21445189055F8242001339A424FEA840B08EB840915
S2144518A0B2FBF3F631D34FF0000E4046AC46F24657
S2144518B050F8042B93B206FB03E34FEA134E9BB254
S2144518C0AAEB0303120CDCF800A006FB02E213FAAF
S2144518D08AF34FEA124E1FFA82FADCF80020CAEB6A
S2144518E0124202EB23429BB243EA024381454CF83F
S2144518F0043B4FEA224ADBD255F80B302BB9019B05
S214451900043B9D421A462ED33C61384601F0F5FB12
S214451910002824DB013628464FF0000C58F8042BE7
S214451920D0F800E093B2ACEB0303120C13FA8EF337
S214451930C2EB1E4202EB23429BB243EA0243C14539
S21445194040F8043B4FEA224CE8D255F8242005EBF4
S214451950840322B9043B9D421A460AD33C6130466D
S21445196003B0BDE8F08F1268043B002ACCD1013C99
S214451970C7E71268043B002AF0D1013CEBE700209C
S214451980EEE70000000000002DE9F04F446A99B0EC
S21445199016461F46CDE90467DDF8948005463CB9F2
S2144519A0102001F01BF9C0E9014468620460C46078
S2144519B06B6A196851B15A684A60012393408B6037
S2144519C0284601F067F96B6A00221A603B1EB9BFCC
S2144519D023F0004305930023C8F80030DDF8149043
S2144519E0A74BBCBF0122C8F8002033EA090319D12A
S2144519F0249A42F20F731360C9F31303334300F07E
S214451A006D85269B53B99F4B23E09F4B0393083325
S214451A10269A1360039819B0BDE8F08F994B039347
S214451A200333F5E7DDE90434CDE90C34DDE90C0193
S214451A3000220023FDF750FC804660B1249A01231E
S214451A401360269B002B00F04685904B269A136024
S214451A50013B0393DEE716AB019317AB009328468D
S214451A60DDE90C2301F054FCC9F30A548346002CE7
S214451A707ED00D9BCDF84C80C3F31303DDE90C01F6
S214451A8043F07F5141F44011A4F2FF34804B0022CD
S214451A90FDF702F874A3D3E90023FDF7B5F974A35F
S214451AA0D3E90023FCF7FAFF064620460F46FDF726
S214451AB041F971A3D3E90023FDF7A6F902460B4683
S214451AC030463946FCF7EAFF06460F46FDF74CFC1E
S214451AD000228246002330463946FDF707FC48B1CA
S214451AE05046FDF727F932463B46FDF7F5FB08B964
S214451AF00AF1FF3ABAF1160F57D8664B03EBCA03FD
S214451B00D3E90023DDE90C01FDF7F0FB00284ED0B4
S214451B100AF1FF3A00230F93169B1C1B631E09937D
S214451B2045BFC4F101030693002300234CBF099328
S214451B300693BAF1000F3CDB099BCDF838A0534419
S214451B40099300230A93229B092B00F2B580052BA7
S214451B50C4BF043B2293229BA3F10203CCBF0024BF
S214451B600124032B00F2B480DFE803F02D987AA415
S214451B70DDE916431C4404F23243202BC3BFC3F1B0
S214451B80400304F2124009FA03F3C3F12003C6BF2B
S214451B9026FA00F0184306FA03F0FDF7BBF80123D2
S214451BA0A1F1F871013C139370E70123B3E70F9059
S214451BB0B2E7069BA3EB0A030693CAF100030A9312
S214451BC000230E93BFE700230B93239B002B00F3C4
S214451BD082804FF00109CDF820904B46CDF88C9089
S214451BE06E6A00227260042202F1140098427168FF
S214451BF077D9284601F01AF86B6A30601B6803935C
S214451C00089B0E2B00F2EE80002C00F0EB80BAF11C
S214451C10000F7ADD1F4A0AF00F0302EBC303D3E930
S214451C2000341AF4807FCDE910344FEA2A145CD08C
S214451C30194BDDE90C01D3E90823FDF70FFACDE989
S214451C40040104F00F040327134E002C4FD1DDE9A1
S214451C501023DDE90401FDF701FACDE904016EE044
S214451C600123B1E7AFF3008061436F63A787D23F97
S214451C70B3C8608B288AC63FFB799F501344D33F31
S214451C800000F07F4286460039864600BF844600FF
S214451C900000F83F888646006086460000230B9382
S214451CA0239B0AEB030909F10103012B0893B8BFEF
S214451CB0012395E70123F2E70124002322930B94A1
S214451CC04FF0FF390022CDF820901223239287E764
S214451CD001230B93F4E7DDF88C90CDF820904B4626
S214451CE07EE70131716052007EE70227ACE7E107E7
S214451CF008D5DDE91001D6E90023FDF785F8CDE9DD
S214451D0010010137641008369FE700F0A580CAF138
S214451D100004A44BA44E04F00F0203EBC203D3E920
S214451D200023DDE90C01FDF76FF8CDE90401241128
S214451D3000230227002C40F08480002B8DD10F9B7A
S214451D40002B00F08B80DDE90434CDE91034DDE965
S214451D501001964B0022FDF7C9FA00287ED0089B55
S214451D60002B7BD0B9F1000F38DDDDE91001904B33
S214451D700022FDF749F8CDE904010AF1FF3801379D
S214451D804C463846FCF7D6FFDDE90423FDF73CF81C
S214451D90884B0022FCF782FEA1F15076CDE9100172
S214451DA01196002C5DD1DDE90401834B0022FCF73A
S214451DB073FE02460B46CDE90423109A3346FDF7DB
S214451DC0B3FA002840F09782DDE90401109A06F13F
S214451DD00043FDF78BFA002840F08B82DDE90C3492
S214451DE0CDE90434179B002BC0F25181BAF10E0F92
S214451DF000F34D816B4B03EBCA03D3E90034CDE9C1
S214451E000634239B002B80F2DB80089B002B00F3D7
S214451E10D78040F06D82684B0022DDE90601FCF76D
S214451E20F3FFDDE90423FDF775FA089C26460028EE
S214451E3040F04382039F312307F8013B0AF1010A2C
S214451E403FE2E20705D5D6E90023FCF7DDFF01377B
S214451E500123641008366DE7022770E7089CD046D4
S214451E608FE703994F4B214412910B9903EBC4031B
S214451E70DDE9106753E90223002946D04F49002083
S214451E80FDF7ECF83B463246FCF706FECDE9100179
S214451E90039FDDE90401FDF767FA0446FCF74AFFB0
S214451EA002460B46DDE90401FCF7F6FD30340246F2
S214451EB00B46CDE9042307F8014BDDE91023FDF772
S214451EC015FA002865D1DDE9042338490020FCF7DA
S214451ED0E3FDDDE91023FDF709FA002840F0B6805A
S214451EE0129B9F423FF47AAFDDE91001304B00224A
S214451EF0FCF78AFF2E4BCDE910010022DDE90401EF
S214451F00FCF782FFCDE90401C3E730463946FCF7C6
S214451F107BFFCDE91001129B039C1493DDE9040178
S214451F20FDF722FA1590FCF705FF02460B46DDE95C
S214451F300401FCF7B1FD159B303304F8013B129BB9
S214451F409C4206460F464FF0000224D11B4BDDE966
S214451F501001FCF7A3FD02460B4630463946FDF711
S214451F60E3F9002871D1DDE9102314490020FCF778
S214451F7093FD02460B4630463946FDF7B7F900282D
S214451F803FF42CAF149F7B1E149317F8013C302B5F
S214451F90F8D0C24649E0064BFCF736FFCDE90401CA
S214451FA0BCE700BF88864600608646000000F03FD6
S214451FB00000244000001C40000014400000E03FA4
S214451FC0DDE90489039FDDE9062340464946FDF7DA
S214451FD045F8FDF7C9F90446FCF7ACFEDDE90623EE
S214451FE0FCF712FF04F130060B46024649464046CA
S214451FF0FCF752FD07F8016B039E089BBE1BB342D8
S21445200038D102460B46FCF749FDDDE906238046F6
S2144520108946FDF789F958BBDDE90623404649461A
S214452020FDF75AF908B1E10722D42846594600F08B
S21445203031FE00233B70249B0AF101001860269B65
S214452040002B3FF4E7AC1F60E4E427463B461F46BB
S21445205013F8012D392A07D1039A9A42F7D10399E5
S214452060302208F101080A701A7801321A7090E792
S214452070D046EBE7A14B0022FCF7C6FE0022002324
S21445208080468946FDF728F900289CD0CDE70B9A6F
S214452090002A00F0CD80229A012A00F3AF80139AD9
S2144520A0002A00F0A78003F233430A9C069F069A4F
S2144520B01A440692099A01211A442846099200F0C4
S2144520C0CAFE0646002F0CDD099B002B09DDBB42E8
S2144520D0069AA8BF3B46D21A0692099AFF1AD31A01
S2144520E009930A9BF3B10B9B002B00F0A580002CAF
S2144520F010DD31462246284600F052FF5A46014634
S2144521000646284600F0B0FE59468046284600F06A
S214452110C1FDC3460A9B1A1B04D05946284600F003
S2144521203FFF83460121284600F095FE0E9B002B77
S214452130044640F383801A460146284600F030FFA1
S214452140229B012B04467CDD4FF00008236904EBF7
S2144521508303186900F031FEC0F12000099B18443E
S21445216010F01F0000F08E80C0F12003042B40F3D2
S2144521708780C0F11C00069B03440693099B0344D5
S21445218007440993069B002B05DD59461A46284603
S21445219000F054FF8346099B002B05DD21461A4671
S2144521A0284600F04BFF04460F9B002B6CD021467B
S2144521B0584600F0A2FF002866DA002359460A2250
S2144521C0284600F07EFD0B9B0AF1FF3A8346002B1E
S2144521D000F08B81314600230A22284600F071FD27
S2144521E0B9F1000F064600F39180229B022B40F37F
S2144521F08D8051E0169BC3F1360356E7089B5C1E5F
S2144522000A9BA342BFBF0A9B0A94E21A0E9BB6BF1F
S2144522109B181C1B0E93089BB8BF0024002BB9BF08
S214452220069B089A069F089BBCBF9F1A00233EE75D
S2144522300A9C069F0B9E45E70A9A6EE7229B012B52
S21445224019DC049BBBB9059BC3F313039BB9059BDC
S21445225023F000431B0D1B0583B1069B01330693F4
S214452260099B013309934FF001080E9B002B7FF421
S2144522706DAF012072E74FF00008F6E79846F4E7A1
S21445228080D018461C3076E7089B002B38DC229B0E
S214452290022B35DDDDF82090B9F1000F0DD1214632
S2144522A04B460522284600F00CFD01460446584696
S2144522B000F023FF00283FF7BDAD239B039F6FEA41
S2144522C0030A4FF000082146284600F0E3FC002E9E
S2144522D03FF4ABAEB8F1000F05D0B04503D041464C
S2144522E0284600F0D7FC3146284600F0D3FC9CE64D
S2144522F000242646E1E7C24626469BE500002440E4
S2144523000B9BDDF82090002B00F0F680002F05DDB6
S21445231031463A46284600F091FE0646B8F1000F8B
S21445232055D07168284600F081FC3269023207466E
S214452330920006F10C010C3000F06AFC0122394689
S214452340284600F07BFE039B01330893039B4B44D2
S2144523500A93049B03F00103B04609930646089B7F
S2144523602146013B58460493FFF780FA034630332F
S2144523700690414658460B9300F0BFFE32468146CE
S2144523802146284600F0D4FEC2680B9B074602BB92
S2144523900146584600F0B1FE0B9B02463946284694
S2144523A0CDE90B3200F076FC229B0C9A089F43EA57
S2144523B00201099B0B430B9B0DD1392B29D0B9F153
S2144523C0000F01DD069B3133049A13707BE73046D8
S2144523D0B9E70122E2E7B9F1000F06DB229941EAA7
S2144523E00909099959EA010120D1002AECDD594627
S2144523F001222846089300F021FE2146834600F038
S2144524007CFE0028089B02DCDED1DA07DCD5392BBA
S214452410D8D1049A392313703B461F46013B17F81B
S214452420012C392A50D001321A704CE7002A03DDB8
S214452430392BEED00133C7E7089A0A9902F8013CD2
S2144524408A422AD0594600230A22284600F039FCFB
S214452450B04583464FF000034FF00A0241462846F2
S21445246007D100F02EFC80460646089B01330893AC
S21445247075E700F026FC3146804600230A222846AA
S21445248000F01FFC0646F0E7B9F1000F039ACCBFF3
S2144524904F46012717444FF0000859460122284663
S2144524A0089300F0CBFD2146834600F026FE002823
S2144524B0B2DC02D1089BDB07AED43B461F4613F879
S2144524C0012D302AFAD0FEE6039A9A42A5D10AF1A2
S2144524D0010A312379E7134BFFF7BBBA269B002B3E
S2144524E07FF493AA104BFFF7B4BAB9F1000F03DC9B
S2144524F0229B022B3FF7D0AE039F21465846FFF757
S214452500B5F900F1300307F8013B039ABA1A91452D
S214452510BADD594600230A22284600F0D2FB8346F8
S214452520EBE700BFBE844600398646000369B3EB39
S214452530611F2DE9F0434FEA611200F1140445DDB1
S21445254011F01F0104EB830604EB82050CD100F164
S21445255010072946B14234D39B1A9B00EA1E964281
S21445256038BF0023234415E054F82270C1F12008F3
S214452570CF4005F1040EA1467645F44615D89B1A7C
S2144525809A00043A0135AE4238BF0022A318A75038
S21445259007B104331A1BA3424FEAA20208BF002321
S2144525A0026108BF4361BDE8F083DCF800C00CFA61
S2144525B008FC4CEA070749F8047B5EF8047BCF40E5
S2144525C0DAE751F804CB47F804CFC3E72346E1E7FB
S2144525D0A0F13003092B02D82038C0B27047A0F1CD
S2144525E06103052B01D84738F7E7A0F14103052BD2
S2144525F001D82738F1E70020704700002DE9F04F55
S2144526008BB08B460693BA4B02901B6803931846CD
S2144526109046FCF7E1F9039BDBF80020034482462D
S21445262013F8013C0793931CC2F1FF2202F57F0283
S214452630FE32D1181F4613F8010B01913028F8D009
S214452640FFF7C6FF044600283AD103995246384656
S21445265001F048F90546002866D117F80A0007EB49
S2144526600A06FFF7B5FF002860D0334618783028AD
S2144526701F4603F10103F9D0FFF7AAFF0123B0FA7D
S21445268080F46409354601933A4616460132307859
S214452690FFF79EFF0028F8D103995246304601F0D1
S2144526A021F980B94DB906EB0A052A461646013288
S2144526B03078FFF78DFF0028F8D1AD1BAD0004E05C
S2144526C000242546E0E7002DF7D1337803F0DF03F5
S2144526D0502B39D173782B2B2AD02D2B2CD0711C0F
S2144526E04FF000090878FFF773FF431EDBB2182B3F
S2144526F02AD8A0F1100211F8010FFFF769FF431E13
S214452700DBB2182B1BD9B9F1000F00D05242154445
S214452710CBF80010D4B1019B002B14BF0027062729
S21445272038460BB0BDE8F08F3E4625460124CCE73B
S2144527304FF00009B11CD5E74FF00109FAE70A2327
S21445274003FB0202103AD6E73146E1E7F31B013BAD
S2144527502146072B50DC029800F068FA4FF0000B34
S21445276000F11409CAF101030446CDF81090CDF8DE
S21445277004B00893B74242D3049F019B47F8043BF5
S214452780A7EB0907BF102761184600F016FB7F0127
S214452790D8F800603F1AB74265DDBF1B394620466C
S2144527A000F056FE8246A8B17B1E591103F01F0263
S2144527B059F821104FF0010A0AFA02F20A4209D0E6
S2144527C0534505DDB91E204600F042FE002847D198
S2144527D04FF0020A39462046FFF7A8FE3D44D8F892
S2144527E00830AB424DDA0298214600F053FA149A67
S2144527F000231360A32793E701315B10A9E7731EF7
S214452800079A059316F8013C934219D0BBF1200F61
S21445281007D1049B019A43F8042B049300230193A4
S2144528209B4616F8010CFFF7D3FE019B00F00F0000
S21445283000FA0BF0034301930BF1040B059B0DE0E7
S214452840059B089A1344BB42E0D31846039909935F
S214452850524601F047F8099B0028D7D11E4689E71E
